:10000300E5E07E5009D3C2CF30CFFDD3C297C2CF34
:100013001330CFFD9297C2CFA5DDF530CFFD30CFA2
:10002300FD22E5E07E5009D3C2CF30CFFDD3C29588
:10003300C2CF1330CFFD9295C2CFA5DDF530CFFDF2
:1000430030CFFD22E5E07E5009D3C2CF30CFFDD3C0
:10005300C297C2CF1330CFFD9297C2CFA5DDF53043
:10006300CFFD30CFFD12006C227E60047E50AA00CB
:10007300000000A5DDF9A5DEF3227E50AA000000F2
:0800830000A5DDF9D5E0F32230
:02FFF800BFFF49
:10D6ED00436F6D6D616E64206572726F72202020C4
:02D6FD0000002B
:10D6FF00436F6D6D616E64206572726F72200D0ADB
:01D70F000019
:10D710000D0A436F6D6D616E643A4D557878782CC3
:10D720004D447878782C46557878782C464478782B
:10D73000782C415A7878785F454C78782C537878F3
:0FD74000782C5478782C3F412C3F2C510D0A0047
:10D74F00547261636B2023204572726F7220210D1A
:02D75F000A00BE
:10D76100415A5F666F726D6174206572726F7220CB
:02D771000000B6
:10D77300417A2F456C20666F726D617420657272F9
:10D783006F72202865782E20417A30373520456C1A
:06D793003135290D0A00EA
:10D799004D5F666F726D6174206572726F722000E1
:01D7A900007F
:10D7AA004D6F646520466F726D6174206572726F89
:10D7BA0072202865782E204D554C53422C4D4446F4
:05D7CA004D290D0A00CD
:10D7CF004D6F6465206572726F72202865782E2008
:0FD7DF004D444C2F4D44552F4D4446290D0A0003
:10D7EE004D6F6465206572726F72202865782E20E9
:0FD7FE004D554C2F4D55552F4D5546290D0A00B1
:10D80D004D6F6465206572726F722020202020009C
:01D81D00000A
:10D81E00465F666F726D6174206572726F72200062
:01D82E0000F9
:10D82F00467265712E20666F726D6174206572721B
:10D83F006F722021202865782E20465531343539D6
:08D84F0030303030290D0A00D1
:10D8570046445F2020202020202020202020202038
:02D867000000BF
:10D8690046555F2020202020202020202020202015
:02D879000000AD
:06D87B0025732025730057
:0DD881000D0A5472616B426F783E3E20002C
:10D88E00202020202020202020202020202020208A
:02D89E00000088
:10D8A0005472616B426F7820486F73746D6F64655A
:02D8B000000076
:10D8B2000D0A436F6D6D616E643A4D557878782C20
:10D8C2004D447878782C46557878782C4644787888
:10D8D200782C415A7878785F454C78782C53787850
:0FD8E200782C5478782C512C3F412C3F0D0A00A4
:10D8F1000D0A0D0A5472616B426F7820686F737460
:07D90100206D6F64652E002C
:10D90800070D0A094572726F722021212075706413
:10D91800617465206E6F7420636F6D706C657465DB
:05D92800642E0D0A0051
:10D92D000D0A0953746174696F6E20696E666F72AA
:10D93D006D6174696F6E20757064617465642E0D10
:02D94D000A00CE
:10D94F00252A63202573202566202566202566203D
:03D95F002566003A
:10D96200252A63202573202566202566202573201D
:09D97200257320256420256400C2
:10D97B00252A632025732025662025662025662011
:06D98B0025662025660060
:10D99100252A63202573202573202562782025629E
:09D9A10078202564202562640051
:10D9AA00252A63202566202566202566202566000F
:10D9BA00252A6320256420256420256420256420E7
:03D9CA00257300C2
:10D9CD00252A6320257320256C6620256C6620256D
:06D9DD006C6620257300BA
:10D9E3000D0A0D0A0955706C6F61642053746174DC
:10D9F300696F6E20696E666F2E20646174612066A4
:10DA0300696C652E2028454F463A6374726C2B5A15
:04DA1300290D0A00CF
:10DA1700536174656C6C69746520282538732920F7
:10DA27007570646174656420616E642073656C65EC
:10DA3700637465642061732023253262640D0A00D4
:10DA47002573202573202573202573202573202512
:08DA57007320257320257300E4
:10DA5F000D0A0A0955706C6F616420667265712F2B
:10DA6F006D6F646520646174612066696C652E203A
:0FDA7F0028454F463A6374726C2B5A290D0A00E2
:03DA8E0020000075
:10DA91000D0A0907536174656C6C697465206973BB
:10DAA100206E6F7420617369676E65642E20476F05
:0FDAB10020746F206D656E7520332D320D0A00C5
:08DAC00020202020202020007E
:0DDAC8002532642E2563252D313473200096
:04DAD5000D0A0A002C
:0BDAD9000D0A0953656C6563743A0088
:0CDAE4002532642E20252D3134732000E3
:0CDAF0002532642E2A252D3134732000CD
:10DAFC000D0A09536174656C6C6974652028257373
:10DB0C00292073656C65637465642061732023251B
:05DB1C0062640D0A0027
:0FDB21004E4153413E232533640925730D0A00FD
:10DB3000070D0A09525320427566666572204675C4
:07DB40006C6C20210D0A00AE
:10DB47000D0A0A0955706C6F6164204B6570656C2E
:10DB57006520646174612066696C652E2028454FD5
:0CDB6700463A6374726C2B5A290D0A00B8
:10DB7300092D2D2D2027512720666F722061626F9A
:10DB830072742027532720666F72207363726F6C41
:06DB93006C202D2D2D0079
:0DDB99002A2A2A2A2A2A2A2A2A2A0A0D00C4
:10DBA60025352E31662F25342E316625392E3166E0
:09DBB600252B392E30660D0A0002
:10DBBF002025303262643A25303262643A253032A1
:07DBCF006264202020200009
:10DBD6002534642F25303262642F2530326264206A
:01DBE600003E
:08DBE700446F70706C65720060
:06DBEF005068617365003F
:03DBF500454C009C
:03DBF800415A008F
:05DBFB0054494D4500F6
:05DC0000444154450001
:10DC05002020253573202020202535732020202035
:10DC150020202025337320202F253373202020201A
:0BDC250020253573253130730D0A00F7
:0BDC300009536563205B305D3A200063
:0BDC3B00094D696E205B315D3A20004E
:0CDC460054696D6520537465700D0A0070
:10DC5200446179206F66207468652059656172207D
:0EDC62005B545D203E2025352E38660D0A00ED
:10DC70005374617274696E67204461792F54696DC1
:10DC800065203F205B59592F4D4D2F444420484873
:09DC90003A4D4D3A53535D20005A
:10DC99000D0A2534642F25303262752F2530326202
:10DCA900752025303262753A25303262753A253051
:06DCB9003262750D0A0045
:10DCBF000D0A0909507265737320616E79206B65C7
:0EDCCF007920746F20636F6E74696E75650046
:10DCDD000D0A09434F4D20706F72742020202020B3
:10DCED0020202020202573204261756420382D4E80
:05DCFD002D310D0A00AD
:10DD02000D0A09526F746F7220737461727420204D
:08DD12002020202020257300D1
:04DD1A00202573004D
:08DD1E0028773D25626429000D
:06DD2600282542582900E7
:08DD2C0020202825425829009F
:0DDD34002020464D4E2D46696C746572002E
:09DD4100202046542D383437002F
:09DD4A00202046542D3733360029
:0CDD5300202054533731312F383131007B
:10DD5F000943415420526967202020202020202091
:09DD6F00202020257320257300FB
:10DD7800094175746F207265636F766572792074D6
:10DD8800696D652066726F6D20726F7461746F7251
:10DD9800206572726F723A20253364206D696E0DAA
:02DDA8000A006F
:10DDAA000954696D656F75742076616C75652066B6
:10DDBA006F7220726F7461746F72206572726F7203
:0CDDCA003A20253364207365630D0A00C5
:10DDD60009526F746F7220736D6F6B652070726F6E
:0EDDE60074656374696F6E094F66660D0A00FE
:10DDF40009526F7461746F72207374617274204578
:10DE04004C3A25352E316620202050312E365F6F56
:10DE14006E20454C3A25352E316620202050312E77
:10DE2400365F6F666620454C3A25352E3166200DE7
:02DE34000A00E2
:10DE360009526F7461746F72206C696D6974202069
:09DE46002020204F66660D0A0041
:10DE4F0009526F7461746F72206C696D6974202050
:10DE5F00202020415A3A2025352E3166202D2025AD
:10DE6F00352E31662020454C3A2025352E3166203F
:0BDE7F002D2025352E3166200D0A00F5
:10DE8A0009416E74656E6E61207061726B696E67AE
:09DE9A002020204F66660D0A00ED
:10DEA3000954525820207061726B696E67202020DC
:09DEB3002020204F66660D0A00D4
:10DEBC0009545258207061726B696E672020205291
:10DECC00583A25362E33662054583A25362E33666A
:10DEDC00202020205258206D6F64653A2573205401
:0CDEEC0058206D6F64653A25730D0A0024
:10DEF80009416E74656E6E61207061726B696E6740
:10DF0800202020415A3A2025352E31662020202015
:10DF1800202020202020454C3A2025352E3166200F
:03DF28000D0A00DF
:10DF2B0009536B65772020202020202020202020E3
:10DF3B00202020415A3A2025352E316620202020E2
:10DF4B00202020202020454C3A2025352E316620DC
:03DF5B000D0A00AC
:10DF5E0009446561642062616E64202020202020C7
:10DF6E00202020415A3A2025352E316620202020AF
:10DF7E00202020202020454C3A2025352E316620A9
:03DF8E000D0A0079
:07DF910028466C69702900AD
:10DF980009414443207370616E2076616C75652079
:10DFA800202020415A3A20253564202D202535642B
:10DFB8002020454C3A20253564202D202535642025
:01DFC8000058
:10DFC9000943616C6C7369676E3A20257320204C94
:10DFD90061743A2025352E316620204C6F6E673AE0
:10DFE9002025352E316620204865696768743A20F6
:08DFF90025352E31660D0A00EA
:05E0010046756C6C0087
:04E00600414F530033
:03E00A00464D0080
:03E00D0043570076
:04E010005553420022
:04E014004C53420027
:06E0180049434F4D2000BA
:08E01E00594145535520200033
:08E026004B454E574F4F4400DB
:10E02E0009456C65766174696F6E20536B65772058
:0EE03E0076616C7565203A2025322E31660021
:10E04C000D0A09417A696D757468202020536B653F
:10E05C00772076616C7565203A2025322E3166006A
:10E06C0009456C65766174696F6E20446561642046
:0EE07C0042616E6420203A2025322E3166006B
:10E08A000D0A0D0A09417A696D75746820202044C9
:10E09A006561642042616E6420203A2025322E3167
:02E0AA0066000E
:10E0AC000D0A094175746F207265636F766572791C
:10E0BC002074696D652066726F6D20726F74617467
:10E0CC006F72206572726F72205B312D36316D6903
:09E0DC006E5D203A20253364003A
:10E0E5000D0A0954696D656F75742076616C7565E7
:10E0F50020666F7220726F7461746F722065727220
:0FE105006F72205B7365635D203A2025336400E1
:10E114000D0A0953657420726F7461746F722073F1
:10E124006D6F6B652070726F74656374696F6E20B8
:0AE134003F205B592F4E5D202000B4
:10E13E0009456C65766174696F6E206D6178696DE5
:10E14E00756D2076616C7565203A2025332E31660B
:01E15E0000C0
:10E15F0009456C65766174696F6E20206D696E6D0F
:10E16F00756D2076616C7565203A2025332E3166EA
:01E17F00009F
:10E1800009417A696D75746820206D6178696D75D3
:10E190006D202076616C7565203A2025332E31661E
:01E1A000007E
:10E1A1000D0A0D0A09417A696D7574682020206D88
:10E1B100696E6D756D202076616C7565203A20253C
:05E1C100332E31660061
:10E1C6000D0A0953657420416E74656E6E61207286
:10E1D6006F746174696F6E206C696D6974203F207D
:08E1E6005B592F4E5D20200063
:10E1EE00095458207061726B696E67206D6F64659B
:0CE1FE002028462F552F4C29203A2000E5
:10E20A00095258207061726B696E67206D6F646580
:0CE21A002028462F552F4C29203A2000C8
:10E22600095458207061726B696E67206672657159
:09E23600203A2025362E33660043
:10E23F000D0A095258207061726B696E6720667201
:0BE24F006571203A2025362E33660052
:10E25A000D0A0953657420545258206D6F64652F56
:10E26A00667265712E20696E207061726B696E67C5
:0BE27A00203F205B592F4E5D2020004C
:10E2850009456C65766174696F6E205061726B69C2
:10E295006E672076616C7565203A2025332E3166D0
:01E2A5000078
:10E2A6000D0A0D0A09417A696D757468202050615E
:10E2B600726B696E67202076616C7565203A202541
:05E2C600332E3166005B
:10E2CB000D0A0D0A0953657420416E74656E6E61FB
:10E2DB00205061726B696E6720706F736974696F20
:0CE2EB006E203F205B592F4E5D2020006C
:10E2F7000D09454C206D6178696D756D2076616CEF
:08E307007565203F203A20005B
:10E30F000D0A09454C206D696D696D756D2076613B
:09E31F006C7565203F203A2000D6
:10E328000D0A09414443207370616E2076616C7553
:10E3380065202020454C3A2025303464202D2025A6
:05E348003034642000E8
:10E34D000D0A0953657420666C6970206D6F6465E4
:10E35D00206F7065726174696F6E20666F722065D3
:0FE36D006C65766174696F6E20726F746F7200E9
:10E37C000D09415A206D6178696D756D2076616C5F
:08E38C007565203F203A2000D6
:10E394000D0A09415A206D696E696D756D207661AB
:09E3A4006C7565203F203A200051
:10E3AD000D0A09414443207370616E2076616C75CE
:10E3BD0065202020415A3A2025303464202D202517
:05E3CD00303464200063
:10E3D2000D0A2020526F7461746520746865206193
:10E3E2006E74656E6E6120746F2066756C6C792038
:10E3F200435720616E6420456C65766174696F6E67
:10E40200206D6178696D756D20706F736974696FC5
:02E412006E009A
:10E414000D0A2020526F7461746520746865206150
:10E424006E74656E6E6120746F2066756C6C7920F5
:10E4340043435720616E6420456C65766174696F4F
:10E444006E206D696E696D756D20706F7369746986
:03E454006F6E00E8
:10E457000D0A202053657420666C6970206D6F6407
:10E4670065206F7065726174696F6E20666F7220C8
:10E47700656C65766174696F6E20726F746F720078
:10E487000D0A0D0A2020414443207370616E2076E7
:10E49700616C7565202020415A3A2025303464206C
:10E4A7002D20253034642020454C3A202530346413
:0AE4B700202D20253034640D0A00EA
:10E4C10020416E742E20646972656374696F6E20D9
:01E4D100004A
:10E4D20009415A3D253464202F2025332E316664AC
:10E4E200656709454C3D253464202F2025332E31A4
:0BE4F200666465672E202020200D00CE
:10E4FD000D0A09456C65766174696F6E3A20253297
:04E50D002E31660045
:10E511000D0A0D0A09417A696D7574683A20253230
:04E521002E31660031
:10E525000D0A0D0A094C6566742834292C20526998
:10E535006768742836292C2055702838292C2044E2
:10E54500776E2832292C2053746F70283529206F57
:0BE5550072205265742E0D0A0D0A00A2
:10E560000D0953656C6563745B312D322C515D3A36
:02E57000200089
:10E5720009322E456E74657220646972656374692E
:0EE582006F6E2076616C75652E0D0A0D0A0015
:10E5900009312E44697265637420726F746F722042
:10E5A000636F6E74726F6C2066726F6D206B65792D
:0AE5B00020626F6172642E0D0A00F4
:05E5BA000D0A0D0A002E
:07E5BF00464F2D3239000028
:05E5C600464E313B0050
:05E5CB00464E303B004C
:08E5D0004D442562643B00008C
:05E5D8004443313B004B
:05E5DD004443303B0047
:0BE5E2004641253031316C753B0000D4
:08E5ED00253031306C7500008F
:07E5F5002530394C640000E1
:0BE5FC004642253031316C753B0000B9
:10E607000709457869742066726F6D204572726FCD
:10E6170072206D6F64652061742025303262643A20
:0FE6270025303262643A25303262640D0A0A00EF
:10E63600436865636B207468652073797374656DD0
:01E6460000D3
:10E64700526F7461746F72204572726F722021204D
:01E6570000C2
:10E65800070D0A09526F7461746F72204572726FE8
:10E66800722061742025303262643A253032626447
:10E678003A25303262640D0A09436865636B20618C
:10E688006E6420706F776572206F6E207265736597
:10E698007420666F722073797374656D2072656378
:09E6A8006F766572792E0D0A00EF
:10E6B10051525820466C697020636865636B2E2E39
:01E6C1000058
:10E6C200070D0A0D0A20205B5072696F7220536198
:10E6D20074656C6C69746520252D3973206973200B
:07E6E200414F535D0D0A00DA
:10E6E900415A2025332E316620454C25322E31667C
:06E6F9002020202020007B
:10E6FF004125332E3066204525322E306620502599
:09E70F00332E3166202020200089
:09E718002563252D357320200036
:10E7210025303262643A25303262643A25303262F1
:02E73100640082
:0AE733002F252D352E3066200D0035
:10E73D0025372E316625382E316625372E31662543
:06E74D002B362E306600A1
:10E7530025382E326625382E326625392E31662528
:05E76300392E316600B3
:10E7680025632025303262643A25303262643A25C6
:05E77800303262640074
:07E77D000D0A25730D0A00CF
:10E78400415A2025332E316620454C25322E3166E0
:05E79400202020200000
:10E7990025303262643A25303262643A2530326279
:08E7A900642563252D37730080
:0EE7B10025362E31662F252D362E31660D00B1
:10E7BF0025362E31662F252D362E316625362E31F4
:09E7CF00662F252D362E3166005F
:10E7D80025352E31662F252D362E316625362E31DC
:09E7E800662F252D362E31660046
:10E7F10025632025303262643A25303262643A253D
:06E80100303262642000C9
:10E80700070D0A094F7574206F66206E756D626576
:10E81700722021202831202D202564292020233112
:10E82700207761732073656C656374656420666F18
:10E8370072204C434420646973706C61790D0A003F
:10E84700202048483A4D4D3A5353202020646567AD
:10E8570020202020206465672020202020204B6D69
:10E8670020202020202020204B6D202020202064E5
:10E87700656720202020206465672020203C3235F2
:0DE88700363E202020202020487A0D0A0077
:10E8940020202020205554432020202020417A6924
:10E8A4006D2E202020456C65762E20202052616E2E
:10E8B4006765202020202020416C742E2020204CCD
:10E8C40061742E2020204C6F6E672E2020506861CA
:0FE8D4007365202020446F70706C65720D0A0010
:10E8E30020205B536174656C6C6974653A20252D37
:07E8F30039735D200D0A00DE
:10E8FA000D0A2020274E2720547261636B206E6513
:10E90A00787420736174656C6C6974652020275073
:10E91A002720546F67676C65207072696F7269741B
:0DE92A007920747261636B696E670D0A00DD
:10E937000D0A202027312F322F332F3427205570EF
:10E947006C696E6B206368616E6E656C2020272B87
:10E957002F2D2F302720446F70706C657220636FE6
:10E967006D70656E736174696F6E2020273F272075
:0AE977006F626A2E207361742E0097
:10E981000D0A202027492720496E697469616C6945
:10E991007A6520746865205452582020202027541D
:10E9A100272054756E65205452582020202753503B
:10E9B100432F42532720204E6578742F507265767D
:0BE9C100696F75732E207361742E00C7
:10E9CC000D0A202027452720546F67676C6520723D
:10E9DC006F746F7220636F6E74726F6C2020275986
:10E9EC002720525443207A65726F2061646A7573D4
:10E9FC007420202751272052657475726E20746F15
:0BEA0C00206D61696E206D656E750065
:10EA17000D0A0D0A09203D3D3D3D3D3D3D3D3D3D36
:10EA2700205265616C74696D6520547261636B690E
:10EA37006E67205B2534642F25303262752F2530B1
:10EA47003262755D203D3D3D3D3D3D3D3D3D0D0AFD
:01EA570000BE
:03EA58000D0A00A4
:0EEA5B0020202D202020202020202020200000
:06EA6900252D313373007E
:0FEA6F00202048483A4D4D3A5353202020200094
:10EA7E000D0A2020274527546F67676C6520726F3B
:10EA8E00746F7220636F6E74726F6C202027502724
:10EA9E00546F67676C65207072696F726974792044
:10EAAE00747261636B2027512752657475726E20E4
:10EABE00746F206D61696E206D656E750D0A0D0A9D
:01EACE000047
:10EACF000D0A0D0A0D0A09203D3D3D3D3D3D3D3DE1
:10EADF003D3D205265616C74696D652054726163B0
:10EAEF006B696E67205B2534642F25303262752F7A
:10EAFF0025303262755D203D3D3D3D3D3D3D3D3D07
:03EB0F000D0A00EC
:10EB12000D0A0953656C6563742046756C6C206F31
:10EB220072626974206F7220414F53204341542016
:10EB3200636F6E74726F6C203F205B462F415D20C5
:02EB42002000B1
:10EB44000D0A09446F776E6C696E6B20446F7070A8
:10EB54006C657220636F7272656374696F6E203FB7
:0BEB6400205B592F4E2F525D20200037
:10EB6F000D0A0955706C696E6B20446F70706C657F
:10EB7F007220636F7272656374696F6E203F205BE2
:07EB8F00592F4E5D2020000C
:10EB96000D0A09506F727420626175642072617487
:10EBA60065203F205B313230302F343830302F39FA
:0CEBB6003630302F31393230305D200015
:0AEBC200205B312D3235355D200057
:10EBCC000D0A09576169742074696D6520666F724E
:10EBDC0020636F6D6D616E64205B2562645D200047
:10EBEC000953657061726174656420545258203FFA
:09EBFC00205B592F4E5D20200022
:10EC050009456E7465722064657374696E61746913
:10EC15006F6E204164647265737320666F72205451
:09EC25005820282542582920003E
:04EC2E0025627800E3
:10EC32000D0A09456E7465722064657374696E61AC
:10EC420074696F6E204164647265737320666F72BB
:0BEC520020525820282542582920009D
:10EC5D000D0A0953656C65637420464D4E206D6F2A
:0CEC6D006465203F205B592F4E5D2000A5
:10EC79000D0A0953656C6563742054525820313A62
:10EC890046542D3733362020323A46542D383437FE
:0CEC99002020333A4F7468657220200080
:10ECA5000D0A092020416C7465726E6174652043FC
:10ECB5004F4D20706F7274206973203830333120C6
:0CECC50050312E352F434E332D362000E9
:10ECD1000D0A092020596F75206D757374207573A5
:10ECE1006520616C7465726E61746520434F4D20BF
:10ECF100706F727420666F722055706C696E6B2034
:04ED01005452580010
:10ED05000D0A09497320746865204341542052490E
:10ED1500472054532D37313120262054532D383177
:10ED25003120636F6D62696E6174696F6E203F207B
:07ED35005B592F4E5D200029
:10ED3C000D0A0A0943415420526967204B454E572E
:10ED4C004F4F442C59414553552C49434F4D205B53
:0BED5C004B2F592F495D203F20200065
:10ED67000D0A09436F6E66696775726520796F755D
:10ED7700722073746174696F6E20656C656D656E62
:0DED87007473203F205B592F4E5D2020004B
:10ED94000D0A09546869732066756E6374696F6E31
:10EDA4002077617320656C696D696E617465642098
:10EDB400696E20433235312076657273696F6E0057
:10EDC40009392E205365742064656661756C74205E
:0EEDD400706172616D657465720D0A0D0A0042
:10EDE20009382E205B4D69632D636C69636B206368
:10EDF2006F6E66696775726174696F6E5D0D0A0088
:10EE020009372E20526164696F2043415420706F8C
:10EE1200727420636F6E66696775726174696F6E72
:03EE22000D0A00D6
:10EE250009362E2044697265637420616E74656EBF
:0DEE35006E6120636F6E74726F6C0D0A00C9
:10EE420009352E204D6F6E69746F72204144432044
:10EE520076616C756520616E6420616E74656E6E9C
:0DEE62006120706F736974696F6E0D0A0096
:10EE6F0009342E2053657420616E74656E6E6120B7
:10EE7F005061726B696E6720616E64204C696D69B9
:0DEE8F007420706F736974696F6E0D0A0056
:10EE9C0009332E2053657420446561642042616EF1
:10EEAC006420616E6420536B65772076616C7565A8
:03EEBC000D0A003C
:10EEBF0009322E2053657420414443207370616ED4
:09EECF002076616C75650D0A00E6
:10EED80009312E2043616C6962726174696F6E201A
:10EEE8006F6620616E74656E6E61207370616E204E
:08EEF80076616C75650D0A00DE
:10EF000009302E20446973706C617920616C6C202B
:10EF1000636F6E666967757265642076616C75658E
:04EF2000730D0A0063
:10EF24000D0A0D0A093D3D3D3D3D3D3D20436F6EBB
:10EF340066696775726174696F6E204D656E7520C0
:0AEF4400203D3D3D3D3D3D0D0A001E
:0DEF4E0009257320257309090920202000E2
:0CEF5B00092573202573090920202000DF
:0DEF670009202046324F46465345543A00DB
:10EF7400256C6620256C6620256C6620256C660051
:10EF84000925732025362E33662025362E33662038
:10EF940025362E33662025362E33660D0A090909D7
:05EFA4002020202000E8
:0DEFA90009202046314F46465345543A009A
:06EFB600090946783A004B
:0AEFBC000925732025362E3066006B
:06EFC600090946313A0082
:0AEFCC000925732025362E33660058
:05EFD600094E313A0074
:07EFDB0009257320256500E4
:06EFE20009094F303A005E
:06EFE800090957303A0050
:06EFEE00090945303A005C
:0AEFF4000925732025362E3766002C
:06EFFE00090949303A0048
:06F0040009094E303A003C
:06F00A0009094D303A0037
:0AF010000925732025362E34660012
:06F01A0009094B303A0029
:09F020000925732025366C6400FB
:06F02900090954303A0011
:0AF02F000925732025362E386600EF
:07F0390009090959303A00F2
:07F04000092573202564007F
:0AF0470009257320252D7309090027
:10F051000D0A0D0A09093D3D3D3D3D3D20536174B9
:10F06100656C6C6974652064617461203D3D3D3D52
:05F071003D3D0D0A0009
:05F07600464D202000C2
:05F07B004357202000B6
:05F08000555342200081
:05F085004C5342200085
:05F08A006E6F6E6500D1
:10F08F002020202020463120736C657728487A296C
:04F09F0020203A00F3
:10F0A3002020204F666673657420666F7220463297
:04F0B30020203A00DF
:10F0B7002020204F666673657420666F7220463184
:04F0C70020203A00CB
:10F0CB0020204C4344204D4120646973706C61795E
:04F0DB0020203A00B7
:10F0DF00446F70706C657220636F72726563742E0B
:04F0EF0020203A00A3
:10F0F30020202045706F6368205965617220593064
:04F1030020203A008E
:10F10700202020202055706C696E6B206D6F646520
:04F1170020203A007A
:10F11B00202020446F776E6C696E6B206D6F646579
:04F12B0020203A0066
:10F12F0020202055706C696E6B204672712E46320E
:04F13F0020203A0052
:10F1430020446F776E6C696E6B204672712E463168
:04F1530020203A003E
:10F1570020202020202020204465636179204E3123
:04F1670020203A002A
:10F16B002020202020522E412E412E4E2E204F307B
:04F17B0020203A0016
:10F17F00202041726720706572696765652057307E
:04F18F0020203A0002
:10F1930020456363656E74726963697479204530D1
:04F1A30020203A00EE
:10F1A7002020496E636C696E6174696F6E20493007
:04F1B70020203A00DA
:10F1BB0020204D65616E204D6F74696F6E204E304F
:04F1CB0020203A00C6
:10F1CF00204D65616E20416E6F6D616C79204D3001
:04F1DF0020203A00B2
:10F1E3002020202045706F636820526576204B30C5
:04F1F30020203A009E
:10F1F70020202045706F63682054696D6520543066
:04F2070020203A0089
:10F20B0020202020202020536174656C6C6974656C
:04F21B0020203A0075
:04F21F0059657300BA
:03F223004E6F002B
:0BF226004D69632D636C69636B200071
:05F231004341542000E0
:10F236000D0A07202120466F726D61742045727297
:05F246006F72202100A1
:10F24B000D0A09202020454E544552207768656EE3
:08F25B002072656164792E0048
:10F263000D0A095365742074696D653A2025730D81
:02F273000A008F
:10F2750009456E746572207769746820666F726DD2
:10F285006174205B59592F4D4D2F44442048483A0D
:08F295004D4D3A53535D20007A
:10F29D002534642F25303262752F2530326275206A
:10F2AD0025303262753A25303262753A2530326238
:04F2BD00750D0A00C1
:10F2C1000D0A0D0A09536574207265616C74696DCC
:10F2D1006520436C6F636B2E0D0A0950726573656F
:0DF2E1006E742054696D653A555443200049
:10F2EE002534642F25303262752F25303262752019
:10F2FE0025303262753A25303262753A25303262E7
:0BF30E007520543A25352E38660D009E
:10F319000950726573656E742054696D653A555468
:03F329004320007E
:10F32C000D0A09456E74657220275265742E2720CC
:10F33C00666F72205265616C2054696D6520436C58
:0CF34C006F636B207365740D0A0D0A00DE
:10F358000D0A09456E7465722027512720666F7261
:06F36800206578697400C5
:10F36E000D0A09456E7465722027592720666F7243
:10F37E00207A65726F207365632E2061646A7573DF
:06F38E00746D656E740051
:0AF39400253135733A20202573005F
:0CF39E00253135733A202025730920002A
:0DF3AA00253135733A202025352E326600BE
:02F3B70009004B
:0EF3B900253135733A2020252B352E33660082
:0BF3C700253135733A20202573090022
:10F3D2000D0A0D0A093D3D3D3D3D3D3D3D3D20535C
:10F3E200746174696F6E20456C656D656E7473200F
:0DF3F2003D3D3D3D3D3D3D3D0D0A0D0A00F8
:10F3FF0009322E2052454C4F41443A20436C6561EF
:10F40F007220646174616261736520262072656188
:10F41F006420696E206E657720646174612E0D0A19
:03F42F000D0A00C3
:10F4320009312E20454449543A20202056696577E7
:10F442002F456469742073746174696F6E20656CF2
:10F45200656D656E74732062792068616E642E0D2D
:02F462000A009E
:10F464000D0A0D0A092020203D3D3D3D3D3D3D3D19
:10F474003D2053746174696F6E2044617461203D52
:0AF484003D3D3D3D3D3D3D0D0A00BC
:10F48E0020202020434F4D20706F727420626175D2
:02F49E00640008
:10F4A000526F746F722073746172742028532F4EE0
:02F4B000290031
:10F4B200202020416E74656E6E6120686569676800
:02F4C2007400D4
:10F4C40020202020202020204C6F6E6769747564F2
:02F4D4006500D1
:10F4D6002020202020202020204C6174697475642F
:02F4E6006500BF
:10F4E80020202020202020202043616C6C73696735
:02F4F8006E00A4
:06F4FA0031393230300010
:05F50000393630300037
:05F50500343830300035
:05F50A00323430300036
:05F50F00313230300034
:05F5140020333030003F
:06F519004E6F72746800E1
:06F51F00536F75746800D3
:10F525000D0A094F7574206F662072616E6765203C
:03F53500210700AB
:10F538000D0A09486F77206D616E792073617465D3
:10F548006C6C6974657320636F6E66696775726544
:10F5580020666F72206D756C746920747261636BBC
:10F56800696E67206D6F6465203F202832202D204A
:05F578003529202000F0
:10F57D000D0A0946696C6520666F726D6174204EC7
:0CF58D0041534120284E29203A20200044
:10F59900070D0A204E6F20726F6F6D20666F722003
:0BF5A900617070656E6420210D0A0087
:10F5B400070D0A0953746F726564206461746120D5
:10F5C400696E206D656D6F72792077696C6C20624D
:10F5D40065206C6F73742E2041726520796F7520DD
:07F5E40073757265203F0002
:10F5EB0009332E2055706C6F6164202020203A2047
:10F5FB0055706C6F61642073656C656374696F6EB5
:0EF60B0020646174612066696C652E0D0A0032
:10F6190009322E2053656C65637420416C6C3A2065
:10F6290053656C65637420616C6C20736174732E0F
:10F6390020696E2074686520646174616261736514
:04F649002E0D0A0078
:10F64D000D0A0D0A09312E2053656C656374202057
:10F65D0020203A2053656C65637420736174732E9A
:0CF66D002062792068616E642E0D0A0096
:10F67900070D0A0953656C6563746564206C6973C9
:10F68900742077696C6C206265206C6F73742E200E
:0FF6990041726520796F752073757265203F008F
:10F6A8000D0A092A2A2A202053656C656374206F85
:10F6B800626A65637420736174656C6C6974652033
:07F6C800202A2A2A0D0A0086
:0CF6CF000D090953656C6563743A200056
:10F6DB0009352E204D554C544920545241434B3A39
:10F6EB0020436F6E666967757265206D756C746902
:10F6FB0020747261636B696E67207361742E206E68
:0BF70B00756D6265722E0D0A0D0A007C
:10F7160009342E20415050454E443A2041707065C0
:10F726006E64206E657720456C656D656E74732E0C
:03F736000D0A00B9
:10F7390009332E2052454C4F41443A20436C6561B0
:10F74900722064617461626173652026207265614B
:10F759006420696E206E657720456C656D656E74F1
:05F76900732E0D0A00E3
:10F76E0009322E2053454C4543543A2053656C655F
:10F77E00637420536174656C6C6974657320667272
:10F78E006F6D207468652064617461626173652EAB
:03F79E000D0A0051
:10F7A10009312E20454449543A2020205669657775
:10F7B1002F4564697420736174656C6C697465208C
:10F7C100456C656D656E74732062792068616E6445
:04F7D1002E0D0A00EF
:10F7D5000D0A0D0A092020203D3D3D3D3D3D3D3DA5
:10F7E5003D20555044415445204D454E55203D3D05
:09F7F5003D3D3D3D3D3D0D0A0086
:10F7FE000D0953656C656374205B312D382C532CC9
:05F80E004D5D3A2000F1
:10F8130009382E2044697265637420416E74656EE5
:10F823006E6120636F6E74726F6C2E0D0A0D0A0089
:10F8330009372E20486F7374206D6F64652E0D0A8F
:01F8430000C4
:10F8440009362E20436F6E66696775726174696F3D
:05F854006E2E0D0A00FC
:10F8590009352E20557064617465205265616C7498
:0DF86900696D6520436C6F636B2E0D0A0006
:10F8760009342E205570646174652053746174696F
:0FF886006F6E20456C656D656E74732E0D0A00F4
:10F8950009332E2055706461746520536174656C5D
:10F8A5006C69746520456C656D656E74732E0D0A03
:01F8B5000052
:10F8B60009322E20446973706C6179205363686540
:08F8C60064756C652E0D0A004B
:10F8CE0009312E205265616C74696D652054726128
:09F8DE00636B696E672E0D0A00D0
:10F8E7000D0A20092D2D2D2D2D2D204D41494E205E
:10F8F7004D454E55202D2D2D2D2D2D0D0A0D0A0070
:10F907000D0A093D3D3D3D204144432076616C751C
:10F917006520616E6420616E74656E6E6120646936
:10F9270072656374696F6E203D3D3D3D0D0A0D0A9A
:01F9370000CF
:0AF93800205B592F4E5D203F200098
:07F94200594F524F4E000027
:08F949004E4F43414C4C0000FD
:10F95100070D0A094461746120696E2052414D20EE
:10F96100776173206C6F737420212120536574209B
:10F9710064656661756C7420706172616D65746532
:06F981007220210D0A00B6
:02F98700070077
:10F989000D0A0D0A092A2A2A202053656C65637419
:10F99900206F626A65637420736174656C6C697445
:09F9A9006520202A2A2A0D0A001B
:10F9B2000D0A092A2A2A2020547261636B696E6734
:10F9C200206F626A65637420736174656C6C69741C
:09F9D2006520202A2A2A0D0A00F2
:04F9DB000A0D07000A
:10F9DF000A0D07546F6F206F6C6420656C656D6541
:08F9EF006E74732E200D0A0056
:10F9F70031332F30312F30312030303A30303A30F8
:02FA07003000CD
:06FA0900594F524F4E0060
:09FA0F0031373A32303A3330004D
:03FA1800202000AB
:0CFA1B0053657020323720323031330048
:04FA270009090900C0
:10FA2B002843294A414D5341542F4A413646544CA1
:02FA3B000000C9
:10FA3D00202076657273696F6E20332E363061200B
:02FA4D000000B7
:10FA4F00205472616B426F78203830433235312049
:02FA5F000000A5
:10FA6100092A2A2A2A2A2A2A2A2A2A2A2A2A2A2A16
:10FA71002A2A2A2A2A2A2A2A2A2A2A2A2A2A2A2AE5
:0CFA81002A2A2A2A2A2A2A2A2A0D0A00E8
:10FA8D00092A202020284329204A414D5341542F33
:10FA9D004A413646544C2020205365702E32322078
:0CFAAD0032303133202020202A0D0A00C6
:10FAB900092A2020202020205472616B426F782D62
:10FAC90049492020383043323531202076332E36CB
:0CFAD90030612020202020202A0D0A008F
:10FAE5000D0A0D0A0D0A092A2A2A2A2A2A2A2A2A49
:10FAF5002A2A2A2A2A2A2A2A2A2A2A2A2A2A2A2A61
:10FB05002A2A2A2A2A2A2A2A2A2A2A2A2A2A2A0D6D
:02FB15000A00E4
:08FB170000FFF51F00FFF519C6
:10FB1F0000FFF51400FFF50F00FFF50A00FFF505D4
:08FB2F0000FFF50000FFF4FAED
:10FB370000FFF4E800FFF4D600FFF4C400FFF4B2BE
:08FB470000FFF4A000FFF48EA2
:08FB4F0000FFF23100FFF22675
:08FB570000FFF22300FFF21F82
:10FB5F0000FFF20B00FFF1F700FFF1E300FFF1CF21
:10FB6F0000FFF1BB00FFF1A700FFF19300FFF17F52
:10FB7F0000FFF16B00FFF15700FFF14300FFF12F82
:10FB8F0000FFF11B00FFF10700FFF0F300FFF0DFB4
:10FB9F0000FFF0CB00FFF0B700FFF0A300FFF08FE6
:10FBAF0000FFF08A00FFF08500FFF08000FFF07B80
:04FBBF0000FFF076DD
:0CFBC30000FFE02600FFE01E00FFE0183D
:08FBCF0000FFF51F00FFF5190E
:10FBD70000FFF08A00FFE01400FFE01000FFE00DD7
:04FBE70000FFE00A31
:08FBEB0000FFE00600FFE0014D
:10FBF30000FFF51400FFF50F00FFF50A00FFF50500
:08FC030000FFF50000FFF4FA18
:10FC0B00002C01000000FFFAE500FFFAB900FFFA33
:10FC1B008D00FFFA6100FFFA4F00FFFA3D00FFFA7B
:10FC2B002B00FFFA2700FFFA1B00FFFA1800FFFA60
:01FC3B000FB9
:0BFC3C00000601005B40D0E8F4FAFD78
:0FFC4700000A010061FD00FF40FF40FFA0FFD059
:10FC5600001A01006D001F1C1F1E1F1E1F1F1E1FE6
:0FFC66001E1F001F1D1F1E1F1E1F1F1E1F1E1FE4
:10FC750000F00100873FD1A0D77B7C78213FD1954B
:10FC8500FAA8A82A563FD1B7F9D6F112FD3FD1AD52
:10FC95001D041CC5333FD1A240314877683FD19739
:10FCA500635E74299E3FD1B9628CBD12453FD1AECA
:10FCB50085B9E8C47A3FD1A3A4B5568E823FD198C1
:10FCC500C7E28240B83FD1BAC710CB295F3FD1AF59
:10FCD500EA3DF6DB943FD1A50D6B228DCA3FD19A43
:10FCE50030984E3FFF3FD1BC2FC69728A63FD1B1D4
:10FCF50052F3C2DADC3FD1A67620EE8D113FD19BBF
:10FD0500994E1A3F463FD1BD944AA53FC03FD1B257
:10FD1500B777D0F1F53FD1A7DAA4FCA42B3FD19C4E
:10FD2500FDD22856603FD1BEFD00713F073FD1B4DB
:10FD3500202D9CF13D3FD1A9435AC8A3723FD19EC6
:10FD45006687F455A83FD1C065B63D3E4F3FD1B556
:10FD550084B1AB08573FD1AAA7DED6BA8C3FD19F55
:05FD6500CB0C026CC292
:100240006CDD12008B7E34FA097E2400FF7E147967
:100250002D7E04000112D626601112596D12008BFA
:100260007E14F9F77E0400FF1201917E347530127E
:10027000B39B900010691E00020BEA001204367452
:10028000C0120218900018691E00020BEA00120446
:100290003612044B7E8440787E94C0009F55907641
:1002A0007C0BEA00691E0002692E0004693E00060C
:1002B00012B7C1280B7E14F9DF7E0400FF1206235B
:1002C00012A99B7CCB4CCC685C90002C0BEA304E86
:1002D0003401001BEA307E14F9DB7E0400FF1206B5
:1002E0002390E102E054F0F012A99B7CCB149079AA
:1002F0002BF01A3B2E3427AB7A71827A6183E0BEF1
:10030000B00048044CCC780712A99B7CCB80D290DB
:10031000002C0BEA305E340200680512326080C1A6
:1003200012389980BC90002C0BEA305E34FEFF1B23
:10033000EA3012B3AA90E102E054F0F090002C0BE6
:10034000EA305E34FDFF1BEA3090002E0BEA304E9F
:100350003404001BEA3090002C0BEA305E341000AD
:1003600068057ED00780051245EE7CDB7CBD1BB1A5
:10037000685F1478030203FF1478030204051478FD
:100380000302040B14780302041114780302041707
:1003900014780302041D249B780302042324FA68C2
:1003A000042472788D7E14F9B27E0400FF120623B5
:1003B000124DA27D73BE74FFFF7803020332907961
:1003C0002AE00A3BBD3718030203321238990203B0
:1003D000327E14F9897E0400FF120623124DA27D9D
:1003E00073BE74FFFF78030203327D372E3427ABD0
:1003F0007A71827A6183E01A3B124ED10203321283
:100400006E3C020332126912020332124756020393
:10041000321265FE02033212A9C902033212929708
:1004200002033290002C0BEA304E3402001BEA30FB
:06043000123260020332EB
:10008B00740290E201F0748290E103F0E490E100DD
:10009B00F0759852758922758780C2CAC28E90E11D
:1000AB0001E054807805758DE8802A90006B7EEB1B
:1000BB00A0BEA0004005BEA005280B740490006BE9
:1000CB00F0758DFA800F0A3A2E34005B7A71827AC2
:1000DB006183E0F58D90006C7EEB707402AC7B2E2F
:1000EB003400617A71827A61830BEA307D235E245E
:1000FB00FF000A54F5CBF5CD7D535E5400FFF5CAD6
:10010B00F5CCD2CAD28E90E00FE05404BEB0046896
:10011B00247E14F9877E0400FF120623740790E0F7
:10012B000FF0740490E00FF090E00DE054FEF074CB
:10013B000490E00FF07438120218740C1202187449
:10014B0006120218740112021890E00DE054FBF035
:01015B002281
:10021800C292C29190E100F07E34000A12B39BD2E0
:0402280090C29022CE
:10022C00D292C29190E100F07E34000A12B39BD2BC
:04023C0090C29022BA
:10596D007E14F9517E0400FF1206231210EB120E65
:10597D00707E340007CA397E34F9497E2400FF7EDB
:10598D001427E87E04000112D6981BFD7E34000614
:10599D00CA397E34F9427E2400FF7E14792D7E04AF
:1059AD00000112D6981BFD90E101E0548078057539
:1059BD008DE88006740490006BF0740290006CF01A
:1059CD00740790E00FF0740490E00FF090E00DE09C
:1059DD0054FEF0740490E00FF07E04403B7E14649E
:1059ED00187E2493747E34BC6A9000321BEA0079D1
:1059FD001E0002792E0004793E00067E0440607E72
:105A0D001415067E2424DD7E342F1B90003A1BEAEC
:105A1D0000791E0002792E0004793E00069F449FF6
:105A2D005590003A0BEA00691E0002692E000469C8
:105A3D003E000612B7C190003A0BEA80699E000243
:105A4D0069AE000469BE0006380D7E04BFF06D110D
:105A5D009F1112B612800D7E0440767E1480009F39
:105A6D001112B4FD9000421BEA00791E0002792E3E
:105A7D000004793E00067E0440496D119F1190008F
:105A8D004A1BEA00791E0002792E0004793E0006B9
:105A9D009F1190769E793E00021BEA209F11907611
:105AAD00A2793E00021BEA206D337E2440409076A1
:105ABD00A6793E00021BEA206D337E243F8090764E
:105ACD00AA793E00021BEA207E3400039076961BD5
:105ADD00EA307E3403459076981BEA307E3400011F
:105AED0090769A1BEA307E3401CC90769C1BEA307E
:105AFD009F119076BA793E00021BEA209F11907695
:105B0D00BE793E00021BEA209F119076F9793E0086
:105B1D00021BEA209F119076F5793E00021BEA20C8
:105B2D007404907708F07404907707F074049077FC
:105B3D0006F07404907705F09F119076C2793E00BF
:105B4D00021BEA206D337E2443B49076C6793E0065
:105B5D00021BEA209F119076CA793E00021BEA20B3
:105B6D006D337E2442B49076CE793E00021BEA203E
:105B7D006D337E24C0009076D6793E00021BEA205C
:105B8D006D337E24C0A09076DA793E00021BEA20A8
:105B9D006D337E24C0E09076DE793E00021BEA2054
:105BAD00E490792BF0740390792CF09F119076F19D
:105BBD00793E00021BEA207E18000A907701793E9B
:105BCD0000021BEA20E49076E2F0742E9076E5F068
:105BDD00742E9076E7F0742E9076E6F0742E907613
:105BED00E8F0742D900052F0742E9076E3F0741E50
:105BFD009076E4F07E3400789079251BEA307E347F
:105C0D00003D9079271BEA307E34684090002C1BB4
:105C1D00EA307E340D8390002E1BEA309000300B5D
:0D5C2D00EA304E3400021BEA3012B05F2254
:10B05F009076960BEA209076980BEA309D3212D4B8
:10B06F00C67D237CB412B8397E8440767E948000EE
:10B07F009F5512B72212B927907692793E00021B84
:10B08F00EA2090002E0BEA305E34400090769A0B47
:10B09F00EA2090769C0BEA3068129D3212D4C67D5E
:10B0AF00237CB412B8397E84406680109D3212D44E
:10B0BF00C67D237CB412B8397E8440567E948000BE
:10B0CF009F5512B72212B92790768E793E00021B38
:03B0DF00EA202242
:1010EB00CAF86CFF9F669F777E7008AC7F7D232EBE
:1010FB0024220B7A51827A41831BEAC079DE0002EB
:10110B0079EE000479FE00067D232E24202B7A51E4
:10111B00827A41831BEAC079DE000279EE00047902
:10112B00FE00069F669F772E3423EB7A71827A61DD
:10113B00831BEAC079DE000279EE000479FE00061B
:10114B009F007E7004AC7F2E3426BB7A71827A614D
:10115B0083791E00021BEA009F669F777E7020AC8E
:10116B007F2E3418877A71827A61831BEAC079DE0D
:10117B00000279EE000479FE00069F669F777E7071
:10118B0020AC7F2E34187F7A71827A61831BEAC080
:10119B0079DE000279EE000479FE00069F669F77E8
:1011AB007E7020AC7F2E3418777A71827A61831B24
:1011BB00EAC079DE000279EE000479FE00069F6634
:1011CB009F777E7020AC7F2E34186F7A71827A6194
:1011DB00831BEAC079DE000279EE000479FE00067B
:1011EB00E40A3F7D232E241FEF7A51827A4183F04C
:1011FB009F669F777E5008AC5F7D122E14168F7AF8
:10120B0031827A21831BEAC079DE000279EE000479
:10121B0079FE00067D122E1414AF7A31827A218367
:10122B001BEAC079DE000279EE000479FE00069F0E
:10123B00669F777D122E1412CF7A31827A21831B0F
:10124B00EAC079DE000279EE000479FE00069F66A3
:10125B009F777D122E1410EF7A31827A21831BEA4D
:10126B00C079DE000279EE000479FE00069F669FCE
:10127B00777D122E140E1F7A31827A21831BEAC0DE
:10128B0079DE000279EE000479FE00069F669F77F7
:10129B007D122E140C3F7A31827A21831BEAC0799E
:1012AB00DE000279EE000479FE00069F669F777DD3
:1012BB00122E140A5F7A31827A21831BEAC079DEFF
:1012CB00000279EE000479FE00069F669F777D127F
:1012DB002E14087F7A31827A21831BEAC079DE00D3
:1012EB000279EE000479FE00066D007E3002AC3F01
:1012FB002E1406277A31827A21831BEA007EC43FA3
:10130B00F06DDD9F772E24069F7A51827A41831BE5
:10131B00EAC079DE000279EE000479FE00067E0851
:10132B0000017E5004AC5F2E240FFF7A51827A416C
:10133B0083791E00021BEA00E42E3426077A7182A1
:10134B007A6183F0E40A3F2E3425CB7A71827A617D
:10135B0083F07E5002AC5F2E2426437A51827A4171
:10136B00830BEA305E34FFFB7A51827A41831BEAAE
:10137B00307A51827A41830BEA305E34FFFE7A5128
:10138B00827A41831BEA307A51827A41830BEA30AD
:10139B005E34FFFD7A51827A41831BEA307A5182A7
:1013AB007A41830BEA305E34FFEF7A51827A4183C4
:1013BB001BEA307E3014AC3F2E1401777E04000103
:1013CB007E340014E412D6C10BF0BEF03C6803026D
:1013DB0010EF6D339000591BEA306CFF74FF0A3F1E
:1013EB002E3427AB7A71827A6183F00BF0BEF03C1E
:0513FB0040ECDAF822CD
:101400009000590BEA30E4800F7D232E2427FC7ACC
:0F14100051827A4183F00B34BE344E2040EB22E0
:0FB39B006D2280020B247D130B14BD1238F62295
:10B3AA0012044B907919693E00020BEA2090792128
:10B3BA00793E00021BEA2090791D793E00021BEAC1
:02B3CA0020223F
:10A99B0090002E0BEA305E341000780990E101E054
:10A9AB0064FF540F2274021201C57E55081E541EFB
:0EA9BB00541E541E541E541E545E54000F228F
:10062300CA3B7F307F130B747E1BB0600512D14B26
:0506330080F2DA3B2219
:10043600CA3B7F307F130B747E1BB0600512022C03
:0504460080F2DA3B2208
:1093EB00CA3B7F307F130B747E1BB06005120003EA
:0593FB0080F2DA3B22C4
:10B4E500CA3B7F307F130B747E1BB06005120025AD
:05B4F50080F2DA3B22A9
:10902000CA3B7F306D33907A8F804412D4B37CABCF
:10903000BEA00D683FBEA00A683ABEA008680FBE79
:10904000A07F781C907A8F0BEA304D336812E47F52
:10905000131B747A1BB0907A8F0BEA301B34800F8D
:109060007F130B747A1BA0907A8F0BEA300B341BA2
:10907000EA3080B7E47F130B747A1BB0907A8F0BC1
:05908000EA30DA3B229A
:1065CB00CA3B7F311206237E1479977E0400011299
:1065DB0090206D331B3A307E1479977E04000112A4
:1065EB00D6691B3A307E1479977E04000112D4E6EB
:0365FB00DA3B2266
:10659800CA3B7F311206237E147A3F7E0400011223
:1065A80090206D331B3A307E147A3F7E040001122E
:1065B800D6691B3A307E147A3F7E04000112B9DF97
:0365C800DA3B2299
:10656E001206237E14F9387E0400FF12062312D47D
:10657E00B37C7B7CA74EA020BEA079780374012249
:0A658E00BEA06E7802E42274FF2222
:1001F80090E00DE04401F090E00DE05402681090AA
:10020800E00DE054FEF07E34000A12B39B80E12238
:10015C001201F86CAA0A2A7E34E00B9D322E340070
:10016C00007A71827A6183E0540F44307C1A2E102D
:10017C000FA5F70BA0BEA00C40DB751B0090E00D8B
:05018C00E054FEF0222A
:100191007EA0106C776C660A2A7F702DF27E7BB090
:1001A10024D00A262E24E0007A51827A4183F01B62
:1001B100A00B70BE700240041BA06C770B60BE6088
:0401C1000C40D422F8
:1001C500540790E200F07E34001E12B39B90E201CA
:1001D500E00A3B90E200E00A2B7C676C774D321E0B
:1001E500341E341E341E341E341E345E3403FF7A2E
:0301F500350822A8
:109085007E14F9077E0400FF12062330980412D4DB
:08909500B32212909D80F42229
:1045EE00900000691E00020BEA00120623900004E0
:1045FE00691E00020BEA00120623900008691E00D5
:10460E00020BEA0012062390000C691E00020BEA50
:10461E00001206237480120218900010691E000208
:10462E000BEA0012043674C0120218900014691EB0
:10463E0000020BEA001204367E14F8E77E0400FF37
:10464E001206237E14F8CE7E0400FF1206237E147B
:10465E00F8B67E0400FF1206237E14F8957E040041
:10466E00FF1206237E14F8767E0400FF1206237EC8
:10467E0014F8597E0400FF1206237E14F8447E04BB
:10468E0000FF1206237E14F8337E0400FF12062369
:10469E007E14F8137E0400FF1206237E14F7FE7EAE
:1046AE000400FF12062330983412D4B37C7BBE7004
:1046BE0030400ABE703838057CB724D0227CA74E15
:1046CE00A020BEA0737803747322BEA06D7803740D
:1046DE006D227E14F7FE7E0400FF12062390002C3E
:1046EE000BEA307D235E24001068BB5E3400046844
:0946FE00B5740112B3E780AE228D
:1068A7007E14F7D57E0400FF1206237E14F7A17E1F
:1068B7000400FF1206237E14F76E7E0400FF120603
:1068C700237E14F7397E0400FF1206237E14F71681
:1068D7007E0400FF1206237E14F6DB7E0400FF12FF
:1068E70006237E14F6CF7E0400FF12062312D4B3CC
:1068F7007CABBEA031400ABEA03538057CBA24D097
:0B690700227CBA4420B471DA747122C3
:106E3C00CA3B1268A77CEB1BB16846147803026F3F
:106E4C0058147803026F58147803026FD424947882
:106E5C0003027011247078DA7E14F6A87E0400FF09
:106E6C00120623124DA27CC7BEC0FF68C51A3C2E69
:106E7C003427AB7A71827A6183E01A3B12822980C3
:106E8C00B17E14F6797E0400FF12656E7CDBBED0F9
:106E9C0000089F6CFF7E5002AC5F2E2426437A5173
:106EAC00827A41830BEA305E34FFEF7A51827A4169
:106EBC00831BEA300BF0BEF03C78DA7E14F64D7E84
:106ECC000400FF1206237E14F6197E0400FF12063E
:106EDC00237E14F5EB7E0400FF1206237E14F6CFFE
:106EEC007E0400FF12062312D4B324CE681014685B
:106EFC00550BB16803026E3E12A17E026E3E6CFF12
:106F0C0080360A3F2E3427AB7A71827A61837AEB12
:106F1C00F07E5002AC5F2E2426437A51827A418354
:106F2C000BEA304E3400107A51827A41831BEA30DE
:106F3C000BF090792A7AEBF0907929E0BCBF38C23B
:106F4C0012A20F026E3E129A1A026E3EBEE0037837
:106F5C001F7E14F5B47E0400FF12656E7CDBBED080
:106F6C00001803026E3E6D339000591BEA30801CF2
:106F7C00BEE0047817907929E0BEB03C400E7E1438
:106F8C00F5997E0400FF120623026E3E7E14F57DF9
:106F9C007E0400FF12062312D4B36CFF7E5002ACA9
:106FAC005F2E2426437A51827A41830BEA305E3479
:106FBC00FFEF7A51827A41831BEA300BF0BEF03C32
:106FCC0078DA129400026E3E7E14F5387E0400FFCF
:106FDC007E3479437E2400011265CB7CE7BEE0024F
:106FEC00400DBEE0053808907929E0BCEB280D7EF9
:106FFC0014F5257E0400FF12062380CC90792C7AA0
:08700C00EBE0026E3EDA3B22CC
:10691200CAD8CA797E34FB177E2400FF7E147959C7
:106922007E040001740812D1187E34FB1F7E2400FD
:10693200FF7E1479617E040001741812D1187E342E
:10694200FB377E2400FF7E1479797E0400017418DF
:1069520012D1187E14F4647E0400FF1206237E1402
:10696200F4327E0400FF1206237E14F3FF7E04003D
:10697200FF1206237E14F6CF7E0400FF12062312B6
:10698200D4B37CDBBED0316813BED032680E7CBD7E
:106992004420BEB0717803026D9580D8BED03278A3
:1069A20006125C3A026D95BED0316803026D957491
:1069B2001A12D14B7E14F3D27E0400FF12062390EA
:1069C2007979693E00020BEA20907B62793E0002EF
:1069D2001BEA207E3427E87E240001907B5E793E0C
:1069E20000021BEA207E14F3C77E0400FF12B95E88
:1069F2007E1479457E0400011290204D3368137E87
:106A02003479457E2400017E1427E87E04000112B9
:106A1200D60790797D693E00020BEA20907B62796D
:106A22003E00021BEA209000320BEA00691E0002BF
:106A3200692E0004693E0006907B5A1BEA00791E0B
:106A42000002792E0004793E00067E14F3B97E041A
:106A520000FF12B95E7E14F3B77E0400FF7E347924
:106A6200437E24000112659890794F1BEA00791E3B
:106A72000002792E0004793E00069079430BEA3039
:106A82004D33682490794F0BEA00691E0002692E8B
:106A92000004693E00069000321BEA00791E0002E3
:106AA200792E0004793E0006907981693E00020B3E
:106AB200EA20907B62793E00021BEA2090003A0BAA
:106AC200EA00691E0002692E0004693E0006907BFE
:106AD2005A1BEA00791E0002792E0004793E000654
:106AE2007E14F3B97E0400FF12B95E7E14F3B77E02
:106AF2000400FF7E3479437E240001126598907968
:106B02004F1BEA00791E0002792E0004793E00062E
:106B12009079430BEA304D33682490794F0BEA00A9
:106B2200691E0002692E0004693E000690003A1BAD
:106B3200EA00791E0002792E0004793E00069F4485
:106B42009F5590003A0BEA00691E0002692E00046C
:106B5200693E000612B7C1501F90003A0BEA8069E5
:106B62009E000269AE000469BE00067E04BFF06D9D
:106B7200119F1112B612803A9F449F5590003A0B12
:106B8200EA00691E0002692E0004693E000612B77F
:106B9200C1403190003A0BEA80699E000269AE0062
:106BA2000469BE00067E0440767E1480009F1112A6
:106BB200B4FD9000421BEA00791E0002792E000407
:106BC200793E0006907985693E00020BEA20907BAF
:106BD20062793E00021BEA2090004A0BEA00691E1D
:106BE2000002692E0004693E0006907B5A1BEA00EF
:106BF200791E0002792E0004793E00067E14F3AA63
:106C02007E0400FF12B95E7E14F3B77E0400FF7E9D
:106C12003479437E24000112659890794F1BEA0073
:106C2200791E0002792E0004793E00069079430B0A
:106C3200EA304D33682490794F0BEA00691E000256
:106C4200692E0004693E000690004A1BEA00791E84
:106C52000002792E0004793E000690002C0BEA1007
:106C62009079571BEA10907989693E00020BEA205D
:106C7200907B62793E00021BEA205E1400081E141B
:106C82001E141E143E143E142E1479597A31827A3F
:106C92002183693E00020BEA20907B5E793E00026E
:106CA2001BEA207E14F39E7E0400FF12B95E7E145E
:106CB20079457E040001129020907945E04420B489
:106CC2006E0C90002C0BEA304E340008800DB47329
:106CD2000D90002C0BEA305E34FFF71BEA309079FE
:106CE20046E0442090002EB461090BEA304E341085
:106CF2000080070BEA305E34EFFF1BEA3090798D9B
:106D0200693E00020BEA20907B62793E00021BEA98
:106D12002090006B7EEB307404AC3B2E1479617AC8
:106D220031827A2183693E00020BEA20907B5E79F0
:106D32003E00021BEA207E14F3947E0400FF12B987
:106D42005E7E14F3B77E0400FF7E3479437E240016
:106D5200011265CB7D73BE74012C7803E48030BED2
:106D62007404B0780474018026BE740960780474D7
:106D720002801CBE7412C0780474038012BE742593
:106D820080780474048008BE744B00780674059001
:086D9200006BF0DA79DAD82277
:10475600CA3B7E14F36E7E0400FF1206237E14F31A
:10476600587E0400FF1206237E14F32C7E0400FFFD
:1047760012062312044B7E350C9079611BEA307EBB
:10478600410E9079637AEB409000557EEB5090791C
:10479600647AEB509000567EEBC09000577EEBD0CB
:1047A6009000587EEBE07CB47C4C7C3D7C2E12560F
:1047B600147E14F3197E0400FF1206237E350C9036
:1047C6007B641BEA30E50E907B63F0900055E09029
:1047D6007B62F0900056E0907B61F0900057E0908D
:1047E6007B60F0900058E0907B5FF090767C0BEA5F
:1047F60000691E0002692E0004693E0006907B5780
:104806001BEA00791E0002792E0004793E00067E1E
:1048160014F2EE7E0400FF12B95E20980302477977
:1048260012D4B37CFB4EF020BEF079780A90E00DEE
:10483600E04408F0024927BEF071780302492712C6
:10484600044B7E14F2C17E0400FF1206237E350C53
:10485600907B641BEA30E50E907B63F0900055E098
:10486600907B62F0900056E0907B61F0900057E0FC
:10487600907B60F0900058E0907B5FF07E14F29D94
:104886007E0400FF12B95E7E14F2757E0400FF12EC
:104896000623E4907948F0E4907945F07E14794354
:1048A6007E0400011290209079487EEBA090794515
:1048B600E04CBAB42F609079517EEBA090794EE02F
:1048C6004CBAB43A51740790E00FF0740490E00FBC
:1048D600F090E00DE054FEF0740490E00FF07E34AA
:1048E60079437E240001907B62793E00021BEA2018
:1048F6007E14F2637E0400FF12B95E7E14F24B7ED4
:104906000400FF12062312D4B37E1479437E0400FA
:1049160001120191800B7E14F2367E0400FF12060E
:0449260023DA3B2233
:10822900CA3B7D637E34FB4F7E2400FF7E1479CBED
:108239007E040001740812D1187E34FB577E240095
:10824900FF7E1479D37E040001740812D1187E349C
:10825900FB5F7E2400FF7E1479DB7E0400017450ED
:1082690012D1187E34FBAF7E2400FF7E147A2B7E58
:10827900040001741412D1187E14F0517E0400FF19
:108289001206239079DB693E00020BEA20907B629B
:10829900793E00021BEA207E340014AD362E3401EB
:1082A900777E240001907B5E793E00021BEA207EE6
:1082B90014F0477E0400FF12B95E7E1479AB7E0488
:1082C90000011290204D3368197E140014AD162E4A
:1082D9001401777E0400017E3479AB7E24000112FB
:1082E900D607907A13693E00020BEA20907B6279E7
:1082F9003E00021BEA207D363E342E3406277A7171
:10830900827A61830BEA30907B601BEA307E14F03D
:10831900407E0400FF12B95E7E14F0397E0400FF2E
:108329007E3479457E24000112659812B8837D73E5
:108339009079450BEA304D3368117D363E342E3441
:1083490006277A71827A61831BEA709079DF693E28
:1083590000020BEA20907B62793E00021BEA207D35
:10836900563E543E543E542E54069F7AB1827AA109
:10837900830BEA00691E0002692E0004693E0006AB
:10838900907B5A1BEA00791E0002792E0004793E7F
:1083990000067E14F02F7E0400FF12B95E7E14F0F1
:1083A900297E0400FF7E3479457E240001126598F8
:1083B9009079BF1BEA00791E0002792E0004793EEC
:1083C90000069079450BEA304D3368339079BF0B3D
:1083D900EAC069DE000269EE000469FE00067D3626
:1083E9003E343E343E342E34069F7A71827A61835C
:1083F9001BEAC079DE000279EE000479FE000690DE
:1084090079E3693E00020BEA20907B62793E000223
:108419001BEA207D163E143E142E140FFF7A31827A
:108429007A2183693E00020BEA20907B5E793E0047
:10843900021BEA207E14F0207E0400FF12B95E7E42
:1084490014F01A7E0400FF7E3479457E240001125F
:10845900659812B9279079C7793E00021BEA2090E6
:1084690079450BEA304D3368269079C7693E000299
:108479000BEA2012CF317F017D363E343E342E3453
:108489000FFF7A71827A6183791E00021BEA0090DC
:1084990079E7693E00020BEA20907B62793E00028F
:1084A9001BEA207D563E543E543E542E54087F7A92
:1084B900B1827AA1830BEA00691E0002692E0004C9
:1084C900693E0006907B5A1BEA00791E0002792E4C
:1084D9000004793E00067E14F0107E0400FF12B9F4
:1084E9005E7E14F00A7E0400FF7E3479457E240006
:1084F900011265989079BF1BEA00791E0002792E56
:108509000004793E00069079450BEA304D33683313
:108519009079BF0BEAC069DE000269EE000469FECA
:1085290000067D363E343E343E342E34087F7A715F
:10853900827A61831BEAC079DE000279EE00047950
:10854900FE00069079EB693E00020BEA20907B62FF
:10855900793E00021BEA207D563E543E543E542E7D
:10856900540A5F7AB1827AA1830BEA00691E00027C
:10857900692E0004693E0006907B5A1BEA00791EA9
:108589000002792E0004793E00067E14F02F7E0445
:1085990000FF12B95E7E14F0047E0400FF7E347978
:1085A900457E2400011265989079BF1BEA00791E67
:1085B9000002792E0004793E00069079450BEA30D5
:1085C9004D3368339079BF0BEAC069DE000269EE6A
:1085D900000469FE00067D363E343E343E342E34B6
:1085E9000A5F7A71827A61831BEAC079DE000279B7
:1085F900EE000479FE00069079EF693E00020BEA6D
:1086090020907B62793E00021BEA207D563E543E53
:10861900543E542E540C3F7AB1827AA1830BEA005E
:10862900691E0002692E0004693E0006907B5A1BF0
:10863900EA00791E0002792E0004793E00067E14B4
:10864900F0107E0400FF12B95E7E14EFFE7E040076
:10865900FF7E3479457E2400011265989079BF1B0D
:10866900EA00791E0002792E0004793E000690790D
:10867900450BEA304D3368339079BF0BEAC069DEA8
:10868900000269EE000469FE00067D363E343E3480
:108699003E342E340C3F7A71827A61831BEAC079A9
:1086A900DE000279EE000479FE00069079F3693E56
:1086B90000020BEA20907B62793E00021BEA207DD2
:1086C900563E543E543E542E540E1F7AB1827AA11E
:1086D900830BEA00691E0002692E0004693E000648
:1086E900907B5A1BEA00791E0002792E0004793E1C
:1086F90000067E14EFF47E0400FF12B95E7E14EFCB
:10870900EE7E0400FF7E3479457E240001126598CF
:108719009079BF1BEA00791E0002792E0004793E88
:1087290000069079450BEA304D3368339079BF0BD9
:10873900EAC069DE000269EE000469FE00067D36C2
:108749003E343E343E342E340E1F7A71827A618370
:108759001BEAC079DE000279EE000479FE0006907A
:1087690079F7693E00020BEA20907B62793E0002AC
:108779001BEA207D563E543E543E542E5410EF7A47
:10878900B1827AA1830BEA00691E0002692E0004F6
:10879900693E0006907B5A1BEA00791E0002792E79
:1087A9000004793E00067E14F0107E0400FF12B921
:1087B9005E7E14EFE87E0400FF7E3479457E240056
:1087C900011265989079BF1BEA00791E0002792E83
:1087D9000004793E00069079450BEA304D33683341
:1087E9009079BF0BEAC069DE000269EE000469FEF8
:1087F90000067D363E343E343E342E3410EF7A7115
:10880900827A61831BEAC079DE000279EE0004797D
:10881900FE00069079FB693E00020BEA20907B621C
:10882900793E00021BEA207D563E543E543E542EAA
:108839005412CF7AB1827AA1830BEA00691E000231
:10884900692E0004693E0006907B5A1BEA00791ED6
:108859000002792E0004793E00067E14F0107E0491
:1088690000FF12B95E7E14EFE27E0400FF7E3479C8
:10887900457E2400011265989079BF1BEA00791E94
:108889000002792E0004793E00069079450BEA3002
:108899004D3368339079BF0BEAC069DE000269EE97
:1088A900000469FE00067D363E343E343E342E34E3
:1088B90012CF7A71827A61831BEAC079DE0002796C
:1088C900EE000479FE00069079FF693E00020BEA8A
:1088D90020907B62793E00021BEA207D563E543E81
:1088E900543E542E5414AF7AB1827AA1830BEA0014
:1088F900691E0002692E0004693E0006907B5A1B1E
:10890900EA00791E0002792E0004793E00067E14E1
:10891900EFDB7E0400FF12B95E7E14EFD67E040001
:10892900FF7E3479457E2400011265989079BF1B3A
:10893900EA00791E0002792E0004793E000690793A
:10894900450BEA304D3368339079BF0BEAC069DED5
:10895900000269EE000469FE00067D363E343E34AD
:108969003E342E3414AF7A71827A61831BEAC0795E
:10897900DE000279EE000479FE0006907A03693E72
:1089890000020BEA20907B62793E00021BEA207DFF
:10899900563E543E543E542E54168F7AB1827AA1D3
:1089A900830BEA00691E0002692E0004693E000675
:1089B900907B5A1BEA00791E0002792E0004793E49
:1089C90000067E14EFCC7E0400FF12B95E7E14EF20
:1089D900C67E0400FF7E3479457E24000112659825
:1089E9009079BF1BEA00791E0002792E0004793EB6
:1089F90000069079450BEA304D3368339079BF0B07
:108A0900EAC069DE000269EE000469FE00067D36EF
:108A19003E343E343E342E34168F7A71827A618325
:108A29001BEAC079DE000279EE000479FE000690A7
:108A39007A27693E00020BEA20907B62793E0002A8
:108A49001BEA207D563E543E543E542E5423EB7A65
:108A5900B1827AA1830BEA00691E0002692E000423
:108A6900693E0006907B5A1BEA00791E0002792EA6
:108A79000004793E00067E14EFBC7E0400FF12B9A3
:108A89005E7E14EFB67E0400FF7E3479457E2400B5
:108A9900011265989079BF1BEA00791E0002792EB0
:108AA9000004793E00069079450BEA304D3368336E
:108AB9009079BF0BEAC069DE000269EE000469FE25
:108AC90000067D363E343E343E342E3423EB7A7133
:108AD900827A61831BEAC079DE000279EE000479AB
:108AE900FE0006907A1F693E00020BEA20907B6225
:108AF900793E00021BEA207D563E543E543E542ED8
:108B090054202B7AB1827AA1830BEA00691E0002F4
:108B1900692E0004693E0006907B5A1BEA00791E03
:108B29000002792E0004793E00067E14EFCC7E0403
:108B390000FF12B95E7E14EFA97E0400FF7E34792E
:108B4900457E2400011265989079BF1BEA00791EC1
:108B59000002792E0004793E00069079450BEA302F
:108B69004D3368339079BF0BEAC069DE000269EEC4
:108B7900000469FE00067D363E343E343E342E3410
:108B8900202B7A71827A61831BEAC079DE0002792F
:108B9900EE000479FE0006907A07693E00020BEAAE
:108BA90020907B62793E00021BEA207D563E543EAE
:108BB900543E543E543E547D452E44186F7A91825A
:108BC9007A81830BEA00691E0002692E0004693E5E
:108BD9000006907B5A1BEA00791E0002792E0004D8
:108BE900793E00067D452E4418777A91827A8183F1
:108BF9000BEA00691E0002692E0004693E00069016
:108C09007B521BEA00791E0002792E0004793E008E
:108C1900067D452E44187F7A91827A81830BEA007A
:108C2900691E0002692E0004693E0006907B4A1BFA
:108C3900EA00791E0002792E0004793E00062E54BE
:108C490018877AB1827AA1830BEA00691E0002694A
:108C59002E0004693E0006907B421BEA00791E0043
:108C690002792E0004793E00067E14EF847E04000A
:108C7900FF12B95E7E1479477E0400011290204DDF
:108C890033686D7D363E343E343E343E343E347D69
:108C9900132E14186F7E040001907B62791E000266
:108CA9001BEA007D132E1418777E040001907B5E69
:108CB900791E00021BEA007D132E14187F7E040022
:108CC90001907B5A791E00021BEA002E3418877E18
:108CD900240001907B56793E00021BEA207E14791C
:108CE900477E0400017E34EF747E2400FF12B9AC84
:108CF900907A23693E00020BEA20907B62793E005C
:108D0900021BEA207D563E543E543E542E54220BFB
:108D19007AB1827AA1830BEA00691E0002692E00EA
:108D290004693E0006907B5A1BEA00791E0002790D
:108D39002E0004793E00067E14EFCC7E0400FF125B
:108D4900B95E7E14EF677E0400FF7E3479457E2488
:108D590000011265989079BF1BEA00791E0002791B
:108D69002E0004793E00069079450BEA304D3368B0
:108D7900339079BF0BEAC069DE000269EE0004692D
:108D8900FE00067D363E343E343E342E34220B7AC4
:108D990071827A61831BEAC079DE000279EE0004F0
:108DA90079FE0006907A0B693E00020BEA20907B5F
:108DB90062793E00021BEA207D362E3426077A713D
:108DC900827A61837EEB307404AC3B2E147A2B7A61
:108DD90031827A2183693E00020BEA20907B5E7919
:108DE9003E00021BEA207E14EF5B7E0400FF12B9ED
:108DF9005E7E1479AB7E0400011290204D336838F1
:108E09009079ABE04420249D681824FD681824F863
:108E1900681824F968082409781E7401800D740201
:108E290080097403800574048001E47D362E34269C
:108E3900077A71827A6183F0907A0F693E00020B9A
:108E4900EA20907B62793E00021BEA207D362E34AF
:108E590025CB7A71827A61837EEB307404AC3B2E28
:108E6900147A2B7A31827A2183693E00020BEA2037
:108E7900907B5E793E00021BEA207E14EF5B7E0444
:108E890000FF12B95E7E1479AB7E040001129020B6
:108E99004D3368389079ABE04420249D681824FD4F
:108EA900681824F8681824F968082409781E7401D8
:108EB900800D740280097403800574048001E47DC7
:108EC900362E3425CB7A71827A6183F0907A1769CC
:108ED9003E00020BEA20907B62793E00021BEA20E9
:108EE9007D363E342E3426437A71827A61830BEAC9
:108EF900105E1400013E143E142E1479CB7A31828F
:108F09007A2183693E00020BEA20907B5E793E005C
:108F1900021BEA207E14EF5B7E0400FF12B95E7E1D
:108F29001479AB7E0400011290204D336841907989
:108F3900ABE04420B463177D263E242E2426437AD1
:108F490051827A41830BEA305E34FFFE8018B46D9A
:108F59001E7D263E242E2426437A51827A41830B94
:108F6900EA304E3400017A51827A41831BEA30900B
:108F79007A1B693E00020BEA20907B62793E00026F
:108F89001BEA207D363E342E3426437A71827A617B
:108F9900830BEA105E1400021E143E143E142E14B4
:108FA90079D37A31827A2183693E00020BEA2090D3
:108FB9007B5E793E00021BEA207E14EF4E7E0400A0
:108FC900FF12B95E7E1479AB7E0400011290204D28
:108FD9003368419079ABE04420B479177D263E246B
:108FE9002E2426437A51827A41830BEA304E34008B
:108FF900028018B46E1E7D263E242E2426437A5103
:10900900827A41830BEA305E34FFFD7A51827A41DC
:07901900831BEA30DA3B2261
:106D9A00CAF87E14EF247E0400FF1206237E14EF45
:106DAA00007E0400FF1206237E14EED87E0400FF44
:106DBA001206237E14EEBF7E0400FF1206237E1401
:106DCA00EE9C7E0400FF1206237E14EE6F7E040002
:106DDA00FF1206237E14EE427E0400FF1206237E73
:106DEA0014EE257E0400FF1206237E14EE027E04B2
:106DFA0000FF1206237E14EDE27E0400FF12062332
:106E0A007E14EDC47E0400FF1206237E14F6CF7EA4
:106E1A000400FF12062312D4B37CFBBEF0393806F5
:106E2A007CBF24D080097CBF4420B471DE7471DA3F
:026E3A00F8223C
:1065FE00CA796D774D776803026699126D9A2400F9
:10660E00682514682714682914682B14682D1468DB
:10661E002F14683114683314683514683F24987841
:10662E00D37E74000180CD127C1580C812669C80CA
:10663E00C312677480BE127AB880B91275F680B430
:10664E0012908580AF12929780AA12492A80A57E59
:10665E0014ED947E0400FF12062380987E14F5B488
:10666E007E0400FF12062312D4B34420B47919120B
:10667E00596D7E14ED677E0400FF12062312D4B30B
:0E668E004420B47903125C3A026602DA7922E3
:10492A00CAD8CA796D777E14ED3C7E0400FF120660
:10493A002312D4B3442024977803024A4B24F06804
:10494A004F240E6803024B46E49076E2F07E14EDA3
:10495A00057E0400FF12062312D4B34420B479233F
:10496A007E14ECD17E0400FF1206237E14ECA57E91
:10497A000400FF12062390002E0BEA304E3400206A
:10498A00024A4590002E0BEA305E34FFDF024A45A8
:10499A0074019076E2F07E14EC797E0400FF120630
:1049AA002312D4B324CE681F1468410BB178637400
:1049BA002E9076E3F0741E9076E4F09000300BEAC5
:1049CA00304E340002803B74219076E3F0741190EB
:1049DA0076E4F09000300BEA305E34FFFD1BEA30DB
:1049EA009000300BEA304E34000480237401907634
:1049FA00E4F074019076E3F09000300BEA305E3414
:104A0A00FFFD1BEA309000300BEA305E34FFFB1BDF
:104A1A00EA307E14EC5D7E0400FF12062312D4B342
:104A2A004420B4790C90002C0BEA304E34004080BC
:104A3A000A90002C0BEA305E34FFBF1BEA30024BAF
:104A4A004674029076E2F09076E5E00A3B907B6449
:104A5A001BEA307E14EC327E0400FF12B95E7E142B
:104A6A0079437E0400011290204D3368257E347606
:104A7A00E57E240001907B62793E00021BEA207EDB
:104A8A001479437E0400017E34EC2E7E2400FF124A
:104A9A00B9AC9076E6E00A3B907B641BEA307E1460
:104AAA00EC057E0400FF12B95E7E1479437E040091
:104ABA00011290204D3368257E3476E67E2400016B
:104ACA00907B62793E00021BEA207E1479437E04C1
:104ADA0000017E34EC2E7E2400FF12B9AC7E14EB6A
:104AEA00EC7E0400FF12B95E12D4B3442090003069
:104AFA00B479090BEA304E34001080070BEA305EB5
:104B0A0034FFEF1BEA30900052E00A3B907B641BB3
:104B1A00EA307E14EBCC7E0400FF12B95E7E14EB01
:104B2A00C27E0400FF7E3479577E2400011265CBD1
:104B3A007CB77CDB60069000527AEBD07E14EB9651
:104B4A007E0400FF7E3479577E2400011265CB7DF6
:104B5A0073BE74258078047403801BBE744B00787E
:104B6A000474048011BE7412C0780474028007BEF3
:104B7A007404B07805E490006CF0C2CA90006C7EB0
:104B8A00EB707402AC7B2E3400617A71827A618395
:104B9A000BEA307D235E24FF000A54F5CBF5CD7D68
:104BAA00535E5400FFF5CAF5CCD2CA7E14EB6F7E71
:104BBA000400FF12062312D4B3442024926810245E
:104BCA00F5781990002C0BEA304E342000800A90B8
:104BDA00002C0BEA305E34DFFF1BEA307E14EB4414
:104BEA007E0400FF12062312D4B344202492683AAA
:104BFA0024F5681D2407784C90002C0BEA304E34BB
:104C0A0040001BEA3090002E0BEA304E3400108030
:104C1A003090002C0BEA304E3440001BEA309000F2
:104C2A002E0BEA305E34FFEF801790002C0BEA302F
:104C3A005E34BFFF1BEA3090002E0BEA305E34FF71
:104C4A00EF1BEA307E14EB127E0400FF12062312D9
:104C5A00D4B34420249F681024FB781990002C0BAD
:104C6A00EA304E340080800A90002C0BEA305E3421
:0A4C7A00FF7F1BEA30DA79DAD82256
:10449F00CAF87E350C907B641BEA30E50E907B6387
:1044AF00F0900055E0907B62F07E14EACF7E04001E
:1044BF00FF12B95E7E14EA7E7E0400FF1206237E91
:1044CF0014EA6F7E0400FF1206236CFF80340A3F4C
:1044DF002E3427AB7A71827A6183E01A2B7E3400F7
:1044EF0014AD322E3401777E240001907B62793E29
:1044FF0000021BEA207E14EA697E0400FF12B95EF7
:10450F000BF090792CE0BCBF38C47CFB800D7E147F
:10451F00EA5B7E0400FF1206230BF0BEF00540EEAF
:0E452F007E14EA587E0400FF120623DAF822FA
:10453D007E350C907B641BEA30E50E907B63F0902A
:10454D000055E0907B62F07E14EA177E0400FF12A6
:10455D00B95E7E14E9CC7E0400FF1206237E14E9B9
:10456D00817E0400FF1206237E14E9377E0400FFCE
:10457D0012062390002C0BEA305E340200680A7E8E
:10458D0014E8FA7E0400FF80087E14EA587E0400C9
:10459D00FF12062390792BE01A3B2E3427AB7A714C
:1045AD00827A6183E01A2B7E340014AD322E3401F1
:1045BD00777E240001907B62793E00021BEA207E0B
:1045CD0014E8E37E0400FF12B95E7E14E8947E04C5
:1045DD0000FF12B95E7E14E8477E0400FF12B95E3B
:0145ED0022AB
:10326000CA3B7EE0206D669F007D363E343E347D55
:10327000232E2479807A51827A4183791E00021BA1
:10328000EA002E34796C7A71827A6183791E0002A9
:103290001BEA000B64BE64000578CCE4907943F02F
:1032A0006CFF90002E0BEA304E3404001BEA309085
:1032B000002C0BEA305E340100681E12A99B1490AA
:1032C0007943F0BEB000480E90792C7EEBA0907947
:1032D00043E0BCBA4852E4804B124DA290792B7E59
:1032E000EBA0BEA0FF78030238961A3A2E3427AB23
:1032F0007A71827A6183E0BEB000480890792CE050
:10330000BCAB481C90792CE00A3B907B641BEA30F4
:103310007E14E8077E0400FF12B95EE490792BF07A
:1033200090792BE0907943F09079297EEBA0907909
:103330002CE0BCBA280690792C7AEBA0907943E077
:103340001A3B2E3427AB7A71827A6183E0907944FC
:10335000F012B3AA12449F90E102E054F0F0900002
:103360002C0BEA307D235E24000468105E340800D4
:1033700068057EE02680087EE02180037EE0206DE7
:10338000660238867D362E3427AB7A71827A618365
:103390007EEBF0BEF0005803023886BEF03C080316
:1033A0000238867CBF12067212044B7CBF12141FB7
:1033B0009078E10BEA00691E0002692E0004693E64
:1033C000000612B9277F717DD63ED43ED47D3D2EB6
:1033D00034796C7A71827A618379FE00021BEAE0AB
:1033E0009078D10BEA00691E0002692E0004693E44
:1033F000000612B9277F017D3D2E3479807A7182D3
:103400007A6183791E00021BEA00907944E0BCFBDC
:10341000782990796479FE00021BEAE09078D10B5C
:10342000EA00691E0002692E0004693E000612B916
:1034300027907968793E00021BEA20E590541078C5
:103440000612909D02368B0A3E907B641BEA3090F8
:103450000056E0907B63F0900057E0907B62F09024
:103460000058E0907B61F07E14E7F17E0400FF12CB
:10347000B95E90796C693E00020BEA2012B8E590C3
:103480007B5E1BEA00791E0002792E0004793E0063
:1034900006907980693E00020BEA2012B8E5907B25
:1034A000561BEA00791E0002792E0004793E0006C0
:1034B000907970693E00020BEA2012B8E5907B4ECD
:1034C0001BEA00791E0002792E0004793E00069066
:1034D0007984693E00020BEA2012B8E5907B461B16
:1034E000EA00791E0002792E0004793E00067E145F
:1034F000E7D87E0400FF12B95E907974693E00023D
:103500000BEA2012B8E5907B5E1BEA00791E0002F0
:10351000792E0004793E0006907988693E00020BFE
:10352000EA2012B8E5907B561BEA00791E0002796A
:103530002E0004793E0006907978693E00020BEA7D
:103540002012B8E5907B4E1BEA00791E0002792E0E
:103550000004793E000690798C693E00020BEA2057
:1035600012B8E5907B461BEA00791E0002792E0016
:1035700004793E00067E14E7BF7E0400FF12B95EA8
:1035800090797C693E00020BEA2012B8E5907B5EE0
:103590001BEA00791E0002792E0004793E00069095
:1035A0007990693E00020BEA2012B8E5907B561B29
:1035B000EA00791E0002792E0004793E00067E148E
:1035C000E7B17E0400FF12B95E7480120218900009
:1035D00056E0907A90F0900057E0907A8FF090004B
:1035E00058E0907A8EF00A3E907A8C1BEA309079FF
:1035F00044E01A2B7E340014AD322E3401777E2441
:103600000001907A88793E00021BEA207E147946F8
:103610007E0400017E34E7997E2400FF12B98A7E81
:103620001479467E04000112043674C01202189008
:103630007964693E00020BEA2012B8E5907A891B92
:10364000EA00791E0002792E0004793E0006907986
:1036500068693E00020BEA2012B8E5907A811BEA05
:1036600000791E0002792E0004793E00067E14794E
:10367000467E0400017E34E7847E2400FF12B98A6E
:103680007E1479467E04000112043690002C0BEA69
:10369000305E340100686912A99B907945F0701082
:1036A00090002C0BEA305E34FDFF1BEA30023896A6
:1036B000907945E014F090792CE09079457EEBA06C
:1036C000BCAB480A9027ABE0907944F080201A3ACE
:1036D0002E3427AB7A71827A61837EEBA090794495
:1036E000E0BCAB68099079447AEBA002335E90E1CC
:1036F00001E064FF0A3B5E340010682D80378029AA
:1037000030986F12D4B34420249B681124F5683498
:1037100014785F90E102E054DFF002389690002CBC
:103720000BEA305E340004680C90002C0BEA305E2B
:1037300034FFFB800A90002C0BEA304E3400041B4F
:10374000EA30802E90002C0BEA305E3408006812BC
:1037500090002C0BEA305E34F7FF1BEA307EE0214C
:10376000801090002C0BEA304E3408001BEA307EAB
:10377000E0269076DA693E00020BEA2012B8E57F77
:10378000407F519078D10BEA00691E0002692E003B
:1037900004693E000612B7C1283E90002C0BEA30A7
:1037A0005E34000468327CBD90792BF07E14F9877A
:1037B0007E0400FF12062390002C0BEA305E34FBDF
:1037C000FF1BEA3012389990002C0BEA305E34046B
:1037D00000680302389680657E84C0086D999F5505
:1037E0009078D10BEA00691E0002692E0004693E40
:1037F000000612B7C1401A90E000E0540168099039
:10380000E102E04420F0803590E102E054DFF080F6
:103810002C90E102E054DFF090002C0BEA307D2385
:103820005E240010680D5E34000468077CBF12B38C
:10383000E7800A90E102E054F0F012B3AA90002E63
:103840000BEAF07DEF5EE40040683990792BE01AD6
:103850001B3E143E142E1479807A31827A218369BA
:103860003E00020BEA209076DE691E00020BEA00A1
:1038700012CEAC500F43904090002E7D3F5E34FF3F
:10388000BF1BEA300B6490792CE00A3BBD3628035D
:0938900002338402335EDA3B22AC
:10389900CA3B7420907A18F07EE02A90002C0BEA3B
:1038A900307D235E2402006816740A90E00EF05EF3
:1038B90034080068057EE026800F7EE021800A7EBC
:1038C900E02A90E00EE04401F090E102E054DFF0DC
:1038D90090002C0BEA307D235E240100681C5E34C5
:1038E9000200781612A99B1490792BF0BEB00048FB
:1038F900DF90792BE0BEB03C18D690002E0BEA3051
:103909004E3404801BEA3090002E0BEA305E345F9F
:10391900FF1BEA3090E00DE054FBF090792BE0902A
:1039290079F7F01A3B2E3427AB7A71827A6183E0FA
:10393900BEB000489B7CFB12067290792BE01A1BE3
:103949003E143E142E1426BB7A31827A2183693EB5
:1039590000020BEA209076F1793E00021BEA2090E2
:1039690076E2E0B40160E46C7712A9809000300B34
:10397900EA305E340002683474C912004774601278
:103989000047E4120047E41200479076E4E0120091
:103999004774051200477410120047E4120047E407
:1039A9001200479076E4E012004780139000300B34
:1039B900EA305E3400046807E47E704E12A980E4A0
:1039C9007E708012A980907709693E00020BEA2077
:1039D9009076E9793E00021BEA2090770D693E0056
:1039E900020BEA209076ED793E00021BEA207CBFAB
:1039F90012A27F7E843FB97E9499997EA499997E7B
:103A0900B4999A9076740BEA00691E0002692E0037
:103A190004693E000612B7C128057CBF12A7177EAC
:103A2900843FB97E9499997EA499997EB4999A9084
:103A3900766C0BEA00691E0002692E0004693E00DB
:103A49000612B7C128057CBF12A4E77E18000A90A8
:103A59007701793E00021BEA20907706E0B4040E54
:103A69007E180064907701793E00021BEA2012B3A8
:103A7900AA12453D90E102E054F0F090002C0BEAC7
:103A8900307D235E2400046808907A177AEBE08081
:103A9900067420907A17F05E340100687812A99BA9
:103AA9009079F6F090002C0BEA307D235E24020019
:103AB900782B9079F6E0700B90002C7D234E240230
:103AC9000080299079F614F090792B7EEBA09079FB
:103AD900F6E0BCBA681C90792BF00238D99079F6D7
:103AE900E0700F90002C7D235E24FDFF1BEA20026D
:103AF900449C90E101E064FF0A2B5E240010680FEA
:103B090090002C7D234E2400041BEA20023D2890BE
:103B1900002C023D37209803023DEF12D4B390796F
:103B2900F8F0442024E07803023C5124F878030299
:103B39003C7024FD7803023D561BB17803023D66B3
:103B490024FD7803023D981BB1686C147803023B8D
:103B5900E3147803023C0624F57803023DA624DA2F
:103B69007803023D0F1BB27803023DE024FB780382
:103B7900023CB21BB17803023CCE147803023C8AA2
:103B890024FD7803023DDE24FB7803023D492448E5
:103B99006803023DEFE41A3F7D232E241FEF7A517B
:103BA900827A4183F07D533E543E543E543E543E06
:103BB900542E54186F806774011A3F7D232E241FD9
:103BC900EF7A51827A4183F07D533E543E543E54FC
:103BD9003E543E542E541877804474021A3F7D2374
:103BE9002E241FEF7A51827A4183F07D533E543E51
:103BF900543E543E543E542E54187F802174031A67
:103C09003F7D232E241FEF7A51827A4183F07D5321
:103C19003E543E543E543E543E542E5418877AB175
:103C2900827AA1830BEA00691E0002692E000469E9
:103C39003E00069076741BEA00791E0002792E0078
:103C490004793E0006023DEF90792BE004F090796B
:103C59002A7EEBA090792BE0BCBA5803023DEF9085
:103C6900792B14F0023DEF90792BE014F090792B29
:103C7900E0BEB0004803023DEF90792B04F0023D0D
:103C8900EF90E102E054F0F090E102E054DFF090AF
:103C9900002E0BEA305E34DFFF1BEA3090002C0B5C
:103CA900EA304E3404000241F590002C0BEA305EF4
:103CB9003402007803023DEF90E102E054DFF01294
:103CC900449F02449C90002C0BEA305E3402007839
:103CD90003023DEF90002C0BEA305E3408006813B4
:103CE90090002C0BEA305E34F7FF1BEA307EE021AE
:103CF900023DEF90002C0BEA304E3408001BEA30ED
:103D09007EE026023DEF90002C0BEA305E34000481
:103D1900781690002C0BEA304E3400041BEA3090E0
:103D29007A177AEBE0023DEF90002C0BEA305E3413
:103D3900FFFB1BEA30907A18E0907A17F0023DEF0A
:103D490012B3AA90E00DE04408F0023DEF9076F13D
:103D5900691E00020BEA002E08000A800E9076F117
:103D6900691E00020BEA009E08000A791E00021B68
:103D7900EA0090792BE01A3B3E343E342E3426BBC0
:103D89007A71827A6183791E00021BEA0080579F4B
:103D9900119076F1793E00021BEA20804990792B37
:103DA900E01A3B2E3427AB7A71827A6183E01A2BB1
:103DB9007E340014AD322E3401777E240001907BCD
:103DC90062793E00021BEA207E14E77D7E0400FF33
:103DD90012B95E801180057CBF12A27F7CBF12A739
:103DE900177CBF12A4E790792B7EEBA09079F7E0BE
:103DF900BCBA680302390312044B7CBF12141F902A
:103E090078E10BEA00691E0002692E0004693E0090
:103E19000612B9279076B2793E00021BEA20907803
:103E2900D10BEA00691E0002692E0004693E0006F2
:103E390012B9279076B6793E00021BEA201A3F1282
:103E49007014E5905410780612909D024154907AAE
:103E590017E00A3B907B641BEA30900056E0907BA8
:103E690063F0900057E0907B62F0900058E0907BFF
:103E790061F07E14E7687E0400FF12B95E9078E174
:103E89000BEA00691E0002692E0004693E000690D3
:103E99007B5E1BEA00791E0002792E0004793E0040
:103EA900069078D10BEA00691E0002692E000469A8
:103EB9003E0006907B561BEA00791E0002792E000F
:103EC90004793E00069078A90BEA00691E00026990
:103ED9002E0004693E0006907B4E1BEA00791E0005
:103EE90002792E0004793E00067E8440B87E94EA69
:103EF900287EA4F5C27EB48F5C9077E90BEA00694D
:103F09001E0002692E0004693E000612B4FD907B72
:103F1900461BEA00791E0002792E0004793E00064C
:103F29007E14E7537E0400FF12B95E9078E90BEA2C
:103F390000691E0002692E0004693E0006907B5E3E
:103F49001BEA00791E0002792E0004793E000690D2
:103F590078F10BEA00691E0002692E0004693E002F
:103F690006907B561BEA00791E0002792E0004791F
:103F79003E00069077B90BEA00691E0002692E001F
:103F890004693E0006907B4E1BEA00791E00027907
:103F99002E0004793E00069079010BEA00691E00A3
:103FA90002692E0004693E0006907B461BEA0079EF
:103FB9001E0002792E0004793E00067E14E73D7E3C
:103FC9000400FF12B95E9076F1693E00020BEA2007
:103FD9007CB412B834907B5E1BEA00791E0002792A
:103FE9002E0004793E00067E14E7337E0400FF129A
:103FF900B95E7480120218900056E0907A90F090A1
:104009000057E0907A8FF0900058E0907A8EF07E19
:104019001479F97E0400017E34E7217E2400FF1221
:10402900B98A7E1479F97E040001120436907A1750
:10403900E00A3B907A8F1BEA3090792BE01A3B2EED
:104049003427AB7A71827A6183E01A2B7E340014AB
:10405900AD322E3401777E240001907A8B793E00AF
:10406900021BEA207E1479F97E0400017E34E718E8
:104079007E2400FF12B98A7E1479F97E04000112A8
:10408900043674C012021890792BE01A3B2E34279B
:10409900AB7A71827A6183E01A3B3E342E3426432F
:1040A9007A71827A61830BEA305E3400029078E19A
:1040B9000BEA00691E0002692E0004693E000690A1
:1040C9007A891BEA00791E0002792E0004793E00E4
:1040D900069078D10BEA00691E0002692E00046976
:1040E9003E0006907A811BEA00791E0002792E00B3
:1040F90004793E000668369077B90BEA00691E001C
:1041090002692E0004693E0006907A791BEA00795B
:104119001E0002792E0004793E00067E1479F97E8C
:104129000400017E34E6FF7E2400FF80107E1479AE
:10413900F97E0400017E34E6E97E2400FF12B98A83
:104149007E1479F97E0400011204369076DA693E0C
:1041590000020BEA2012B8E57F407F519078D10B1D
:10416900EA00691E0002692E0004693E000612B7C2
:10417900C140415390BF90002E0BEA304E340040AD
:104189001BEA3090002E0BEA307D235E2440007834
:104199000302424C90002C0BEA205E2400047803B1
:1041A90002424C5E348000680302424C7CBF12B06C
:1041B900E202424C90002C0BEA305E340200683275
:1041C90090E102E054F0F012449F7E14F9877E04D6
:1041D90000FF12062390002E0BEA304E3404001B18
:1041E900EA3090002E0BEA305E34DFFF1BEA300222
:1041F900449C90002E0BEAF07DEF5EE4004068439A
:104209009076DE693E00020BEA2012B8E57F407F16
:10421900519078D10BEA00691E0002692E000469E9
:104229003E000612B7C1381B4390409F119076F1AA
:10423900793E00021BEA2090002E7D3F5E345FBF6D
:104249001BEA3090002E0BEA305E340080682D9F07
:10425900449F559076B6693E00020BEA2012B8E5F4
:1042690012B7C128177CBF12A27F7CBF12A7179073
:10427900002E0BEA305E34FF7F1BEA3090002C0BD6
:10428900EA307D235E24000168030243495E34005D
:1042990080781D9076B6693E00020BEA2012B8E5D7
:1042A9007E84C0086D999F5512B7C13803024349EE
:1042B90090770D691E00020BEA009076ED693E00C9
:1042C900020BEA209F1012D4D6BE1800640825906C
:1042D900002C0BEA305E342000681990770D693E96
:1042E90000020BEA209076ED793E00021BEA207C61
:1042F900BF12A717907709691E00020BEA00907692
:10430900E9693E00020BEA209F1012D4D69077018A
:10431900691E00020BEA00BF10282590002C0BEA49
:10432900305E3440006819907709693E00020BEA53
:10433900209076E9793E00021BEA207CBF12A4E7AF
:1043490090791D691E00020BEA00907919693E00F7
:10435900020BEA207F219F209079250BEA106D003E
:10436900BF203810907921695E00020BEA409F1244
:10437900BF10280312AF7C90E00DE05404780302CB
:10438900449190002C0BEA307D235E2408007803C9
:104399000244915E340200780302449190E00DE0FA
:0E43A90054FBF06D6602447F7D362E3427AB48
:1043B7007A71827A6183E09079F5F0BEB000580394
:1043C70002447D9079F5E0BEB03C080302447D903D
:1043D70079F5E012067212044B9079F5E012141F7A
:1043E7007E84C0006D999F559078D10BEA00691EB5
:1043F7000002692E0004693E000612B7C1287790B3
:10440700792BE01A3BBD63503D7C7D90792B7AEB8D
:10441700701A372E3427AB7A71827A6183E01A2BB0
:104427007E340014AD322E3401777E240001907B58
:1044370062793E00021BEA207E14E6C27E0400FF7A
:1044470012B95E02390390792BE01A3BBD63283518
:104457009F009076B6693E00020BEA2012CEAC5060
:104467002490002E0BEA305E34008078187CBD90D3
:10447700792BF00239030B6490792CE00A3BBD637A
:1044870050030243B17CBF1206721A3F1270140226
:084497003A840238D9DA3B2215
:10B3E700CAF87CFB12044B90002E0BEA307D235EDB
:10B3F70024020068775E34040068717EF424007EBE
:10B40700E449749076F5693E00020BEA207F071243
:10B41700CD8B12CF31907709793E00021BEA20903D
:10B4270076F9693E00020BEA207F0712CD8B12CF17
:10B437003190770D793E00021BEA20907707E09064
:10B447007705F0907708E0907706F07CBF12A27F2F
:10B457007CBF12A7177CBF12A4E790002E0BEA301F
:10B467005E34FBFF1BEA307CBF12067290002E0B86
:10B47700EA305E34DFFF1BEA309076BE693E000299
:10B487000BEA209076B6793E00021BEA209076BA46
:10B49700693E00020BEA209076B2793E00021BEA71
:10B4A7002012728090791D691E00020BEA009079C4
:10B4B70019693E00020BEA207F219F209079250B16
:10B4C700EA106D00BF203810907921695E00020BE9
:0EB4D700EA409F12BF10280312AF7CDAF82261
:10B0E200CAF87CFB9078E10BEA00691E0002692E27
:10B0F2000004693E0006907A191BEA00791E0002DC
:10B10200792E0004793E000690E102E054F0F07ED0
:10B112008440246D999F5590764C0BEA00691E007D
:10B1220002692E0004693E000612B7C140127E84F5
:10B132003F567E94C16B7EA4FE527EB46C39801061
:10B142007E843F8C7E9471C57EA4EB067EB448C497
:10B1520090767C0BEA00691E0002692E0004693EAB
:10B16200000612B5011BEA00791E0002792E0004C6
:10B17200793E00067CBF12141F74C01202187E149E
:10B18200E6B17E0400FF12043690002C0BEA305E1A
:10B19200340008680302B2637E8440567E948000C5
:10B1A2009F55907A190BEAC069DE000269EE00042D
:10B1B20069FE00067F067F1712B7C128377E8440DA
:10B1C200667E9480009F557F067F1712B7C1502478
:10B1D2007E8440667E9480009F559078E10BEA0061
:10B1E200691E0002692E0004693E000612B7C128DA
:10B1F2000302B3197E8440707E94E0009F55907ADA
:10B20200190BEA00691E0002692E0004693E00065D
:10B2120012B7C1400302B3257EC440667ED48000CB
:10B222009F77907A190BEA00691E0002692E0004CA
:10B23200693E00067F467F5712B7C1380302B32525
:10B242009078E10BEA00691E0002692E0004693E53
:10B2520000067F467F5712B7C1400302B32502B3EF
:10B26200197E8440707E94E0009F55907A190BEA13
:10B27200C069DE000269EE000469FE00067F067FF7
:10B282001712B7C128347E8440767E9480009F5581
:10B292007F067F1712B7C150217E8440567E94806C
:10B2A200009F559078E10BEA00691E0002692E00AA
:10B2B20004693E000612B7C1405D7E8440567E940A
:10B2C20080009F55907A190BEA00691E0002692ED0
:10B2D2000004693E000612B7C150489F449F559032
:10B2E2007A190BEA00691E0002692E0004693E0009
:10B2F2000612B7C1282D7E8440707E94E0009F55CF
:10B302009078E10BEA00691E0002692E0004693E92
:10B31200000612B7C1280C90002E0BEA304E3420E2
:10B322000080329076DA693E00020BEA2012B8E51C
:10B332007F407F519078D10BEA00691E0002692E8E
:10B342000004693E000612B7C1500F90002E0BEAAE
:10B35200305E34DFFF1BEA3080279078E10BEA0091
:10B36200691E0002692E0004693E0006907A191BCC
:10B37200EA00791E0002792E0004793E000602B12D
:10B382001190002E0BEA304E3480001BEA3012047A
:09B392004B7CBF12141FDAF822F3
:10AF7C00CA3B90002E0BEA305E340800680302B026
:10AF8C005C90E102E054F0F0900056E00A3B907BBC
:10AF9C00641BEA30900057E00A3B907B621BEA305E
:10AFAC00900058E00A3B907B601BEA307E14E65818
:10AFBC007E0400FF12B95E74801202187E14E647FC
:10AFCC007E0400FF12043674C01202187E14E6369A
:10AFDC007E0400FF120436900057E00A7B90005864
:10AFEC00E00A6B90E000E0540190E102E068054457
:10AFFC0020F0800354DFF012044B900057E00A3B22
:10B00C009D37BE3400005806900057243CF0900049
:10B01C00587EEBA00A3ABD3678C99000577EEB708B
:10B02C000A179D179079270BEA20BD1278B590006E
:10B03C0056E0907B65F0907B647AEB70907B637A42
:10B04C00EBA07E14E6077E0400FF12B95E12B3AAD1
:03B05C00DA3B22BA
:10A98000CAF87CF7120047E4120047E4120047E4DB
:0BA990001200477CBF120047DAF822DB
:10B3CC00CAF87CFB74FE12000374FE1200037CBFEF
:0BB3DC001200037402120003DAF822D2
:10A4E700CA3B7CCB9076E2E07066907709693E00C4
:10A4F700020BEA20907A8D793E00021BEA207E1437
:10A507007A1E7E0400017E34E5FC7E2400FF12B92A
:10A517008A90002E0BEA305E34002068251A3C3EF4
:10A52700342E3426437A71827A61830BEA305E34A3
:10A537000008680E7E147A1E7E04000112B4E5023C
:10A54700A7147E147A1E7E0400011293EB02A7144F
:10A557009076E2E0B40102800302A64FE46C771222
:10A56700A9807E08000A907709693E00020BEA205D
:10A5770012D0E4907A1A793E00021BEA20907A8D75
:10A58700793E00021BEA207E147A1E7E0400017EBB
:10A5970034E5F57E2400FF12B98A6CDD6CFF907AF2
:10A5A7001E7EEBC0BEC0317819907A1FE0B432121C
:10A5B700907A207EEBF09EF0305EF00F7CBF44C0B7
:10A5C7008026BEC0307828907A1F7EEBD09ED03090
:10A5D7005ED00F907A207EEBF09EF0305EF00F7C1D
:10A5E700BDC454F054F04CBF907A19F01200477E66
:10A5F700E0036CDD6CFF1A3E7D232E247A1E7A5110
:10A60700827A41837EEBD09ED0305ED00F2E347A93
:10A617001F7A71827A61837EEBF09EF0305EF00FD5
:10A627007CBDC454F054F04CBF907A19F012004727
:10A637000BE1BEE00848BB9076E4E0120047E47EF9
:10A64700708012A98002A7149076E2E0B40202801B
:10A657000302A714907709693E00020BEA20907A5B
:10A667001A793E00021BEA20907A8D793E00021B80
:10A67700EA207E147A1E7E0400017E34E5ED7E24F6
:10A6870000FF12B98A9000300BEA305E3400107870
:10A697001D9076E7E012B3CC740712000374D11251
:10A6A700000374FD120003900052E012007D9076C3
:10A6B700E7E012B3CCE41200037EE0096CDD6CFF27
:10A6C7001A3E7D232E247A1E7A51827A41837EEBAD
:10A6D700F09EF0305EF00F2E347A1D7A71827A6127
:10A6E700837EEBD09ED0305ED00F7CBDC454F05437
:10A6F700F04CBF907A19F01200031BE1BEE000187E
:10A70700BB74FD120003900052E012007DDA3B2279
:10A71700CA3B7CCB9076E2E0600302A7C090770D3E
:10A72700693E00020BEA20907A8D793E00021BEA0F
:10A73700207E147A1A7E0400017E34E5E27E24002E
:10A74700FF12B98A90002E0BEA305E34002068456C
:10A757001A3C3E342E3426437A71827A61830BEA9F
:10A76700305E34000868157E14E5DD7E0400FF12B4
:10A7770093EB7E147A1A7E04000180377E14E5DDA0
:10A787007E0400FF12B4E57E147A1A7E04000112DB
:10A79700B4E502A97D7E14E5DD7E0400FF1293EB8C
:10A7A7007E147A1A7E0400011293EB7E14E5D87E9C
:10A7B7000400FF1293EB02A97D9076E2E0B4010258
:10A7C700800302A8B8E46C7712A9807E08000A907B
:10A7D700770D693E00020BEA2012D0E4907A4279A5
:10A7E7003E00021BEA20907A8D793E00021BEA2088
:10A7F7007E147A1A7E0400017E34E5F57E2400FF7C
:10A8070012B98A6CDD6CFF907A1A7EEBC0BEC0313C
:10A817007819907A1BE0B43212907A1C7EEBF09E86
:10A82700F0305EF00F7CBF44C08026BEC030782871
:10A83700907A1B7EEBD09ED0305ED00F907A1C7E34
:10A84700EBF09EF0305EF00F7CBDC454F054F04C3A
:10A85700BF907A19F01200477EE0036CDD6CFF1A97
:10A867003E7D232E247A1A7A51827A41837EEBD059
:10A877009ED0305ED00F2E347A1B7A71827A618334
:10A887007EEBF09EF0305EF00F7CBDC454F054F0C8
:10A897004CBF907A19F01200470BE1BEE00848BBA5
:10A8A7009076E3E0120047E47E708012A98002A947
:10A8B7007D9076E2E0B40202800302A97D90770DD5
:10A8C700693E00020BEA20907A42793E00021BEAB9
:10A8D70020907A8D793E00021BEA207E147A1A7E38
:10A8E7000400017E34E5ED7E2400FF12B98A900052
:10A8F700300BEA305E340010781D9076E8E012B332
:10A90700CC740712000374D012000374FD12000305
:10A91700900052E012007D9076E8E012B3CCE4128A
:10A9270000037EE0096CDD6CFF1A3E7D232E247A3E
:10A937001A7A51827A41837EEBF09EF0305EF00FF7
:10A947002E347A197A71827A61837EEBD09ED03069
:10A957005ED00F7CBDC454F054F04CBF907A19F010
:10A967001200031BE1BEE00018BB74FD1200039048
:09A977000052E012007DDA3B22DF
:10A27F00CAD8CA797CDB9076E27EEBE04CEE6803BD
:10A28F0002A3A4907705E00A3B907A8F1BEA307EF9
:10A29F00147A197E0400017E34E5D07E2400FF126B
:10A2AF00B98A907706E00A3B907A8F1BEA307E14CA
:10A2BF007A417E0400017E34E5D07E2400FF12B97E
:10A2CF008A90002E0BEA305E340020780302A35FE1
:10A2DF007E7002AC7D2E3426437A71827A61830BB5
:10A2EF00EA305E34000868457E14E5DD7E0400FF29
:10A2FF001293EB7E14E5CB7E0400FF1293EB7E14DA
:10A30F007A197E0400011293EB7E14E5D87E0400C7
:10A31F00FF12B4E57E14E5C67E0400FF12B4E57E9D
:10A32F00147A417E04000112B4E502A4E27E14E522
:10A33F00DD7E0400FF12B4E57E14E5CB7E0400FF42
:10A34F0012B4E57E147A197E04000112B4E580215F
:10A35F007E14E5DD7E0400FF1293EB7E14E5CB7EC9
:10A36F000400FF1293EB7E147A197E0400011293FE
:10A37F00EB7E14E5D87E0400FF1293EB7E14E5C646
:10A38F007E0400FF1293EB7E147A417E04000112CB
:10A39F0093EB02A4E2BEE001786BE46C7712A98024
:10A3AF00907705E060201BB1680C1BB1680D24038A
:10A3BF0078096CFF80087EF00180037EF0087CBF77
:10A3CF007E702712A980907706E01BB1680C1BB135
:10A3DF00680D240378096CFF80197EF001801490BA
:10A3EF00002C0BEA305E34004068057EF088800355
:10A3FF007EF0087CBF7E701712A980E47E708012F9
:10A40F00A98002A4E2BEE002680302A4E290003039
:10A41F000BEA305E340010781D9076E8E012B3CC72
:10A42F00740712000374D012000374FD120003901E
:10A43F000052E012007D9076E8E012B3CC74011266
:10A44F000003907705E01BB1680D14680E14680FB8
:10A45F002403780BE4800A7401800674038002746D
:10A46F000512000374FD120003900052E012007DEC
:10A47F009000300BEA305E340010781D9076E7E0E4
:10A48F0012B3CC740712000374D112000374FD12BF
:10A49F000003900052E012007D9076E7E012B3CCFB
:10A4AF007401120003907706E01BB1680D14680E5B
:10A4BF0014680F2403780BE4800A74018006740378
:10A4CF008002740512000374FD120003900052E025
:08A4DF0012007DDA79DAD822BF
:10044B00CA7912015CE50F0A0B9E0400307E140082
:10045B000AAD10E5100A3B9E3400302D312E3407C7
:10046B006C7A350CE50FBEB039680A7E350C2E342C
:10047B0000647A350C7E71119E70307E600AAC760A
:10048B007E41129E40302C477A410E7E71139E7036
:10049B00307E600AAC767E51149E50302C57900003
:1004AB00557AEB507E71159E70307E600AAC76E506
:1004BB001624D02CB7900056F07E71179E70307EAC
:1004CB00600AAC76E51824D02CB7900057F07E71FB
:1004DB00199E70307E600AAC76E51A24D02CB7904A
:1004EB000058F07E350C7CB41206387D23E412B82C
:1004FB00399076841BEA00791E0002792E0004796C
:10050B003E0006900056E00A3B6D227E080E10124C
:10051B00D0D37CB412B8347F407F51CA4BCA5B7EB8
:10052B008440F57E9418009F559076840BEA006901
:10053B001E0002692E0004693E000612B612DA5B39
:10054B00DA4B12B5017F607F71900057E00A3B6D6B
:10055B00227E08003C12D0D37CB412B8347F407F8B
:10056B00517F067F1712B5017F607F71900058E0B5
:10057B000A3B6D227CB412B8347F407F517F067FDB
:10058B001712B50112B883907919793E00021BEA54
:10059B0020E412B8347E8440F57E9418009F5512E7
:1005AB00B72290767C1BEA00791E0002792E00049C
:1005BB00793E000690768C0BEA207EF50C7D3F9DF4
:1005CB00327DE368507E74000180467D3F1B345EB4
:1005DB003400037E84407678067E94E00080047EAF
:1005EB0094D0009F5590767C0BEA00691E0002693F
:1005FB002E0004693E000612B5011BEA00791E00AD
:10060B0002792E0004793E0006BE74000538060BF5
:08061B0074BDE750B6DA792244
:100638007C357C4B0A435E340003780674017C5B8E
:1006480080026C557EA001801A7E700DAC750A1A66
:100658002D312E34006D7A71827A6183E00A3B2D48
:0A066800430BA0BCA440E27D342245
:10067200CAD8CA797CDBBED0005803020E6B1AFDC1
:100682007D4F3E447D542E5406277AB1827AA1834F
:100692000BEA507DE52EE4076C90768C1BEAE0BEF7
:1006A20054005A500D90768C0BEA502E5400641B65
:1006B200EA5090768C0BEA709E7407C7BE740000F5
:1006C2004806BE74001D08047E74001D7DEF3EE4E2
:1006D2003EE43EE47D5E2E54069F7AB1827AA18387
:1006E2000BEA00691E0002692E0004693E000690B2
:1006F200765C1BEA00791E0002792E0004793E0026
:10070200067D5F3E543E542E540FFF7AB1827AA189
:1007120083693E00020BEA20E412B8349076541B3F
:10072200EA00791E0002792E0004793E00067D5E01
:100732002E54087F7AB1827AA1830BEA00691E00E7
:1007420002692E0004693E00069076441BEA007995
:100752001E0002792E0004793E00067D5E2E540AA8
:100762005F7AB1827AA1830BEA00691E0002692EC8
:100772000004693E000690764C1BEA00791E0002D6
:10078200792E0004793E00067D5E2E540C3F7AB12C
:10079200827AA1830BEA00691E0002692E000469B5
:1007A2003E00069076241BEA00791E0002792E0094
:1007B20004793E00067D5E2E540E1F7AB1827AA124
:1007C200830BEA00691E0002692E0004693E0006DE
:1007D2009076341BEA00791E0002792E0004793EDD
:1007E20000067D5E2E5410EF7AB1827AA1830BEA65
:1007F20000691E0002692E0004693E000690763CE4
:100802001BEA00791E0002792E0004793E00067D63
:100812005E2E5412CF7AB1827AA1830BEA00691E4E
:100822000002692E0004693E000690762C1BEA0045
:10083200791E0002792E0004793E00067D5E2E5458
:1008420014AF7AB1827AA1830BEA00691E000269B1
:100852002E0004693E00069076641BEA00791E00B1
:1008620002792E0004793E00067D5E2E54168F7AA0
:10087200B1827AA1830BEA00691E0002692E00048C
:10088200693E000690766C1BEA00791E0002792E02
:100892000004793E00067D5F2E541FEF7AB1827A02
:1008A200A1837EEB707408AC7B7D5F3E543E543E68
:1008B200543E543E542D532E54186F7AB1827AA16D
:1008C200830BEA00691E0002692E0004693E0006DD
:1008D2009076741BEA00791E0002792E0004793E9C
:1008E20000067D5F2E5425CB7AB1827AA183E090F7
:1008F2007705F07D5F2E5426077AB1827AA183E0D4
:10090200907706F07D342E3426437A71827A6183A1
:100912000BEA307D235E24000190002C0BEA206854
:10092200064E24000180045E24FFFE1BEA205E3492
:100932000004680D9076E6E09076E7F09076E58028
:100942000B9076E5E09076E7F09076E6E09076E838
:10095200F07E84412E7E9484809F5590766C0BEAC3
:1009620000691E0002692E0004693E000612B612DA
:1009720012B883907709793E00021BEA201A5D3E85
:10098200543E543E542E54202B7AB1827AA1830BCA
:10099200EA00691E0002692E0004693E00067E8498
:1009A200412E7E9484809F5512B61212B8837F0125
:1009B200907709693E00020BEA202F10793E00026F
:1009C2001BEA207E84412E7E9484809F559076740B
:1009D2000BEA00691E0002692E0004693E0006123D
:1009E200B61212B88390770D793E00021BEA201AE4
:1009F2005D3E543E543E542E54220B7AB1827AA16B
:100A0200830BEA00691E0002692E0004693E00069B
:100A12007E84412E7E9484809F5512B61212B88332
:100A22007F0190770D693E00020BEA202F10793E7C
:100A320000021BEA207D573E543E543E542E540081
:100A4200877AB1827AA1830BEA00691E0002692EBD
:100A52000004693E000690761C1BEA00791E000223
:100A6200792E0004793E00067E843F917E94DF4613
:100A72007EA499637EB4E11D9076240BEA00691E80
:100A82000002692E0004693E000612B61212BB7DF6
:100A92009077911BEA00791E0002792E0004793EBC
:100AA20000067E843F917E94DF467EA499637EB4E5
:100AB200E11D9076240BEA00691E0002692E0004F3
:100AC200693E000612B61212BB5C9077991BEA00CF
:100AD200791E0002792E0004793E00067E843F9141
:100AE2007E94DF467EA499637EB4E11D9000320BB2
:100AF200EA00691E0002692E0004693E000612B671
:100B0200129078791BEA00791E0002792E0004798E
:100B12003E000612BB7D9078811BEA00791E00021E
:100B2200792E0004793E00069078790BEA00691E5E
:100B32000002692E0004693E000612BB5C907889AF
:100B42001BEA00791E0002792E0004793E0006900D
:100B520000420BEA80699E000269AE000469BE0091
:100B6200067E04BFF06D119F1112B6127E843F9172
:100B72007E94DF467EA499637EB4E11D12B6121202
:100B8200BB7D9078911BEA00791E0002792E000449
:100B9200793E00067E843F917E94DF467EA499636F
:100BA2007EB4E11D9000420BEA00691E0002692E2C
:100BB2000004693E000612B61212BB5C9078991BC3
:100BC200EA00791E0002792E0004793E0006907830
:100BD200790BEA80699E000269AE000469BE0006D4
:100BE2007E0440006D119F1112B61212BB5C7F4051
:100BF2007F517E043F5B7E14775B7E24DE587E3419
:100C02000DF012B6127E843FEF7E94F2447EA4521F
:100C1200107EB4D3F912B5017F407F517E0440B8F3
:100C22007E14EA287E24F5C27E348F5C12B612CA84
:100C32000BCA1B7E84408F7E9440009F5590004AD1
:100C42000BEA00691E0002692E0004693E000612CA
:100C5200B7227F407F51DA1BDA0B12B5019077F190
:100C62001BEA00791E0002792E0004793E000690EC
:100C720078810BEA80699E000269AE000469BE00B9
:100C8200067E043FEF7E14C9287E2487217E348BA2
:100C9200B012B6129078890BEA80699E000269AEA2
:100CA200000469BE000612B72212BCF49078791BC8
:100CB200EA00791E0002792E0004793E000612BB7A
:100CC2007D7F407F519077F10BEA00691E00026937
:100CD2002E0004693E000612B6129078511BEA00FB
:100CE200791E0002792E0004793E00069078790B75
:100CF200EA00691E0002692E0004693E000612BB6A
:100D02005C7F407F519077F10BEA00691E00026917
:100D12002E0004693E000612B6129078990BEA8002
:100D2200699E000269AE000469BE000612B6129006
:100D320078091BEA00791E0002792E0004793E0030
:100D4200069078790BEA00691E0002692E00046998
:100D52003E000612BB5C7F407F519077F10BEA00A8
:100D6200691E0002692E0004693E000612B6129046
:100D720078910BEA80699E000269AE000469BE00A8
:100D82000612B6129078291BEA00791E0002792E0B
:100D92000004793E00069078790BEA00691E000291
:100DA200692E0004693E000612BB5C7F407F5190B1
:100DB20077F10BEA00691E0002692E0004693E0009
:100DC2000612B82612B6129078910BEA80699E003C
:100DD2000269AE000469BE000612B6127E843F1399
:100DE2007E941DA77EA4F6BA7EB4019812B6129024
:100DF20079091BEA00791E0002792E0004793E006F
:100E0200069078790BEA00691E0002692E000469D7
:100E12003E000612BB5C7F407F519077F10BEA00E7
:100E2200691E0002692E0004693E000612B6129085
:100E320078990BEA80699E000269AE000469BE00DF
:100E42000612B6127E843F137E941DA77EA4F6BAC4
:100E52007EB4019812B6129079111BEA00791E0035
:0E0E620002792E0004793E0006DA79DAD822F1
:10141F00CA69CAF87CFB90765C0BEA80699E000271
:10142F0069AE000469BE000690767C0BEA00691E67
:10143F000002692E0004693E000612B4FD907AB9CD
:10144F001BEA00791E0002792E0004793E000690F7
:10145F007AB90BEA80699E000269AE000469BE008A
:10146F00067E0440006D119F1112B6129076640B28
:10147F00EA80699E000269AE000469BE000612B6DA
:10148F00127F407F5190764C0BEA00691E00026973
:10149F002E0004693E000612B501907A211BEA0066
:1014AF00791E0002792E0004793E00067E043FD596
:1014BF007E1455557E2454F97E34B516CA0BCA1BBB
:1014CF00907A210BEA00691E0002692E0004693E22
:1014DF0000067F407F5112B6127F407F517E04423B
:1014EF00D17E1423197E246F447E34900012B722CC
:1014FF0012D1AE9EF800089077791BEA00791E0092
:10150F0002792E0004793E0006907A210BEA806959
:10151F009E000269AE000469BE00069077790BEA5F
:10152F0000691E0002692E0004693E000612B61201
:10153F007E843F137E94104B7EA457D37EB49B8141
:10154F0012B612907A291BEA00791E0002792E003A
:10155F0004793E00069076340BEA00691E0002699A
:10156F002E0004693E00067F407F5112B6127F4065
:10157F007F517E043FF06D119F1112B4FD907A8957
:10158F001BEA00791E0002792E0004793E00061234
:10159F00BA0E9077891BEA00791E0002792E00049B
:1015AF00793E00067E8440767E9480009F5590762B
:1015BF00440BEA00691E0002692E0004693E000612
:1015CF0012B7229076540BEA80699E000269AE0032
:1015DF000469BE000612B501907AC91BEA00791E94
:1015EF000002792E0004793E00067E04400C6D1136
:1015FF009F11CA0BCA1B9077790BEA80699E000274
:10160F0069AE000469BE00067E0440B87E14EA2865
:10161F007E24F5C27E348F5C12B72212D1AE7F408A
:10162F007F519EF800087E0440237E14E6667E24D8
:10163F0066667E34666612B612CA0BCA1B907A892A
:10164F000BEA00691E0002692E0004693E00067F46
:10165F00407F5112B6127F407F51DA1BDA0B12B75F
:10166F0022907A911BEA00791E0002792E000479EC
:10167F003E0006907A910BEA80699E000269AE00E7
:10168F000469BE0006907AB90BEA00691E00026970
:10169F002E0004693E000612B6129077990BEA806D
:1016AF00699E000269AE000469BE000612B6127F81
:1016BF00407F5190762C0BEA00691E0002692E00C4
:1016CF0004693E000612B4FD9077A11BEA00791E53
:1016DF000002792E0004793E00067E843F917E94AD
:1016EF00DF467EA499637EB4E11D9077A10BEA00DB
:1016FF00691E0002692E0004693E000612B612121E
:10170F00BB7D907A811BEA00791E0002792E0004BE
:10171F00793E00067E843F917E94DF467EA49963D6
:10172F007EB4E11D9077A10BEA00691E0002692EBD
:10173F000004693E000612B61212BB5C907A791B48
:10174F00EA00791E0002792E0004793E0006907798
:10175F00990BEA00691E0002692E0004693E00061B
:10176F007F407F5112B6127F407F517E0440046D3F
:10177F00119F1112B6127E843FE06D999F5512B4DE
:10178F00FDCA0BCA1B907A910BEA80699E00026911
:10179F00AE000469BE0006907AB90BEA00691E001C
:1017AF0002692E0004693E000612B612DA5BDA4BAC
:1017BF0012B6127F407F5190763C0BEA00691E00F3
:1017CF0002692E0004693E000612B5019077A91B2D
:1017DF00EA00791E0002792E0004793E00067E840D
:1017EF003F917E94DF467EA499637EB4E11D90778E
:1017FF00A90BEA00691E0002692E0004693E00066B
:10180F0012B61212BB7D907AA11BEA00791E00025C
:10181F00792E0004793E00067E843F917E94DF4648
:10182F007EA499637EB4E11D9077A90BEA00691E2F
:10183F000002692E0004693E000612B61212BB5C4C
:10184F00907A991BEA00791E0002792E0004793EE6
:10185F000006907A810BEA80699E000269AE00044F
:10186F0069BE0006907AA10BEA00691E0002692E7C
:10187F000004693E000612B6129077990BEA806950
:10188F009E000269AE000469BE000612B612CA0BB2
:10189F00CA1B907A790BEA80699E000269AE000438
:1018AF0069BE0006907A990BEA00691E0002692E44
:1018BF000004693E000612B612DA5BDA4B12B4FD71
:1018CF009077411BEA00791E0002792E0004793EC1
:1018DF000006907A810BEA80699E000269AE0004CF
:1018EF0069BE0006907A990BEA00691E0002692E04
:1018FF000004693E000612B6129077990BEA8069D0
:10190F009E000269AE000469BE000612B612CA0B31
:10191F00CA1B907A790BEA80699E000269AE0004B7
:10192F0069BE0006907AA10BEA00691E0002692EBB
:10193F000004693E000612B6127F407F517E04BF3D
:10194F00F06D119F1112B612DA5BDA4B12B4FD90E3
:10195F0077611BEA00791E0002792E0004793E00A0
:10196F0006907A790BEA80699E000269AE000469DD
:10197F00BE0006907AA10BEA00691E0002692E00D4
:10198F0004693E000612B6129077990BEA80699EA1
:10199F00000269AE000469BE000612B612CA0BCA75
:1019AF001B907A810BEA80699E000269AE00046980
:1019BF00BE0006907A990BEA00691E0002692E009C
:1019CF0004693E000612B612DA5BDA4B12B50190CB
:1019DF0077491BEA00791E0002792E0004793E0038
:1019EF0006907A790BEA80699E000269AE0004695D
:1019FF00BE0006907A990BEA00691E0002692E005C
:101A0F0004693E000612B6129077990BEA80699E20
:101A1F00000269AE000469BE000612B612CA0BCAF4
:101A2F001B907A810BEA80699E000269AE000469FF
:101A3F00BE0006907AA10BEA00691E0002692E0013
:101A4F0004693E000612B6127F407F517E04BFF03C
:101A5F006D119F1112B612DA5BDA4B12B501907746
:101A6F00691BEA00791E0002792E0004793E0006F8
:101A7F009077910BEA80699E000269AE000469BEFF
:101A8F000006907AA10BEA00691E0002692E00047D
:101A9F00693E000612B6129077511BEA00791E00BC
:101AAF0002792E0004793E00069077910BEA806947
:101ABF009E000269AE000469BE0006907A990BEA97
:101ACF0000691E0002692E0004693E000612B6125C
:101ADF009077711BEA00791E0002792E0004793E7F
:101AEF0000067E0440006D119F11CA0BCA1B907A2D
:101AFF00B90BEA00691E0002692E0004693E000658
:101B0F0012D1AE7F407F519EF800089076640BEAA9
:101B1F0000691E0002692E0004693E000612B6120B
:101B2F00CA0BCA1B907AB90BEA80699E000269AE94
:101B3F00000469BE000690764C0BEA00691E000295
:101B4F00692E0004693E000612B6127F407F519045
:101B5F007AC90BEA00691E0002692E0004693E0073
:101B6F000612B501DA5BDA4B12B501907AC11BEAA6
:101B7F0000791E0002792E0004793E00067E843E15
:101B8F00B07E94C6F77EA4A0B57EB4ED8D907AC1D9
:101B9F000BEA00691E0002692E0004693E0006125E
:101BAF00B50112D315907AA91BEA00791E000279AC
:101BBF002E0004793E0006907AA90BEA80699E00F8
:101BCF000269AE000469BE0006907AC10BEA006993
:101BDF001E0002692E0004693E000612B4FD7E84C9
:101BEF003EB07E94C6F77EA4A0B57EB4ED8D12B53F
:101BFF00017E8440706D999F5512B6129077B91B74
:101C0F00EA00791E0002792E0004793E0006907AD0
:101C1F00A90BEA80699E000269AE000469BE000646
:101C2F00907AC10BEA00691E0002692E0004693E1A
:101C3F00000612B4FD7E8440197E9421FB7EA454CD
:101C4F00417EB4174412B6129077C11BEA00791E79
:101C5F000002792E0004793E00069077C10BEA80CE
:101C6F00699E000269AE000469BE00067E04400052
:101C7F006D119F1112B61212BB7DCA0BCA1B907643
:101C8F00340BEA00691E0002692E0004693E00064B
:101C9F007F407F5112B6127F407F517E043FE06D2F
:101CAF00119F1112B612DA5BDA4B12B612CA0BCAB7
:101CBF001B9077C10BEA00691E0002692E000469B0
:101CCF003E000612BB7D7F407F519076340BEA00B9
:101CDF00691E0002692E0004693E000612B6127FCB
:101CEF00407F519077C10BEA00691E0002692E00F8
:101CFF0004693E000612B501DA5BDA4B12B50190AA
:101D0F007781021E8D9077810BEA00691E000269B0
:101D1F002E0004693E000612BB7D9077C91BEA00B6
:101D2F00791E0002792E0004793E00069077810B10
:101D3F00EA00691E0002692E0004693E000612BB0C
:101D4F005C9077D11BEA00791E0002792E0004798E
:101D5F003E00069077D10BEA80699E000269AE00C3
:101D6F000469BE00069076340BEA00691E00026912
:101D7F002E0004693E000612B6127F407F517E048A
:101D8F003FF06D119F1112B4FD9077D91BEA0079C6
:101D9F001E0002792E0004793E00069077C90BEAE7
:101DAF0080699E000269AE000469BE000690763419
:101DBF000BEA00691E0002692E0004693E0006123C
:101DCF00B6127F407F519077810BEA00691E0002A7
:101DDF00692E0004693E000612B4FD9077E11BEAFC
:101DEF0000791E0002792E0004793E00069077C11B
:101DFF000BEA80699E000269AE000469BE0006907E
:101E0F0077E10BEA00691E0002692E0004693E00AB
:101E1F000612B4FD907A711BEA00791E0002792E2A
:101E2F000004793E000612B9D07E843EB07E94C67F
:101E3F00F77EA4A0B57EB4ED8D12B7C14052907756
:101E4F00D90BEA80699E000269AE000469BE0006E4
:101E5F00907A710BEA00691E0002692E0004693E38
:101E6F00000612B7227F407F519077810BEA0069FD
:101E7F001E0002692E0004693E000612B4FD1BEA23
:101E8F0000791E0002792E0004793E0006021D140F
:101E9F009076340BEA80699E000269AE000469BE39
:101EAF0000069077D10BEA00691E0002692E00042C
:101EBF00693E000612B4FD7F407F519077790BEA9F
:101ECF0000691E0002692E0004693E000612B61258
:101EDF009078011BEA00791E0002792E0004793EEA
:101EEF0000069077890BEA80699E000269AE0004B4
:101EFF0069BE00069077790BEA00691E0002692E11
:101F0F000004693E000612B6129077C90BEA806989
:101F1F009E000269AE000469BE000612B6129078E8
:101F2F00211BEA00791E0002792E0004793E00067B
:101F3F009077D90BEA80699E000269AE000469BEF2
:101F4F0000069077790BEA00691E0002692E0004E3
:101F5F00693E000612B6129077E91BEA00791E005F
:101F6F0002792E0004793E0006907A290BEA006967
:101F7F001E0002692E0004693E000612B8269077F3
:101F8F00C90BEA80699E000269AE000469BE0006B3
:101F9F0012B6129077D90BEA80699E000269AE00E3
:101FAF000469BE000612B722907AD11BEA00791E8F
:101FBF000002792E0004793E00069077890BEA80A3
:101FCF00699E000269AE000469BE0006907A290B73
:101FDF00EA00691E0002692E0004693E000612B66F
:101FEF00129077D10BEA80699E000269AE000469F6
:101FFF00BE000612B6129077D90BEA80699E0002D6
:10200F0069AE000469BE000612B722907AD91BEAA6
:10201F0000791E0002792E0004793E000690776148
:10202F000BEA80699E000269AE000469BE0006904B
:10203F0078210BEA00691E0002692E0004693E0038
:10204F000612B612CA0BCA1B9077410BEA80699E23
:10205F00000269AE000469BE00069078010BEA0029
:10206F00691E0002692E0004693E000612B612DADC
:10207F005BDA4B12B501907A491BEA00791E000218
:10208F00792E0004793E00069077690BEA80699EED
:10209F00000269AE000469BE00069078210BEA00C9
:1020AF00691E0002692E0004693E000612B612CAAC
:1020BF000BCA1B9077490BEA80699E000269AE003C
:1020CF000469BE00069078010BEA00691E000269E0
:1020DF002E0004693E000612B612DA5BDA4B12B517
:1020EF0001907A511BEA00791E0002792E000479C3
:1020FF003E00069077710BEA80699E000269AE0080
:10210F000469BE00069078210BEA00691E0002697F
:10211F002E0004693E000612B612CA0BCA1B907736
:10212F00510BEA80699E000269AE000469BE000689
:10213F009078010BEA00691E0002692E0004693EC7
:10214F00000612B612DA5BDA4B12B5019078491B12
:10215F00EA00791E0002792E0004793E000690777E
:10216F00610BEA80699E000269AE000469BE000639
:10217F00907AD90BEA00691E0002692E0004693EAD
:10218F00000612B612CA0BCA1B9077410BEA806980
:10219F009E000269AE000469BE0006907AD10BEA78
:1021AF0000691E0002692E0004693E000612B61275
:1021BF00DA5BDA4B12B501907A591BEA00791E00EF
:1021CF0002792E0004793E00069077690BEA806948
:1021DF009E000269AE000469BE0006907AD90BEA30
:1021EF0000691E0002692E0004693E000612B61235
:1021FF00CA0BCA1B9077490BEA80699E000269AE31
:10220F00000469BE0006907AD10BEA00691E000235
:10221F00692E0004693E000612B612DA5BDA4B1221
:10222F00B501907A611BEA00791E0002792E000435
:10223F00793E00069077710BEA80699E000269AEC5
:10224F00000469BE0006907AD90BEA00691E0002ED
:10225F00692E0004693E000612B612CA0BCA1B9003
:10226F0077510BEA80699E000269AE000469BE00D7
:10227F0006907AD10BEA00691E0002692E000469EC
:10228F003E000612B612DA5BDA4B12B501907A698C
:10229F001BEA00791E0002792E0004793E00067EAB
:1022AF00843FF07E940B367EA4E7EE7EB472569098
:1022BF00767C0BEA00691E0002692E0004693E005D
:1022CF000612B61290761C0BEA80699E000269AE68
:1022DF00000469BE000612B5019078611BEA00790F
:1022EF001E0002792E0004793E000612D3157F409E
:1022FF007F519078610BEA00691E0002692E00047D
:07230F00693E000612B4FD57
:102316007E8440197E9421FB7EA454417EB41744EA
:1023260012B6129078611BEA00791E0002792E001F
:1023360004793E00069078610BEA00691E00026986
:102346002E0004693E000612BB7D7F407F517E044D
:10235600BFF06D119F1112B6129078691BEA0079D1
:102366001E0002792E0004793E00069078610BEA81
:1023760000691E0002692E0004693E000612BB5C5D
:102386009078711BEA00791E0002792E0004793ECE
:1023960000069078690BEA80699E000269AE000427
:1023A60069BE0006907A510BEA00691E0002692E8A
:1023B6000004693E000612B612CA0BCA1B90787159
:1023C6000BEA80699E000269AE000469BE000690B1
:1023D6007A490BEA00691E0002692E0004693E0074
:1023E6000612B612DA5BDA4B12B4FD9077F91BEAE5
:1023F60000791E0002792E0004793E00069078715D
:102406000BEA80699E000269AE000469BE00069070
:102416007A510BEA00691E0002692E0004693E002B
:102426000612B612CA0BCA1B9078690BEA80699E1F
:10243600000269AE000469BE0006907A490BEA0004
:10244600691E0002692E0004693E000612B612DA01
:102456005BDA4B12B5019078191BEA00791E00026F
:10246600792E0004793E00069078490BEA00691E31
:102476000002692E0004693E00069078391BEA00C6
:10248600791E0002792E0004793E00069078690BC9
:10249600EA80699E000269AE000469BE0006907A71
:1024A600610BEA00691E0002692E0004693E0006FF
:1024B60012B612CA0BCA1B9078710BEA80699E008D
:1024C6000269AE000469BE0006907A590BEA0069FB
:1024D6001E0002692E0004693E000612B612DA5B7F
:1024E600DA4B12B4FD907A311BEA00791E000279AC
:1024F6002E0004793E00069078710BEA80699E00F2
:102506000269AE000469BE0006907A610BEA0069B2
:102516001E0002692E0004693E000612B612CA0B9E
:10252600CA1B9078690BEA80699E000269AE0004B6
:1025360069BE0006907A590BEA00691E0002692EF0
:102546000004693E000612B612DA5BDA4B12B501D8
:10255600907A391BEA00791E0002792E0004793E32
:102566000006907A690BEA00691E0002692E0004D3
:10257600693E0006907A411BEA00791E0002792E18
:102586000004793E00069078090BEA80699E0002F5
:1025960069AE000469BE00069077F90BEA00691E71
:1025A6000002692E0004693E000612B4FD907811FF
:1025B6001BEA00791E0002792E0004793E0006907F
:1025C60078290BEA80699E000269AE000469BE00A4
:1025D600069078190BEA00691E0002692E0004694C
:1025E6003E000612B4FD9078311BEA00791E000207
:1025F600792E0004793E00069078510BEA80699E98
:10260600000269AE000469BE00069078390BEA0044
:10261600691E0002692E0004693E000612B4FD9090
:1026260078591BEA00791E0002792E0004793E00D3
:10263600069078310BEA00691E0002692E000469D3
:102646003E00067F407F5112B612CA0BCA1B907815
:10265600110BEA00691E0002692E0004693E00069D
:102666007F407F5112B612DA5BDA4B12B501CA0B04
:10267600CA1B9078590BEA00691E0002692E0004F5
:10268600693E00067F407F5112B6127F407F51DAC5
:102696001BDA0B12B50112BA0E9078A91BEA007963
:1026A6001E0002792E0004793E00069078910BEA0E
:1026B60080699E000269AE000469BE00069078310A
:1026C6000BEA00691E0002692E0004693E0006122C
:1026D600B6129078890BEA80699E000269AE000402
:1026E60069BE000612B612CA0BCA1B9078990BEA8D
:1026F60080699E000269AE000469BE0006907811EA
:102706000BEA00691E0002692E0004693E000612EB
:10271600B6129078890BEA80699E000269AE0004C1
:1027260069BE000612B612DA5BDA4B12B501CA0BA5
:10273600CA1B9078810BEA80699E000269AE00048C
:1027460069BE00069078590BEA00691E0002692EE0
:102756000004693E000612B6127F407F51DA1BDA8A
:102766000B12B5019078B11BEA00791E0002792E92
:102776000004793E00069078990BEA80699E000273
:1027860069AE000469BE00069078110BEA00691E66
:102796000002692E0004693E000612B61290788186
:1027A6000BEA80699E000269AE000469BE0006124B
:1027B600B6127F407F517E04BFF06D119F1112B695
:1027C60012CA0BCA1B9078910BEA80699E000269B7
:1027D600AE000469BE00069078310BEA00691E005F
:1027E60002692E0004693E000612B6129078810B2B
:1027F600EA80699E000269AE000469BE000612B650
:10280600127F407F51DA1BDA0B12B4FDCA0BCA1BCA
:102816009078890BEA80699E000269AE000469BE61
:1028260000069078590BEA00691E0002692E000422
:10283600693E000612B6127F407F51DA1BDA0B1290
:10284600B5019078B91BEA00791E0002792E0004C2
:10285600793E00069078910BEA80699E000269AE87
:10286600000469BE00069078110BEA00691E00029A
:10287600692E0004693E000612B612CA0BCA1B90E6
:1028860078990BEA80699E000269AE000469BE0071
:10289600069078310BEA00691E0002692E00046971
:1028A6003E000612B612DA5BDA4B12B4FD9078C11E
:1028B6001BEA00791E0002792E0004793E0006907C
:1028C60078A90BEA80699E000269AE000469BE0021
:1028D600069078B10BEA00691E0002692E000469B1
:1028E6003E000612B7229078A11BEA00791E00026C
:1028F600792E0004793E00069078A10BEA00691E45
:102906000002692E0004693E00067F407F5112B620
:10291600127F407F517E043FF06D119F1112B4FD6E
:1029260012BA0E9078C91BEA00791E0002792E00B1
:1029360004793E00069078C90BEA80699E00026918
:10294600AE000469BE00069078A10BEA00691E007D
:1029560002692E0004693E000612B72212BCF47EFC
:10296600843F917E94DF467EA499637EB4E11D1276
:10297600B7229078D11BEA00791E0002792E000456
:10298600793E00069078B90BEA80699E000269AE2E
:10299600000469BE00069078C10BEA00691E0002B9
:1029A600692E0004693E000612B72212BCF47E842A
:1029B6003F917E94DF467EA499637EB4E11D12B7F3
:1029C600229078E11BEA00791E0002792E00047934
:1029D6003E00069077E90BEA80699E000269AE0028
:1029E6000469BE00069078390BEA00691E00026988
:1029F6002E0004693E000612B7229078D91BEA0021
:102A0600791E0002792E0004793E00069078D90BD3
:102A1600EA00691E0002692E0004693E00067F4036
:102A26007F5112B6127F407F517E043FF06D119F99
:102A36001112B4FD12BA0E7F407F519078D90BEA7D
:102A460000691E0002692E0004693E000612B722C4
:102A560012BCF47E84404C7E94A5E57EA4F30E7EE3
:102A6600B47FF612B6129078E91BEA00791E0002CE
:102A7600792E0004793E00069077F90BEA80699E6C
:102A8600000269AE000469BE00069078190BEA00E0
:102A9600691E0002692E0004693E000612B7221262
:102AA600BCF47E84404C7E94A5E57EA4F30E7EB4F1
:102AB6007FF612B6129078F11BEA00791E000279B1
:102AC6002E0004793E00069F449F559077F90BEA45
:102AD60000691E0002692E0004693E000612B7C195
:102AE60050199078F10BEA80699E000269AE0004E5
:102AF60069BE00067E044066022BA39F449F559044
:102B060077F90BEA00691E0002692E0004693E008F
:102B16000612B7C1283B9F449F559078190BEA00CF
:102B2600691E0002692E0004693E000612B7C150F4
:102B3600209078F10BEA80699E000269AE00046974
:102B4600BE00067E04BFF06D119F1112B612022C54
:102B5600379F449F559077F90BEA00691E0002697A
:102B66002E0004693E000612B7C1283D9F449F55BA
:102B76009078190BEA00691E0002692E0004693E6E
:102B8600000612B7C128229078F10BEA80699E00F0
:102B96000269AE000469BE00067E0440767E14809B
:102BA600009F1112B4FD022C379077F90BEA0069E9
:102BB6001E0002692E0004693E0006BE0800007869
:102BC60004BE18000078279F449F559078190BEA99
:102BD60000691E0002692E0004693E000612B7C194
:102BE600400C7E0440707E14E0009F118043907775
:102BF600F90BEA00691E0002692E0004693E000610
:102C0600BE0800007804BE18000078379F449F5520
:102C16009078190BEA00691E0002692E0004693ECD
:102C2600000612B7C1501C7E0440567E1480009FD9
:102C3600119078F11BEA00791E0002792E000479C2
:102C46003E00067E8440667E9480009F559078F113
:102C56000BEA00691E0002692E0004693E00061296
:102C6600B7C1501F9078F10BEA80699E000269AEE9
:102C7600000469BE00067E04BFF06D119F1112B6F6
:102C86001280407E8440667E9480009F559078F145
:102C96000BEA00691E0002692E0004693E00061256
:102CA600B7C140319078F10BEA80699E000269AEA7
:102CB600000469BE00067E0440767E1480009F11E3
:102CC60012B4FD9078F11BEA00791E0002792E00FD
:102CD60004793E00069F449F559078B90BEA006937
:102CE6001E0002692E0004693E000612B7C1500696
:102CF6007E844066803A9F449F559078B90BEA00DF
:102D0600691E0002692E0004693E000612B7C1283A
:102D16003D9F449F559078C10BEA00691E000269E9
:102D26002E0004693E000612B7C150227E8440760A
:102D36007E9480009F559078E10BEA00691E0002A0
:102D4600692E0004693E000612B501022DE2907854
:102D5600B90BEA00691E0002692E0004693E0006EE
:102D6600BE0800007804BE180000782A9F449F55CC
:102D76009078C10BEA00691E0002692E0004693EC4
:102D8600000612B7C1400F7E0440567E1480009F95
:102D9600119078E180469078B90BEA00691E00022E
:102DA600692E0004693E0006BE0800007804BE18BD
:102DB600000078379F449F559078C10BEA00691E42
:102DC6000002692E0004693E000612B7C1501C7E3F
:102DD6000440707E14E0009F119078E11BEA0079B0
:102DE6001E0002792E0004793E00069079110BEA46
:102DF60080699E000269AE000469BE0006907A39B9
:102E06000BEA00691E0002692E0004693E000612E4
:102E1600B4FD9078310BEA80699E000269AE000429
:102E260069BE000612B612CA0BCA1B9079090BEAD4
:102E360080699E000269AE000469BE0006907A3180
:102E46000BEA00691E0002692E0004693E000612A4
:102E5600B4FD9078110BEA80699E000269AE000409
:102E660069BE000612B612DA5BDA4B12B501CA0B5E
:102E7600CA1B9078590BEA80699E000269AE00046D
:102E860069BE0006907A410BEA00691E0002692EAF
:102E96000004693E000612B6127F407F51DA1BDA43
:102EA6000B12B5019078A90BEA80699E000269AE03
:102EB600000469BE000612B722907AB11BEA0079B7
:102EC6001E0002792E0004793E000690766C0BEA0D
:102ED60080699E000269AE000469BE00067E04BFDA
:102EE600F06D119F1112B612907AB10BEA80699EAD
:102EF600000269AE000469BE000612B6127E844066
:102F06000A7E94AF647EA406397EB4D5E512B61265
:102F16009079011BEA00791E0002792E0004793EA1
:102F2600000690002E0BEA305E3400107803023063
:102F36003E7E8440C37E9488009F559079010BEABB
:102F460000691E0002692E0004693E000612B722BF
:102F560012B8837F61907AE179DE00021BEAC090A5
:102F660079010BEA00691E0002692E0004693E0021
:102F76000612B8837E5827107F0512D0E47F709022
:102F86007AE579FE00021BEAE07F167F0512D0D3B0
:102F9600907AE9793E00021BEA20BE7809C4580CF3
:102FA600907AE9693E00020BEA20802E907AE56964
:102FB6003E00020BEA20BE181D4C4810907AE969C3
:102FC6003E00020BEA202E182710800E907AE9693F
:102FD6003E00020BEA202E1813887CB412B83490F7
:102FE60079011BEA00791E0002792E0004793E0061
:102FF600069F449F55907AB10BEA00691E0002694C
:103006002E0004693E000612B7C1282C7E84BFF04C
:103016006D999F559079010BEA00691E0002692E91
:103026000004693E000612B6121BEA00791E000271
:10303600792E0004793E00067E84412E7E9484809B
:103046009F5590766C0BEA00691E0002692E0004FB
:10305600693E000612B61212B8837F719079010B91
:10306600EA00691E0002692E0004693E000612B8D5
:10307600837F072F019076F1693E00020BEA202F2D
:1030860010907709793E00021BEA201A6F7D563EA2
:10309600543E543E542E54202B7AB1827AA1830B8F
:1030A600EA00691E0002692E0004693E00067E845D
:1030B600412E7E9484809F5512B61212B8837F01EA
:1030C600907709693E00020BEA202F10793E000234
:1030D6001BEA207D563E543E543E542E5423EB7A32
:1030E600B1827AA1830BEA00691E0002692E0004F0
:1030F600693E000612B8837F01907709693E000297
:103106000BEA202F10793E00021BEA209076740B02
:10311600EA80699E000269AE000469BE00067E046C
:10312600BFF06D119F1112B612907AB10BEA806949
:103136009E000269AE000469BE000612B6127E84C5
:10314600400A7E94AF647EA406397EB4D5E512B6F5
:10315600129078F91BEA00791E0002792E00047994
:103166003E00067E84412E7E9484809F5590767420
:103176000BEA00691E0002692E0004693E00061271
:10318600B61212B8837F719078F90BEA00691E00B7
:1031960002692E0004693E000612B8837F017F177C
:1031A6009F1090770D793E00021BEA201A5F3E546D
:1031B6003E543E542E54220B7AB1827AA1830BEAF6
:1031C60000691E0002692E0004693E00067E8441E5
:1031D6002E7E9484809F5512B61212B8837F01907A
:1031E600770D693E00020BEA202F10793E00021B84
:1031F600EA209076840BEA00691E0002692E00041C
:07320600693E000612D30B24
:10320D00CA0BCA1B90767C0BEA00691E0002692E60
:10321D000004693E000612D30BDA5BDA4B12B7C11C
:10322D00682C7E843FF06D999F559076840BEA0053
:10323D00691E0002692E0004693E000612B5011BCD
:10324D00EA00791E0002792E0004793E0006DAF8B4
:03325D00DA692209
:100E7000CAF87E34000D9006271BEA307E04406FCE
:100E80007E14D7C67E247CB67E34B4DD90069F1BCC
:100E9000EA00791E0002792E0004793E00067E34B5
:100EA000494D7E240001900FFF793E00021BEA208D
:100EB0007E0440657E1447C47E2432CA7E3457A81F
:100EC00090087F1BEA00791E0002792E0004793E0B
:100ED00000067E04402B7E140F627E24E9AF7E3430
:100EE00030B0900A5F1BEA00791E0002792E0004E0
:100EF000793E00067E0440587E14A2EC7E24BFB1E9
:100F00007E345B57900C3F1BEA00791E0002792E5D
:100F10000004793E00067E043FA17E14E4F47E24A2
:100F20000AFF7E343783900E1F1BEA00791E0002F1
:100F3000792E0004793E00067E0440727E14BE7D48
:100F40007E24566C7E34F41F9010EF1BEA00791E4D
:100F50000002792E0004793E00067E0440727E1461
:100F6000DB177E24C1BD7E34A5129012CF1BEA0090
:100F7000791E0002792E0004793E00067E043E7A36
:100F80007E14D7F27E249ABC7E34AF489014AF1BF7
:100F9000EA00791E0002792E0004793E00067E04E4
:100FA000407B7E143E8F7E245C287E34F5C39016F1
:100FB0008F1BEA00791E0002792E0004793E00069C
:100FC0007E0440627E143BD77E240A3D7E3470A4AA
:100FD00090186F1BEA00791E0002792E0004793EFA
:100FE00000067E0440627E143B337E2433337E341D
:100FF00033339018771BEA00791E0002792E000423
:10100000793E00067E0440627E143C7A7E24E147ED
:101010007E34AE1490187F1BEA00791E0002792EF0
:101020000004793E00067E0440627E143D1E7E244C
:10103000B8517E34EB859018871BEA00791E0002B8
:10104000792E0004793E00067404902607F074049B
:101050009025CBF09026430BEA305E34FFFE1BEA6E
:10106000309026430BEA305E34FFFD1BEA309F00D0
:101070009F1190220B1BEA00791E0002792E0004BA
:10108000793E000690202B1BEA00791E0002792E83
:101090000004793E00069026430BEA304E340010DF
:1010A0001BEA307E340006CA397E34E5BF7E240058
:1010B000FF7E1401777E04000112D6981BFDE49098
:1010C00027ABF07EF0010A3F2E3427AB7A71827A8B
:1010D00061837AEBF00BF0BEF03C40EA743C90790F
:0B10E0002AF0743C907929F0DAF82225
:10470700CAF87E14E5BA7E0400FF1206237E14E57C
:10471700907E0400FF1206237E14E5727E0400FFDC
:104727001206237E14E5607E0400FF12062312D4CE
:10473700B37CFBBEF031400BBEF03238067CBF24A1
:0F474700D080097CBF4420B471D97471DAF82294
:10929700CA3B124707907945F0907945E01BB178B2
:1092A70003029336249178030293E8247078E37ECF
:1092B70014E5257E0400FF12062390E102E04480B6
:1092C700F0E4907946F030985512D4B324CE681E56
:1092D70024FD682614680D1BB1680E0BB2782B129B
:1092E7007597800D12758A80081275C080031275F4
:1092F700CD90E102E04420F0802490E102E054F0B8
:10930700F090E102E054DFF0801490E102E054F0C5
:10931700F090E102E054DFF07401907946F0907923
:1093270046E0600302929912909D809A029299906A
:1093370076B2693E00020BEA2012B8E5907B5E1B0D
:10934700EA00791E0002792E0004793E00067E1499
:10935700E5117E0400FF12B95E7E14F3B77E0400A8
:10936700FF7E3479437E24000112659812B9277F66
:10937700319079430BEA304D33680A9076B2797EA3
:1093870000021BEA609076B6693E00020BEA2012E3
:10939700B8E5907B5E1BEA00791E0002792E000477
:1093A700793E00067E14E4FD7E0400FF12B95E7E5E
:1093B70014F3B77E0400FF7E3479437E2400011244
:1093C700659812B9277F319079430BEA304D33689E
:1093D7000A9076B6797E00021BEA601292440292E6
:0493E70099DA3B22B2
:1092440090002C0BEA304E3400041BEA3090E1020B
:10925400E04420F07E14EA587E0400FF1206231234
:10926400728090E102E0540F680D30980512D4B377
:10927400800512909D80E890002C0BEA305E34FF4C
:10928400FB1BEA3090E102E054DFF090E102E0548D
:03929400F0F022D5
:10909D00CA3BE41201C59076960BEA107E35087D29
:1090AD00239D212E250A7A250A0E247A250A907AE7
:1090BD003B1BEA3074011201C590769A0BEA207EB3
:1090CD0035087D139D129000530BEA202D211BEACC
:1090DD00209000530BEA200E241BEA20907A3D1BB2
:1090ED00EA307E250A7CB412CEF7907692691E0086
:1090FD00020BEA0012CE2B7F319000530BEA207C3D
:10910D00B412CEF790768E691E00020BEA0012CED5
:10911D002B907A37793E00021BEA2090002C0BEA47
:10912D00305E34000878386D117E0443347F13129D
:10913D00CEAC28147F1312B8E57E8440667E9480F1
:10914D00009F5512B4FD80127F1312B8E57E844046
:10915D00667E9480009F5512B50112B9277F31901C
:10916D007A3B0BEA30907B641BEA307F1312B8E533
:10917D00907B5C1BEA00791E0002792E0004793E7B
:10918D000006907A3D0BEA30907B5A1BEA30907ABC
:10919D0037693E00020BEA2012B8E5907B521BEABC
:1091AD0000791E0002792E0004793E00067E14E43B
:1091BD00D27E0400FF12B95E7E147A197E0400017E
:1091CD007E34E4C17E2400FF12B98A748012021825
:1091DD007E147A197E0400011204367F1312B8E54D
:1091ED00907A891BEA00791E0002792E0004793EDF
:1091FD000006907A37693E00020BEA2012B8E5901E
:10920D007A811BEA00791E0002792E0004793E0056
:10921D00067E147A197E0400017E34E7847E2400D4
:10922D00FF12B98A74C01202187E147A197E0400D6
:07923D0001120436DA3B22A6
:10701400CA3B7D7390002C0BEA607D365E3400041D
:10702400785C90E102E054F0F0907919693E000236
:107034000BEA20907921793E00021BEA2090791D09
:10704400793E00021BEA209076D6691E00020BEA04
:10705400009076B6693E00020BEA2012CEAC2814EA
:1070640090E000E05401680C90E102E04420F0025A
:10707400727D800090E102E054DFF002727D907630
:10708400D6691E00020BEA009076B669FE00020B78
:10709400EAE07F1712CEAC40030271297F1712B8C1
:1070A400E57E84C0086D999F5512B7C1401890E0E1
:1070B40000E05401680990E102E04420F080079068
:1070C400E102E054DFF07F1712B8E57E84C0086D5A
:1070D400999F5512B7C1500790E102E054DFF07D4B
:1070E400365E34001068319076DA691E00020BEACD
:1070F400009076B6693E00020BEA2012CEAC50181E
:107104007CBF12B3E76D337E24C1709076B6793EAE
:1071140000021BEA2002727D12B3AA90E102E0543D
:10712400F0F002727D7D365E340001684F90002ECF
:107134000BEAF07DEF5EE4010068417E843FB97E96
:107144009499997EA499997EB4999A90766C0BEA55
:1071540000691E0002692E0004693E000612B7C1D0
:10716400281A7D3F5E34000268127CBF12A4E790A7
:10717400002E0BEA305E34FEFF1BEA3090E102E0A1
:107184004420F090002C0BEA305E34002078030297
:10719400727A9076CE69FE00020BEAE09076B669C8
:1071A400DE00020BEAC07F167F0712CEAC280280F5
:1071B400139076CA69FE00020BEAE07F167F07127D
:1071C400CEAC500A9076B679FE00021BEAE09076C7
:1071D400C2697E00020BEA609076C669FE00020B6B
:1071E400EAE07F177F0312CEAC28209076B269DEE6
:1071F40000020BEAC07F167F0712CEAC2802806C17
:107204007F167F0312CEAC506D80307F177F031240
:10721400CEAC50629076B269DE00020BEAC07F16F3
:107224007F0312CEAC50207F1612B8E57E844066F0
:107234007E9480009F5512B7C1280C9076B2797E57
:1072440000021BEA60802F9076C6691E00020BEADA
:10725400007F1612CEAC281E7F1612B8E57E84403D
:10726400667E9480009F5512B7C1500A9076B27919
:0C727400FE00021BEAE0127280DA3B22EE
:10728000CA3BE41201C59076960BEA207E35089D34
:10729000322E350A7A350A0E347A350A7401120113
:1072A000C590769A0BEA307E25089D239000530BFB
:1072B000EA302D321BEA309000530BEA300E341BBB
:1072C000EA307E250A7CB412CEF7907692691E00D1
:1072D000020BEA0012CE2B907A19793E00021BEACB
:1072E000209000530BEA207CB412CEF790768E6982
:1072F0001E00020BEA0012CE2B907A1D793E00028E
:107300001BEA2090002C0BEA305E34000878539082
:1073100076B269FE00020BEAE07F1712B8E57E84C0
:1073200040667E9480009F5512B7C150147F17129B
:10733000B8E57E8440667E9480009F5512B501803A
:107340001A9076B2693E00020BEA2012B8E57E84FC
:1073500040667E9480009F5512B4FD12B9277F319C
:10736000800A9076B2697E00020BEA609076B66978
:10737000FE00020BEAE0907A2179FE00021BEAE0AF
:1073800090769E691E00020BEA007F1312CCD37F19
:10739000319076A2691E00020BEA00907A217F17D5
:1073A00012CCD3793E00021BEA2090002E0BEA306B
:1073B0005E34200068347F1312B8E57E8440667E18
:1073C0009480009F5512B50112B9277F31907A2120
:1073D000691E00020BEA006D337E24433412CCD0C8
:1073E000907A21793E00021BEA207F1312B8E57ED5
:1073F0008440767E9480009F5512B7C128147F1375
:1074000012B8E57E8440767E9480009F5512B4FDCC
:10741000801B9F007F1312CEAC50177F1312B8E56C
:107420007E8440767E9480009F5512B50112B92764
:107430007F31907A2169DE00020BEAC07F1612B814
:10744000E57E8440667E9480009F5512B7C140124D
:107450006D337E244334907A21793E00021BEA206A
:1074600080159F777F167F0712CEAC380A907A215D
:1074700079FE00021BEAE0907A19693E00020BEAED
:10748000207F0312CCD012B8E512B9D07F607F7193
:107490009076A6691E00020BEA006D337E24404000
:1074A00012CD8B12B8E57F407F517F067F1712B750
:1074B000C190E102E028054480F08003547FF09001
:1074C0007A19693E00020BEA207F0312CCD012B871
:1074D000E512B9D07F607F719076A6693E00020BFD
:1074E000EA2012B8E57F407F517F067F1712B7C1AF
:1074F000281B907A19691E00020BEA007F1312CE36
:10750000AC280512758A800812759780031275A43D
:10751000907A21691E00020BEA00907A1D693E00F4
:10752000020BEA2012CCD012B8E512B9D07F607FEE
:10753000719076AA693E00020BEA2012B8E57F40FE
:107540007F517F067F1712B7C12839907A1D691EB7
:1075500000020BEA00907A21693E00020BEA201239
:10756000CEAC28051275C0801E9F449F55907A218D
:10757000693E00020BEA2012B8E512B7C1400812BA
:0A75800075CD80031275DADA3B22A4
:0D758A0090E102E054FC440290E102F02286
:0D75970090E102E054FC440190E102F0227A
:1075A400907919693E00020BEA2090791D793E001A
:0C75B400021BEA2090E102E054FCF022EF
:0D75C00090E102E054F3440890E102F02253
:0D75CD0090E102E054F3440490E102F0224A
:1075DA00907919693E00020BEA20907921793E00E0
:0C75EA00021BEA2090E102E054F3F022C2
:10669C00CAF89076960BEA30907B641BEA309076C1
:1066AC00980BEA30907B621BEA3090769A0BEA30BA
:1066BC00907B601BEA3090769C0BEA30907B5E1BE3
:1066CC00EA307E14E4877E0400FF12B95E7E14E487
:1066DC00577E0400FF12656E7CFBBEF001780C90B7
:1066EC00002E0BEA304E344000800E4CFF780D909B
:1066FC00002E0BEA305E34BFFF1BEA307E14E4142C
:10670C007E0400FF12656E7CFBBEF00168064CFF38
:10671C00685380E8E41201C57E35089076961BEA32
:10672C003074011201C57E350890769A1BEA307ED2
:10673C0014E3D27E0400FF12656E7CFBBEF0016890
:10674C00064CFF682080E8E41201C57E350890767F
:10675C00981BEA3074011201C57E350890769C1B9B
:08676C00EA3012B05FDAF822F6
:10677400CA3B9076960BEA30907B641BEA309076A5
:10678400980BEA30907B621BEA307E14E3AD7E0402
:1067940000FF12B95E7E14E3947E0400FF7E347918
:1067A400437E24000112659812B9277F3190794302
:1067B4000BEA304D33680B7F1312CF319076961B62
:1067C400EA307E14E37C7E0400FF7E3479437E2429
:1067D400000112659812B9277F319079430BEA3092
:1067E4004D33680B7F1312CF319076981BEA307EBD
:1067F40014E34D7E0400FF12656E907945F0B401F8
:106804000C90002E0BEA304E3440008010907945F5
:10681400E0700D90002E0BEA305E34BFFF1BEA30AF
:1068240090769A0BEA30907B641BEA3090769C0B4E
:10683400EA30907B621BEA307E14E3287E0400FF7A
:1068440012B95E7E14E30F7E0400FF7E3479437E2A
:1068540024000112659812B9277F319079430BEA1D
:10686400304D33680B7F1312CF3190769A1BEA3088
:106874007E14E2F77E0400FF7E3479437E24000117
:1068840012659812B9277F319079430BEA304D3362
:10689400680B7F1312CF3190769C1BEA3012B05FE5
:0368A400DA3B22BA
:1075F600CA3B7E14E2CB7E0400FF12062312D4B3EC
:107606004420907947F0B4790280030278429000D2
:107616002C0BEA304E3400101BEA309076BA693EE5
:1076260000020BEA2012B8E5907B5E1BEA00791E89
:107636000002792E0004793E00067E14E2A67E043E
:1076460000FF12B95E7E14F3B77E0400FF7E347924
:10765600437E24000112659812B9277F3190794341
:107666000BEA304D33680A9076BA797E00021BEA3F
:10767600609076BE693E00020BEA2012B8E5907B68
:107686005E1BEA00791E0002792E0004793E000690
:107696007E14E2857E0400FF12B95E7E14F3B77E87
:1076A6000400FF7E3479437E24000112659812B9E6
:1076B600277F319079430BEA304D33680A9076BEC6
:1076C600797E00021BEA607E14E25A7E0400FF12F5
:1076D600062312D4B34420907947F0B4790280038C
:1076E60002783690002E0BEA304E3402001BEA3048
:1076F6009076F5693E00020BEA2012B8E5907B5EB3
:107706001BEA00791E0002792E0004793E00067EEF
:1077160014E23F7E0400FF12B95E7E14F3B77E04C6
:1077260000FF7E3479437E24000112659812B92742
:107736007F319079430BEA304D33680A9076F579BC
:107746007E00021BEA609076F9693E00020BEA2091
:1077560012B8E5907B5E1BEA00791E0002792E00C6
:1077660004793E00067E14E2267E0400FF12B95E0E
:107776007E14F3B77E0400FF7E3479437E24000135
:1077860012659812B9277F319079430BEA304D3351
:10779600680A9076F9797E00021BEA607E14E20A96
:1077A6007E0400FF12B95E7E1479487E0400011241
:1077B60090204D33682F907948E04420249D681826
:1077C60024FD681824F8681824F96808240978152F
:1077D6007401800D740280097403800574048001AD
:1077E600E4907708F07E14E1EE7E0400FF12B95EA5
:1077F6007E1479487E0400011290204D3368519022
:107806007948E04420249D681824FD681824F86807
:107816001824F96808240978377401800D740280E9
:10782600097403800574048001E4907707F08020D2
:1078360090002E0BEA305E34FDFF8011907947E010
:10784600B46E0D90002C0BEA305E34FFEF1BEA306D
:107856007E14E1C67E0400FF12062312D4B3442030
:10786600907947F0B4790280030279D990002C0B05
:10787600EA304E3400201BEA309076C2693E0002A0
:107886000BEA2012B8E5907B5E1BEA00791E000227
:10789600792E0004793E00067E14E1A17E0400FFE5
:1078A60012B95E7E14F3B77E0400FF7E3479437E00
:1078B60024000112659812B9277F319079430BEAAB
:1078C600304D33680A9076C2797E00021BEA6090DA
:1078D60076C6693E00020BEA2012B8E5907B5E1B75
:1078E600EA00791E0002792E0004793E00067E1415
:1078F600E1807E0400FF12B95E7E14F3B77E0400B9
:10790600FF7E3479437E24000112659812B9277FE1
:10791600319079430BEA304D33680A9076C6797E0A
:1079260000021BEA609076CA693E00020BEA20124A
:10793600B8E5907B5E1BEA00791E0002792E0004F2
:10794600793E00067E14E15F7E0400FF12B95E7E7A
:1079560014F3B77E0400FF7E3479437E24000112BF
:10796600659812B9277F319079430BEA304D336819
:107976000A9076CA797E00021BEA609076CE693E4E
:1079860000020BEA2012B8E5907B5E1BEA00791E26
:107996000002792E0004793E00067E14E13E7E0444
:1079A60000FF12B95E7E14F3B77E0400FF7E3479C1
:1079B600437E24000112659812B9277F31907943DE
:1079C6000BEA304D3368209076CE797E00021BEAB2
:1079D600608014907947E0B46E0D90002C0BEA306D
:1079E6005E34FFDF1BEA307E14E1147E0400FF12D2
:1079F600062312D4B34420907947F0B47902800369
:107A0600027AA190002E0BEA305E34F7FF1BEA30B3
:107A16009079250BEA30907B641BEA307E14E0E512
:107A26007E0400FF12B95E7E14F3B77E0400FF7E6B
:107A36003479437E2400011265CB9079451BEA30E8
:107A46009079430BEA304D33680C9079450BEA3058
:107A56009079251BEA309079270BEA30907B641BDE
:107A6600EA307E14E0AC7E0400FF12B95E7E14F3A9
:107A7600B77E0400FF7E3479437E2400011265CB75
:107A86009079451BEA309079430BEA304D33681FF5
:107A96009079450BEA309079278011907947E0B4C8
:107AA6006E0D90002E0BEA304E3408001BEA30DAD9
:027AB6003B2271
:107AB800CA3B9076A6693E00020BEA2012B8E59010
:107AC8007B5E1BEA00791E0002792E0004793E00D5
:107AD800067E14E08A7E0400FF12B95E7E14F3B7B6
:107AE8007E0400FF7E3479437E24000112659812DB
:107AF800B9277F319079430BEA304D33680A907685
:107B0800A6797E00021BEA609076AA693E00020B05
:107B1800EA2012B8E5907B5E1BEA00791E00027924
:107B28002E0004793E00067E14E06C7E0400FF12ED
:107B3800B95E7E14F3B77E0400FF7E3479437E2459
:107B4800000112659812B9277F319079430BEA300A
:107B58004D33680A9076AA797E00021BEA60907617
:107B68009E693E00020BEA2012B8E5907B5E1BEA94
:107B780000791E0002792E0004793E00067E14E08A
:107B88004C7E0400FF12B95E7E14F3B77E0400FF3A
:107B98007E3479437E24000112659812B9277F311B
:107BA8009079430BEA304D33680A90769E797E00CF
:107BB800021BEA609076A2693E00020BEA2012B826
:107BC800E5907B5E1BEA00791E0002792E0004799D
:107BD8003E00067E14E02E7E0400FF12B95E7E147D
:107BE800F3B77E0400FF7E3479437E2400011265DA
:107BF8009812B9277F319079430BEA304D33680AE0
:0D7C08009076A2797E00021BEA60DA3B2232
:107C1500CA3B7E34FBC37E2400FF7E1479437E0479
:107C25000001740C12D1187E34FBCF7E2400FF7E38
:107C350014794F7E040001740812D1187E34FBD7E5
:107C45007E2400FF7E1479577E040001741412D13E
:107C5500187E34FBEB7E2400FF7E14796B7E0400D6
:107C650001740812D1187E34FBF37E2400FF7E14C4
:107C750079737E040001741812D11890002C0BEA58
:107C8500707E14E5BA7E0400FF1206237E3427E8D1
:107C95007E240001907B62793E00021BEA20900061
:107CA500320BEA00691E0002692E0004693E0006D7
:107CB500907B5A1BEA00791E0002792E0004793E5A
:107CC500000690003A0BEA00691E0002692E0004C6
:107CD500693E0006907B521BEA00791E0002792E50
:107CE5000004793E000690004A0BEA00691E000276
:107CF500692E0004693E0006907B4A1BEA00791E46
:107D05000002792E0004793E00067E14DFC97E0448
:107D150000FF12B95E9076960BEA30907B641BEA01
:107D2500309076980BEA30907B621BEA3090769A19
:107D35000BEA30907B601BEA3090769C0BEA309022
:107D45007B5E1BEA307E14DF987E0400FF12B95E6D
:107D550090002E0BEA607D365E344000680B7E1481
:107D6500DF917E0400FF12B95E7E14EA587E04009E
:107D7500FF12B95E9076A6693E00020BEA2012B8A2
:107D8500E5907B5E1BEA00791E0002792E000479DE
:107D95003E00069076AA693E00020BEA2012B8E57D
:107DA500907B561BEA00791E0002792E0004793E6D
:107DB50000067E14DF5E7E0400FF12B95E90769E9B
:107DC500693E00020BEA2012B8E5907B5E1BEA00D3
:107DD500791E0002792E0004793E00069076A2698C
:107DE5003E00020BEA2012B8E5907B561BEA0079AB
:107DF5001E0002792E0004793E00067E14DF2B7EDC
:107E05000400FF12B95E90002C0BEA305E340010BE
:107E15007803027F0D9076BA693E00020BEA2012C4
:107E2500B8E5907B5E1BEA00791E0002792E0004FE
:107E3500793E00069076BE693E00020BEA2012B834
:107E4500E5907B561BEA00791E0002792E00047925
:107E55003E00067E14DEF87E0400FF12B95E7D3614
:107E65005E3402007803027F009076F5693E0002D9
:107E75000BEA2012B8E5907B5E1BEA00791E000232
:107E8500792E0004793E00069076F9693E00020BD2
:107E9500EA2012B8E5907B561BEA00791E000279AC
:107EA5002E0004793E00069077087EEB307404AC12
:107EB5003B2E1479577A31827A2183693E00020B71
:107EC500EA20907B52793E00021BEA209077077EDC
:107ED500EB307404AC3B2E1479577A31827A2183C6
:107EE500693E00020BEA20907B4E793E00021BEAB8
:107EF500207E14DEBC7E0400FF80157E14DEA37E8A
:107F05000400FF120623800B7E14DE8A7E0400FF28
:107F150012B95E90002C0BEA305E34002078030223
:107F25007FAD9076C2693E00020BEA2012B8E5905B
:107F35007B5E1BEA00791E0002792E0004793E0063
:107F4500069076C6693E00020BEA2012B8E5907BE2
:107F5500561BEA00791E0002792E0004793E0006C0
:107F65009076CA693E00020BEA2012B8E5907B4E76
:107F75001BEA00791E0002792E0004793E00069066
:107F850076CE693E00020BEA2012B8E5907B461BCF
:107F9500EA00791E0002792E0004793E00067E145F
:107FA500DE4F7E0400FF80087E14DE367E0400FF6F
:107FB50012B95E9076D6693E00020BEA2012B8E54A
:107FC500907B5E1BEA00791E0002792E0004793E43
:107FD50000069076DA693E00020BEA2012B8E590B9
:107FE5007B561BEA00791E0002792E0004793E00BB
:107FF500069076DE693E00020BEA2012B8E5907B1A
:108005004E1BEA00791E0002792E0004793E000617
:108015007E14DDF47E0400FF12B95E90002E0BEA9B
:10802500305E340800680D7E14DDD67E0400FF1234
:10803500062380349079250BEA30907B641BEA3067
:108045007E14DDAA7E0400FF12B95E9079270BEA43
:1080550030BE34003D5011907B641BEA307E14DD48
:10806500787E0400FF12B95E9076E27EEBD07E301A
:1080750004AC3D2E1479437A31827A2183693E001E
:10808500020BEA20907B62793E00021BEA207D17F5
:108095005E1400801E141E141E141E141E141E14BD
:1080A5001E143E143E142E14796B7A31827A218384
:1080B500693E00020BEA20907B5E793E00021BEAD6
:1080C500207E14DD5F7E0400FF12B95E1BD068249C
:1080D5001BD068640BD1680302818290002E0BEAE5
:1080E500305E34002078030281827E14DD537E04E5
:1080F50000FF803F9000300BEA607D365E34000261
:10810500680A7E14DD4A7E0400FF80107D365E34E9
:108115000004680B7E14DD417E0400FF12062390E7
:10812500002C0BEA305E34004068527E14DD347E4C
:108135000400FF12062380459076E5E00A3B907B1C
:10814500641BEA307E14DD2C7E0400FF12B95E90BC
:1081550076E6E00A3B907B641BEA307E14DD267EE2
:108165000400FF12B95E900052E00A3B907B641B4D
:10817500EA307E14DD1E7E0400FF12B95E90006CAD
:108185007EEB307404AC3B2E1479777A31827A21F8
:1081950083693E00020BEA20907B62793E00021B58
:1081A500EA207E14DD1A7E0400FF12B95E7D175E9B
:1081B5001400081E141E141E143E143E142E1479A9
:1081C5004F7A31827A2183693E00020BEA20907B47
:1081D50062793E00021BEA207E14DD027E0400FF68
:1081E50012B95E90006B7EEB307404AC3B2E1479B3
:1081F500737A31827A2183693E00020BEA20907BF3
:1082050062793E00021BEA207E14DCDD7E0400FF5D
:1082150012B95E7E14DCBF7E0400FF12B95E12D473
:04822500B3DA3B226B
:104ED100CA3B7D63E4907971F06CEE7E043FF06D26
:104EE100119F119079741BEA00791E0002792E003E
:104EF10004793E00069F009F1190797C1BEA00799E
:104F01001E0002792E0004793E00067CBD12067255
:104F110012044B7E350C907B641BEA30E50E907BCE
:104F210063F0900055E0907B62F0900056E0907B3A
:104F310061F0900057E0907B60F0900058E0907B2A
:104F41005FF07E14DC997E0400FF12B95E7E14DCF2
:104F5100707E0400FF120623E490794EF0E490790C
:104F61004BF07E1479497E04000112902090794E15
:104F71007EEBA090794BE04CBAB42F028003025033
:104F8100509079577EEBA0907954E04CBAB43A0234
:104F910080030250509079497EEBA00A0A9E0400DA
:104FA100307E14000AAD1090794AE00A3B9E34002D
:104FB100302D312E34076C90793B1BEA30BEA0397D
:104FC100680D90793B0BEA302E3400641BEA309077
:104FD100794C7EEB709E70307E600AAC7690794D94
:104FE100E024D02CB7907943F090794F7EEB709EFE
:104FF10070307E600AAC76907950E024D02CB79066
:105001007944F09079527EEB709E70307E600AACEC
:1050110076907953E024D02CB7907945F09079556A
:105021007EEB709E70307E600AAC76907956E024FB
:10503100D02CB7907946F09079587EEB709E703005
:105041007E600AAC76907959E024D02CB7802B7E13
:10505100350C90793B1BEA30E50E907943F09000D6
:1050610055E0907944F0900056E0907945F0900039
:1050710057E0907946F0900058E0907947F09079A8
:105081003B0BEA30907943E09079447EEB50907984
:10509100457EEB409079467EEB309079477EEB2060
:1050A1001256147E8440787E94C0009F5590767C81
:1050B1000BEA00691E0002692E0004693E00061217
:1050C100B7C1280B7E14F9DF7E0400FF120623907E
:1050D100767C0BEA00691E0002692E0004693E001D
:1050E10006907B5E1BEA00791E0002792E0004798E
:1050F1003E00067E14DC527E0400FF12B95E7E146F
:10510100DC467E0400FF1206237E14DC3B7E040095
:10511100FF7E3479727E2400011265989079941B88
:10512100EA00791E0002792E0004793E000690798A
:10513100720BEA304D3368249079940BEA00691EB2
:105141000002692E0004693E00069079741BEA0092
:10515100791E0002792E0004793E00067E14DC30AF
:105161007E0400FF7E3479727E24000112659890DE
:10517100799C1BEA00791E0002792E0004793E0019
:10518100069079720BEA304D33682490799C0BEAD2
:1051910000691E0002692E0004693E000690797CB8
:1051A1001BEA00791E0002792E0004793E00067E7A
:1051B100843F467E94C16C7EA416BB7EB42ACF90F8
:1051C10079740BEA00691E0002692E0004693E0031
:1051D1000612B6121BEA00791E0002792E0004792C
:1051E1003E00067E843EE87E9445C87EA4A0A97E4A
:1051F100B49EFC90797C0BEA00691E0002692E00C6
:1052010004693E000612B6121BEA00791E000279FB
:105211002E0004793E000690797C0BEA80699E009D
:105221000269AE000469BE00069079740BEA006958
:105231001E0002692E0004693E000612B501907934
:10524100841BEA00791E0002792E0004793E0006D3
:105251007E34DC007E2400FF907B62793E00021BDD
:10526100EA207E34DBFB7E2400FF907B5E793E00EA
:10527100021BEA207E34DBF87E2400FF907B5A7902
:105281003E00021BEA207E34DBF57E2400FF907B8A
:1052910056793E00021BEA207E34DBEF7E2400FFBC
:1052A100907B52793E00021BEA207E34DBE77E24AC
:1052B10000FF907B4E793E00021BEA207E14DC0544
:1052C1007E0400FF12B95EE4907948F030980A122A
:1052D100D4B37CFB6CEE0255DA7CBD12141F9076C0
:1052E1007C0BEA00691E0002692E0004693E00067B
:1052F10012B8839079391BEA307D237CB412B83916
:105301007F407F5190767C0BEA00691E0002692E76
:105311000004693E000612B4FD90798C1BEA007905
:105321001E0002792E0004793E00067E34793D7E0E
:105331002400019079AC793E00021BEA207E347989
:105341003E7E2400019079B0793E00021BEA209054
:1053510079390BEA307E1479377E04000112579DAA
:105361007E3479417E2400019079B0793E00021BA0
:10537100EA2090798C0BEA00691E0002692E000474
:10538100693E00069079B41BEA00791E0002792E6D
:105391000004793E00067E14793F7E0400017E34CC
:1053A10079407E24000112583E7E84BFF06D999FA2
:1053B100559078D10BEA00691E0002692E0004693C
:1053C1003E000612B7C138030254FB9079370BEA4D
:1053D10030907B641BEA3090793DE0907B63F090E4
:1053E100793EE0907B62F07E14DBD67E0400FF12F2
:1053F100B95E90793FE0907B65F0907940E0907BD9
:1054010064F0907941E0907B63F07E14DBBF7E0411
:1054110000FF12B95E9078E10BEA00691E00026993
:105421002E0004693E0006907B5E1BEA00791E0097
:1054310002792E0004793E00069078D10BEA0069CA
:105441001E0002692E0004693E0006907B561BEA8D
:1054510000791E0002792E0004793E00069077B98A
:105461000BEA00691E0002692E0004693E000690E5
:105471007B4E1BEA00791E0002792E0004793E0062
:10548100069079010BEA00691E0002692E00046989
:105491003E0006907B461BEA00791E0002792E0031
:1054A10004793E00067E14DBA67E0400FF12B95E7D
:1054B1009079A40BEA80699E000269AE000469BE7E
:1054C10000069078D10BEA00691E0002692E0004E3
:1054D100693E000612B7C128067401907971F090F7
:1054E1007948E004F09079840BEA80699E000269B2
:1054F100AE000469BE00060255869079A40BEA80CD
:10550100699E000269AE000469BE00069078D10B65
:10551100EA00691E0002692E0004693E000612B706
:10552100C15017907971E0B401107E14DB997E04AB
:1055310000FF120623E4907971F07E843F467E9449
:10554100C1627EA48B657EB479579079840BEA00A1
:10555100691E0002692E0004693E000612B7C128C7
:10556100149079840BEA80699E000269AE00046997
:10557100BE000680107E843F467E94C1627EA48B6D
:10558100657EB4795790767C0BEA00691E0002694A
:105591002E0004693E000612B5011BEA00791E00C7
:1055A10002792E0004793E00069078D10BEA006959
:1055B1001E0002692E0004693E00069079A41BEAD0
:1055C10000791E0002792E0004793E000690794888
:1055D100E0BEB01650030252CD4CEE6803025251A8
:1055E1007E14DB737E0400FF12062312D4B37CFB0E
:1055F1004420BEB0716819B4730280030252517E17
:10560100E0017E14EA587E0400FF12062302525183
:03561100DA3B225F
:10561400CAD8CA797CF27CE37CD47DE31206387D57
:1056240023E412B8399076841BEA00791E000279CB
:105634002E0004793E00067C4DE412B83E7E844080
:10564400386D999F5512B7229079AE1BEA00791EE6
:105654000002792E0004793E00067C4EE412B83E26
:105664007E8440967E9480009F5512B7229079B62E
:105674001BEA00791E0002792E0004793E00067CA4
:105684004FE412B83E7E8440F57E9418009F551274
:10569400B7229079BE1BEA00791E0002792E00041D
:1056A400793E000690768C0BEA207D3E9D329079FF
:1056B400AC1BEA3068567EF4000180467D3E9D3F77
:1056C4005E3400037E84407678067E94E000800495
:1056D4007E94D0009F559076840BEA00691E0002E8
:1056E400692E0004693E000612B5011BEA00791E0A
:1056F4000002792E0004793E0006BEF40005380C41
:105704000BF49079AC0BEA30BDF328B09076840B9F
:10571400EA00691E0002692E0004693E00069076C4
:105724007C1BEA00791E0002792E0004793E0006F3
:105734009079B60BEA80699E000269AE000469BEE6
:1057440000069079AE0BEA00691E0002692E00047F
:10575400693E000612B5019079BE0BEA80699E008D
:105764000269AE000469BE000612B5017F407F5194
:1057740090767C0BEA00691E0002692E0004693EE3
:10578400000612B5011BEA00791E0002792E0004FE
:09579400793E0006DA79DAD82228
:10579D00CA797DF37E700190768C0BEA207DE25EF6
:1057AD00E40003780674017C7B80026C777D4F7E6C
:1057BD00A0018022BEA00C183A1AC77ED4000DADF0
:1057CD00DC1A7A2D7D2E74006D7AF1827AE183E0F8
:1057DD000AEB9D4E0BA01AC77ED4000DADDC1A7AD4
:1057ED002D7D2E74006D7AF1827AE183E00AEBBD96
:1057FD004E38C1BEA00C0817BEA00C08B24C77687D
:10580D00069EF4016E80049EF4016D0B24808E9033
:10581D0079AC69FE00020BEAE07A7BA07C69907995
:10582D00B069FE00020BEAE07A7B601B0A20DA7990
:01583D002248
:10583E00CA3B7F319079AC1BEA00791E00027E8450
:10584E0040386D999F559079B40BEA00691E00029D
:10585E00692E0004693E000612B6129079BC1BEA4E
:10586E0000791E0002792E0004793E000612B883DC
:10587E009079C41BEA307D237CB412B8397F407F07
:10588E00519079BC0BEA00691E0002692E00046972
:10589E003E000612B4FD1BEA00791E0002792E00AE
:1058AE0004793E00067E84404E6D999F559079BCDA
:1058BE000BEA00691E0002692E0004693E00061202
:1058CE00B61212B8839079C61BEA307D237CB412CF
:1058DE00B8397E84404E6D999F5512B7227F407F16
:1058EE00519079BC0BEA00691E0002692E00046912
:1058FE003E000612B4FD1BEA00791E0002792E004E
:10590E0004793E00067E8440AC7E9420009F559024
:10591E0079BC0BEA00691E0002692E0004693E0084
:10592E000612B61212B8839079C81BEA309079C469
:10593E000BEA109079AC693E00020BEA207A1B301C
:10594E009079C60BEA307A3B709079C80BEA1090CA
:0F595E0079B0693E00020BEA207A1B30DA3B2257
:10940000CA3B6D661214007E14DB477E0400FF1217
:1094100006239000590BEA30907945802412D4B38A
:109420007CEB9079450BEA307D232E2427FC7A5182
:10943000827A41837AEBE0BEE01A68149079450B9A
:10944000341BEA309079450BEA30BE344E1F40CDD4
:109450009079450BEA309000591BEA30BE344E1E1D
:10946000400B7E14DB307E0400FF1206231210EB4B
:109470007E14EA587E0400FF1206236D339079456E
:109480001BEA306CFF9079450BEA307D230B241BDF
:10949000EA202E3427FC7A71827A61837EEBE0BE6B
:1094A000E01A6822BEE00D681DBEE00A68187CAFB5
:1094B0000BF00A3A2E3479977A71827A61837AEBCB
:1094C000E0BEF04F40BFBEE01A7803029A14E40AEF
:1094D0003F2E3479977A71827A6183F0907997E0A0
:1094E000BEB020689E609C7E3400147D16AD132EA5
:1094F0001401777E040001E412D6C17E34000FCA45
:10950000397E140014AD162E1401777E0400017EFE
:109510003479977E24000112D6981BFD6CFF907958
:10952000450BEA307D230B241BEA202E3427FC7ADE
:1095300071827A61837EEBE0BEE01A6822BEE00DA4
:10954000681DBEE00A68187CAF0BF00A3A2E347929
:10955000477A71827A61837AEBE0BEF04F40BF9028
:109560007947E0B431028003029483907949E0BEE8
:10957000B0417803029483907959E00A2B9E24002D
:10958000307E34000AAD3290795AE00A2B9E2400D6
:10959000302D237D363E342E3406277A71827A614F
:1095A000831BEA206CFF0A3F7D232E24795B7A51CE
:1095B000827A4183E02E3479977A71827A6183F0DE
:1095C0000BF0BEF00C78DFE49079A3F07E1479976D
:1095D0007E04000112B9DF7F607F717D363E343E2C
:1095E000343E342E34069F7A71827A61831BEAC03E
:1095F00079DE000279EE000479FE00066CFF0A3F76
:109600007D232E2479687A51827A4183E02E347941
:10961000977A71827A6183F00BF0BEF00A78DFE40A
:109620009079A1F07E1479977E04000112B9DF7F52
:10963000607F717D363E343E343E342E3414AF7A32
:1096400071827A61831BEAC079DE000279EE000440
:1096500079FE00066CFF9079450BEA307D230B24E0
:109660001BEA202E3427FC7A71827A61837EEBE03C
:10967000BEE01A6822BEE00D681DBEE00A68187CD4
:10968000AF0BF00A3A2E3479477A71827A61837A85
:10969000EBE0BEF04F40BF907947E0B43202800368
:1096A0000294836CFF0A3F7D232E24794F7A5182E6
:1096B0007A4183E02E3479977A71827A6183F00B54
:1096C000F0BEF00878DFE490799FF07E1479977E01
:1096D00004000112B9DF7F607F717D363E343E3475
:1096E0003E342E340C3F7A71827A61831BEAC07952
:1096F000DE000279EE000479FE00066CFF0A3F7D71
:10970000232E2479587A51827A4183E02E34799736
:109710007A71827A6183F00BF0BEF00878DFE49012
:10972000799FF07E1479977E04000112B9DF7F6083
:109730007F717D363E343E343E342E3412CF7A7102
:10974000827A61831BEAC079DE000279EE00047937
:10975000FE00067EF0020A3F7D232E24795F7A51B7
:10976000827A4183E02E3479977A71827A6183F02C
:109770000BF0BEF00978DFE49079A0F074309079B6
:1097800097F0742E907998F07E1479977E040001FA
:1097900012B9DF7F607F717D363E343E343E342E19
:1097A000340E1F7A71827A61831BEAC079DE00026F
:1097B00079EE000479FE00066CFF0A3F7D232E241B
:1097C00079697A51827A4183E02E3479977A71826D
:1097D0007A6183F00BF0BEF00878DFE490799FF0B7
:1097E0007E1479977E04000112B9DF7F607F717D5E
:1097F000363E343E343E342E3410EF7A71827A6134
:10980000831BEAC079DE000279EE000479FE0006CF
:109810006CFF0A3F7D232E2479727A51827A41832C
:10982000E02E3479977A71827A6183F00BF0BEF082
:109830000878DFE490799FF07E1479977E04000128
:1098400012B9DF7F607F717D363E343E343E342E68
:1098500034087F7A71827A61831BEAC079DE000264
:1098600079EE000479FE00066CFF0A3F7D232E246A
:10987000797B7A51827A4183E02E3479977A7182AA
:109880007A6183F00BF0BEF00B78DFE49079A2F000
:109890007E1479977E04000112B9DF7F607F717DAD
:1098A000363E343E343E342E340A5F7A71827A6119
:1098B000831BEAC079DE000279EE000479FE00061F
:1098C0006CFF0A3F7D232E2479867A51827A418368
:1098D000E02E3479977A71827A6183F00BF0BEF0D2
:1098E0000578DFE490799CF07E1479977E0400017E
:1098F00012D5677F017D363E343E342E340FFF7A19
:1099000071827A6183791E00021BEA009F669F774D
:109910007D363E343E343E342E34168F7A71827A50
:1099200061831BEAC079DE000279EE000479FE0053
:10993000067D363E343E343E343E343E342E3418BA
:10994000877A71827A61831BEAC079DE000279EE40
:10995000000479FE00069F669F777D363E343E34D4
:109960003E343E343E342E34187F7A71827A6183DD
:109970001BEAC079DE000279EE000479FE00069F42
:10998000669F777D363E343E343E343E343E342E40
:109990003418777A71827A61831BEAC079DE00021B
:1099A00079EE000479FE00069F669F777D363E348F
:1099B0003E343E343E343E342E34186F7A71827A0F
:1099C00061831BEAC079DE000279EE000479FE00B3
:1099D000067D360B34907B641BEA307E340014AD78
:1099E000362E3401777E240001907B60793E0002A0
:1099F0001BEA207E14DB217E0400FF12B95E0B649B
:109A00007CBD907929F0BE64003C5008BEE01A6825
:0A9A100003029483129A1ADA3B2233
:10A17E00CA3B7E14EA587E0400FF1206236CEE6C76
:10A18E00FF74FF0A3F2E3427AB7A71827A6183F017
:10A19E000BF0BEF03C78EC6CFF124C847D63BE6419
:10A1AE0000005807BEE0002845804A7CBD0A3F2EBD
:10A1BE003427AB7A71827A6183F07E340014AD3627
:10A1CE002E3401777E240001907B62793E00021BC3
:10A1DE00EA200A3E0B34907B601BEA307E14DAFCD8
:10A1EE007E0400FF12B95E0BE0BEE03C50070BF0A0
:10A1FE00BEF03C40A490792A7AEBE012A20FDA3B33
:01A20E00222D
:104C8400CA3B6D339079451BEA307E14EA587E04A2
:104C940000FF1206236D77907929E00A3BBD734823
:104CA40003024D4A4D7768187E2400047D3712D0E4
:104CB400A14D22780B7E14EA587E0400FF120623CD
:104CC4007D373E342E3426437A71827A61830BEA2F
:104CD400305E340010682C7D370B34907B641BEA03
:104CE400307E340014AD372E3401777E24000190D9
:104CF4007B60793E00021BEA207E14DAF07E040019
:104D0400FF802A7D370B34907B641BEA307E3400AD
:104D140014AD372E3401777E240001907B60793EF8
:104D240000021BEA207E14DAE47E0400FF12B95E5E
:104D34009079450BEA300B341BEA300B74BE7400D7
:104D44003C5803024C9B7E14DAD97E0400FF7E3467
:104D540079477E2400011265CB7D639079450BEA87
:104D640030BD6308028030BE640000082ABE6400BF
:104D74003C18247D263E242E2426417A51827A41F1
:104D8400830BEA304E3400107A51827A41831BEA55
:0E4D9400307D361B3480047E34FFFFDA3B2274
:104DA200CA3B7E14DAD57E0400FF1206236D777D9E
:104DB200372E3427AB7A71827A6183E0BEB0005815
:104DC20003024E4B90792AE00A3BBD730803024E60
:104DD200564D7768187E2400047D3712D0A14D22EB
:104DE200780B7E14EA587E0400FF12062390792B7A
:104DF200E01A3BBD737804742A800274209079967D
:104E0200F07D370B34907B641BEA30907996E00A90
:104E12003B907B621BEA307D372E3427AB7A71825E
:104E22007A6183E01A2B7E340014AD322E3401777E
:104E32007E240001907B5E793E00021BEA207E14F4
:104E4200DAC87E0400FF12B95E0B74BE74003C58CF
:104E520003024DB17E14EA587E0400FF1206237E3F
:104E6200340007CA399027ABE01A0B7E140014AD48
:104E7200102E1401777E0400017E34DAC07E2400F5
:104E8200FF12D6341BFD70117E14DA917E0400FFEE
:104E92001206237E34FFFF80337E14DAD97E0400AB
:104EA200FF7E3479947E2400011265CB7D631B64FE
:104EB20090792AE00A3BBD6358DFBE6400005804C3
:0F4EC2007E64FFFF7CBD90792BF07D36DA3B22BA
:10A20F00CA796CEE6CFF0A3F2E3427AB7A71827AD3
:10A21F0061837EEBA0BEA00048137C7E0BE00A3763
:10A22F002E3427AB7A71827A61837AEBA00BF0BE62
:10A23F00F03C78D274FF7CFE802E0A3F2E3427AB81
:10A24F007A71827A6183F07E340002CA397E14FFFC
:10A25F00EC2E1401777E0400017E34DA8E7E24000A
:10A26F00FF12D6981BFD0BF0BEF03C40CDDA7922E1
:109A1A00CA3B6CDD1214006D339079E71BEA30748F
:109A2A00FF9079E70BEA307D232E2427AB7A518207
:109A3A007A4183F09079E70B341BEA309079E70B8F
:109A4A00EA30BE34003C78D77E14DA5F7E0400FF29
:109A5A001206239000590BEA309079E71BEA30800E
:109A6A002412D4B39079EDF09079E70BEA307D2394
:109A7A000B241BEA202E3427FC7A71827A6183F048
:109A8A00BEB01A680C9079E70BEA30BE344E1F401C
:109A9A00D09079E70BEA30BE344E1F400B7E14DBC0
:109AAA00307E0400FF1206237E14EA587E0400FF6B
:109ABA001206239000590BEA302E3427FC7A718261
:109ACA007A6183E0B41A456CDD80360A3D2E34276C
:109ADA00AB7A71827A61837AEBD07E5002AC5D2ECA
:109AEA002426437A51827A41830BEA304E3400109D
:109AFA007A51827A41831BEA300BD090792A7AEB29
:109B0A00D0907929E0BCDB40C202A1786CDD9000DC
:109B1A00590BEA309079E71BEA306CFF9079E70B32
:109B2A00EA307D230B241BEA202E3427FC7A71822B
:109B3A007A6183E09079EDF0BEB01A68279079EDEA
:109B4A00E0BEB00A681E9079ED7EEBA07C7F0BF038
:109B5A000A372E3479EE7A71827A61837AEBA0BE63
:109B6A00F05040B89079EDE0BEB01A780302A178BF
:109B7A00E40A3F2E3479EE7A71827A6183F0907921
:109B8A00EEE0BEB03B6893BEB020688E608C7E3437
:109B9A007A527E240001907B62793E00021BEA2001
:109BAA007E347A667E240001907B5E793E00021B39
:109BBA00EA207E347AA27E240001907B5A793E0004
:109BCA00021BEA207E347B1A7E240001907B5679A0
:109BDA003E00021BEA207E347B227E240001907B19
:109BEA0052793E00021BEA207E347B2A7E24000141
:109BFA00907B4E793E00021BEA207E347B327E2423
:109C0A000001907B4A793E00021BEA207E347B38B1
:109C1A007E240001907B46793E00021BEA207E14D6
:109C2A0079EE7E0400017E34DA477E2400FF12B901
:109C3A00AC7E147A527E04000112D6697CB7907900
:109C4A00E9F06CEE02A16A9079E9E00A3BCA397E32
:109C5A003014AC3E2E1401777E0400017E347A5211
:109C6A007E24000112D6341BFD600302A168BED017
:109C7A003C400302A1686CCC7E147A667E04000123
:109C8A0012D6697CB79079EAF07E147A667E04006F
:109C9A0001742F12D679BE1800007803029D6B6CEE
:109CAA00FF80310A3F7D232E247A667A51827A41D7
:109CBA00837EEBA02E347A8E7A71827A61837AEB74
:109CCA00A00BC0BEA02F780AE47A71827A6183F071
:109CDA00800A0BF09079EAE0BCFB40C77E147A8ECA
:109CEA007E04000112B9DF7F607F717E7008AC7E4E
:109CFA002E34168F7A71827A61831BEAC079DE006C
:109D0A000279EE000479FE00066CFF80200A2F0A11
:109D1A003C2D322E347A667A71827A6183E00A3F68
:109D2A002E347A8E7A71827A6183F00BF00A3C9033
:109D3A0079EAE00A2B9D230A3FBD3240D0E40A3F6C
:109D4A002E347A8E7A71827A6183F07E147A8E7ECC
:109D5A0004000112B9DF7F607F717E7008AC7E80DB
:109D6A00337E147A667E04000112B9DF7F607F7148
:109D7A007E7008AC7E7D232E24168F7A51827A411A
:109D8A00831BEAC079DE000279EE000479FE000640
:109D9A009F669F772E34202B7A71827A61831BEA21
:109DAA00C079DE000279EE000479FE00066CCC7EF2
:109DBA00147AA27E04000112D6697CB79079EAF07F
:109DCA00E49079EBF0E49079EBF06CFF80380A2CA0
:109DDA000A3F2D322E347AA27A71827A6183E00A9E
:109DEA003F2E347B067A71827A6183F07A71827AA5
:109DFA006183E0BEB02C6802700AE47A71827A61EB
:109E0A0083F080120BF00A3C9079EAE00A2B9D233A
:109E1A000A3FBD3240B87E147B067E04000112B9A7
:109E2A00DF7F607F719079EB7EEB507408AC5B7ECC
:109E3A007020AC7E2D322E34186F7A71827A61834B
:109E4A001BEAC079DE000279EE000479FE00060AF8
:109E5A002C0A3F2D322E347AA27A71827A6183E0FB
:109E6A00704A9079EBE0049079EC9F669F77F080D6
:109E7A00309079EC7EEB507408AC5B7E7020AC7E3F
:109E8A002D322E34186F7A71827A61831BEAC07977
:109E9A00DE000279EE000479FE00069079ECE00417
:109EAA00F09079ECE0BEB00440C780177CBF042C68
:109EBA00CB9079EBE004F09079EBE0BEB00450036C
:109ECA00029DD46CCC7E147AA27E040001742F12F7
:109EDA00D679BE18000068756CFF80160BC00A3F61
:109EEA002E347AA27A71827A6183E0BEB02F680A30
:109EFA000BF09079EAE0BCFB40E26CFF80200A2F6D
:109F0A000A3C2D322E347AA27A71827A6183E00A6F
:109F1A003F2E347B067A71827A6183F00BF00A3C19
:109F2A009079EAE00A2B9D230A3FBD3240D0E40A29
:109F3A003F2E347B067A71827A6183F07E147B0627
:109F4A007E04000112B9DF7F607F7180049F669FE3
:109F5A00777E7008AC7E2E34220B7A71827A618306
:109F6A001BEAC079DE000279EE000479FE00069051
:109F7A007B1AE04420249D681424FD681424F168A7
:109F8A0008240978107401800D7402800974038012
:109F9A000574048001E40A3E2E3426077A71827A17
:109FAA006183F0907B22E04420249D681424FD689C
:109FBA001424F16808240978107401800D74028051
:109FCA00097403800574048001E40A3E2E3425CB0B
:109FDA007A71827A6183F0907B2A7EEBA04EA02070
:109FEA00BEA06378187E5002AC5E2E2426437A51B6
:109FFA00827A41830BEA305E34FFFE801BBEA06D7D
:10A00A00781F7E5002AC5E2E2426437A51827A4112
:10A01A00830BEA304E3400017A51827A41831BEA7B
:10A02A0030907B32E04420B46D187E5002AC5E2E34
:10A03A002426437A51827A41830BEA304E34000255
:10A04A0080167E5002AC5E2E2426437A51827A41D3
:10A05A00830BEA305E34FFFD7A51827A41831BEA30
:10A06A0030907B387EEBA04EA020BEA0697821906C
:10A07A007B39E04420B472187E5002AC5E2E24264E
:10A08A00437A51827A41830BEA304E3400048016B7
:10A09A007E5002AC5E2E2426437A51827A41830B8B
:10A0AA00EA305E34FFFB7A51827A41831BEA30BE82
:10A0BA00A06B7821907B39E04420B472187E50025C
:10A0CA00AC5E2E2426437A51827A41830BEA304EC3
:10A0DA0034000880167E5002AC5E2E2426437A5144
:10A0EA00827A41830BEA305E34FFF77A51827A41F1
:10A0FA00831BEA300A3D7D232E2427AB7A51827ACC
:10A10A0041837AEBE07E3002AC3E2E1426437A314C
:10A11A00827A21830BEA204E2400107A31827A2136
:10A12A00831BEA207E3014AC3E2E1401777E040095
:10A13A0001907B62791E00021BEA000B34907B605F
:10A14A001BEA307E14DA177E0400FF12B95EE4902F
:10A15A007B38F00BD090792A7AEBD0029B240BE063
:10A16A00907929E0BCEB5003029C51029B2412A275
:04A17A000FDA3B229B
:105C3A00CA3B6D339079911BEA306D339079931B8F
:105C4A00EA301214007E14D9E37E0400FF12062300
:105C5A009000590BEA60801B12D4B37CFB7D360B93
:105C6A00642E3427FC7A71827A61837AEBF0BEF073
:105C7A001A6806BE644E1F40DF9000590BEA606C3A
:105C8A00EE7D360B642E3427FC7A71827A61837E2C
:105C9A00EBF0BEF01A7803026560BEF00A68187C61
:105CAA00AE0BE00A3A2E3479957A71827A61837A58
:105CBA00EBF0BEE03C40CAE40A3E2E3479957A7194
:105CCA00827A6183F0907995E0B431B37E3427E823
:105CDA007E240001907B62793E00021BEA207E341A
:105CEA0000327E240001907B5E793E00021BEA208E
:105CFA007E34003A7E240001907B5A793E00021BD2
:105D0A00EA207E34004A7E240001907B56793E00C8
:105D1A00021BEA207E347A0D7E240001907B5279A0
:105D2A003E00021BEA207E3479917E240001907B9A
:105D3A004E793E00021BEA207E1479957E0400010A
:105D4A007E34D9CD7E2400FF12B9AC907A0EE0449D
:105D5A002090002EB472090BEA304E3400108007EE
:105D6A000BEA305E34FFEF1BEA3090002EB4610973
:105D7A000BEA304E34100080070BEA305E34EFFF36
:105D8A001BEA30907A0DE04420B4730C90002C0B7F
:105D9A00EA305E34FFF7800DB46E0D90002C0BEAEA
:105DAA00304E3400081BEA309F449F5590003A0B4E
:105DBA00EA00691E0002692E0004693E000612B755
:105DCA00C190003A0BEA80699E000269AE0004693C
:105DDA00BE0006500D7E04BFF06D119F1112B6125F
:105DEA00800D7E0440767E1480009F1112B4FD90CF
:105DFA0000421BEA00791E0002792E0004793E0057
:105E0A00069079910BEA30BE34012C7803E4803095
:105E1A00BE3404B0780474018026BE340960780464
:105E2A007402801CBE3412C0780474038012BE341B
:105E3A002580780474048008BE344B007806740503
:105E4A0090006BF06CEE7D360B642E3427FC7A7171
:105E5A00827A61837EEBF0BEF01A7803026560BE37
:105E6A00F00A68187CAE0BE00A3A2E3479957A71FA
:105E7A00827A61837AEBF0BEE03C40CAE40A3E2EA5
:105E8A003479957A71827A6183F0907995E0B432A7
:105E9A00B37E3476967E240001907B62793E0002BE
:105EAA001BEA207E3476987E240001907B5E793E40
:105EBA0000021BEA207E34769A7E240001907B5AE7
:105ECA00793E00021BEA207E34769C7E24000190F3
:105EDA007B56793E00021BEA207E3479E57E240057
:105EEA0001907B52793E00021BEA207E1479957E4E
:105EFA000400017E34D9BA7E2400FF12B9AC90792D
:105F0A00E5E0442090002EB466090BEA304E344096
:105F1A000080070BEA305E34BFFF1BEA3012B05F25
:105F2A006CEE7D360B642E3427FC7A71827A61839B
:105F3A007EEBF0BEF01A7803026560BEF00A6818BC
:105F4A007CAE0BE00A3A2E3479957A71827A6183B3
:105F5A007AEBF0BEE03C40CAE40A3E2E3479957AE8
:105F6A0071827A6183F0907995E0B433B37E3476A6
:105F7A00A67E240001907B62793E00021BEA207E05
:105F8A003476AA7E240001907B5E793E00021BEAE9
:105F9A00207E34769E7E240001907B5A793E000250
:105FAA001BEA207E3476A27E240001907B56793E3D
:105FBA0000021BEA207E1479957E0400017E34D902
:105FCA00AA7E2400FF12B9AC6CEE7D360B642E3427
:105FDA0027FC7A71827A61837EEBF0BEF01A78032D
:105FEA00026560BEF00A68187CAE0BE00A3A2E34ED
:105FFA0079957A71827A61837AEBF0BEE03C40CA85
:10600A00E40A3E2E3479957A71827A6183F0907926
:10601A0095E0B434B37E3479E57E240001907B6246
:10602A00793E00021BEA207E3479F97E2400019031
:10603A007B5E793E00021BEA207E3476E57E2400F0
:10604A0001907B5A793E00021BEA207E3476E67E76
:10605A00240001907B56793E00021BEA207E3479A7
:10606A00937E240001907B52793E00021BEA207E37
:10607A003400527E240001907B4E793E00021BEAD6
:10608A00207E1479957E0400017E34D9917E240005
:10609A00FF12B9AC9079E5E04420249778030261B5
:1060AA008024F06827240E68030261A9E49076E24E
:1060BA00F09079ECE04420B4370280030261A990A1
:1060CA00002E0BEA304E3400200261A6740190764D
:1060DA00E2F09079EAE0442090002CB477090BEAC8
:1060EA00305E34FFBF80070BEA304E3400401BEAB3
:1060FA00309079EB7EEBA0BEA0387825742190769B
:10610A00E3F074119076E4F09000300BEA304E34EC
:10611A0000041BEA309000300BEA305E34FFFD8049
:10612A007B9079EB7CBA4420F0B46F2574019076A9
:10613A00E3F074019076E4F09000300BEA305E34BC
:10614A00FFFB1BEA309000300BEA305E34FFFD8023
:10615A004B742E9076E3F0741E9076E4F090003043
:10616A000BEA305E34FFFB1BEA309000300BEA305A
:10617A004E340002802674029076E2F09079E9E0CB
:10618A004420F0B4730C9000300BEA304E34001007
:10619A00800A9000300BEA305E34FFEF1BEA309041
:1061AA0079F9E04420B4660C90002C0BEA304E34A6
:1061BA000080800DB4610D90002C0BEA305E34FF34
:1061CA007F1BEA309079930BEA30BE34258078043D
:1061DA0074038015BE344B0078047404800BBE34FB
:1061EA0004B07803E48002740290006CF0C2CA9092
:1061FA00006C7EEB707402AC7B2E3400617A718283
:10620A007A61830BEA307D235E24FF000A54F5CBC2
:10621A00F5CD7D535E5400FFF5CAF5CCD2CA6CEEBB
:10622A007D360B642E3427FC7A71827A61837EEB89
:10623A00F0BEF01A7803026560BEF00A68187CAEF8
:10624A000BE00A3A2E3479957A71827A61837AEB75
:10625A00F0BEE03C40CAE40A3E2E3479957A718257
:10626A007A6183F0907995E0B435B37E3479E57E2E
:10627A00240001907B62793E00021BEA207E34767C
:10628A00BA7E240001907B5E793E00021BEA207EE2
:10629A003476BE7E240001907B5A793E00021BEAC6
:1062AA00207E3476D67E240001907B56793E000209
:1062BA001BEA207E3476DA7E240001907B52793EF6
:1062CA0000021BEA207E3476DE7E240001907B4E9B
:1062DA00793E00021BEA207E1479957E0400017E35
:1062EA0034D97B7E2400FF12B9AC9079E5E09000A6
:1062FA002CB431090BEA304E34001080070BEA3017
:10630A005E34FFEF1BEA306CEE7D360B642E3427C9
:10631A00FC7A71827A61837EEBF0BEF01A7803020E
:10632A006560BEF00A68187CAE0BE00A3A2E347932
:10633A00957A71827A61837AEBF0BEE03C40CAE4D6
:10634A000A3E2E3479957A71827A6183F090799532
:10635A00E0B436B37E347A0D7E240001907B6279F4
:10636A003E00021BEA207E3476F57E240001907BF3
:10637A005E793E00021BEA207E3476F97E24000113
:10638A00907B5A793E00021BEA207E3479E57E240E
:10639A000001907B56793E00021BEA207E3479F98F
:1063AA007E240001907B52793E00021BEA207E3453
:1063BA0079257E240001907B4E793E00021BEA205B
:1063CA007E3479277E240001907B4A793E00021BA5
:1063DA00EA207E1479957E0400017E34D9627E24F7
:1063EA0000FF12B9AC907A0DE090002EB431090B7F
:1063FA00EA304E34020080070BEA305E34FDFF1BA0
:10640A00EA30907A0EE090002EB431090BEA305E41
:10641A0034F7FF80070BEA304E3408001BEA30904D
:10642A0079E5E04420249D681424FD681424F16869
:10643A0008240978107401800D740280097403809D
:10644A000574048001E4907707F09079F9E044201C
:10645A00249D681424FD681424F16808240978101E
:10646A007401800D7402800974038005740480012C
:10647A00E4907708F06CEE7D360B642E3427FC7AB4
:10648A0071827A61837EEBF0BEF01A78030265604E
:10649A00BEF00A68187CAE0BE00A3A2E3479957A77
:1064AA0071827A61837AEBF0BEE03C40CAE40A3E2C
:1064BA002E3479957A71827A6183F0907995E0B475
:1064CA0037B37E3479E57E240001907B62793E0001
:1064DA00021BEA207E3476C27E240001907B5E791C
:1064EA003E00021BEA207E3476C67E240001907BA1
:1064FA005A793E00021BEA207E3476CA7E240001C5
:10650A00907B56793E00021BEA207E3476CE7E24AA
:10651A000001907B52793E00021BEA207E14799595
:10652A007E0400017E34D94F7E2400FF12B9AC905C
:10653A0079E5E090002CB431090BEA304E340020A2
:10654A0080070BEA305E34FFDF1BEA307E14D92D58
:10655A007E0400FF80087E14D9087E0400FF12061C
:04656A0023DA3B22D3
:10A9C900CA3B90002C0BEA304E3410001BEA309041
:10A9D900002C0BEA305E340002687690792BE01A7D
:10A9E9003B2E3427AB7A71827A6183E01A4B3E445D
:10A9F9003E443E447D542E54202B7AB1827AA18361
:10AA09000BEA00691E0002692E0004693E00061265
:10AA1900B8837EF486A07EE400017F0712D0D3902C
:10AA290079ED793E00021BEA207D542E54220B7ADF
:10AA3900B1827AA1830BEA00691E0002692E000423
:10AA4900693E000612B8837F0712D0D39079F1804E
:10AA59000F9F119079F1793E00021BEA209079ED60
:10AA6900793E00021BEA207E14D8F17E0400FF1211
:10AA790006237E14D8B27E0400FF120623748012C6
:10AA890002187E14D8A07E0400FF12043674C01286
:10AA990002187E14D88E7E0400FF02AF737E14D88C
:10AAA900817E0400FF1206237E1479617E04000171
:10AAB9001290207E1479617E04000112D6697CE728
:10AAC9007E3479B17E240001907B62793E00021BBD
:10AAD900EA207E3479CF7E240001907B5E793E00A6
:10AAE900021BEA207E1479617E0400017E34D87B42
:10AAF9007E2400FF12B9AC9079617EEBD07CBD4415
:10AB09002024C1780302AF3E24DE780302ADBE24BF
:10AB1900FB682B24F9780302AC9C24FA780302AE73
:10AB2900E214780302AE642403680302AF5B900069
:10AB39002C0BEA305E34EFFF1BEA3002AF799079D3
:10AB4900627EEBC07CBC4420B47502800302ABE793
:10AB59006CFF0A3F7D232E2479637A51827A4183DF
:10AB6900E02E3479437A71827A6183F00BF0BEF07A
:10AB79000978DFE490794CF07E1479437E04000172
:10AB890012D5679079F1691E00020BEA002F109027
:10AB9900770D793E00021BEA207E08000A90770DA6
:10ABA90012D0D3793E00021BEA2090792BE01A3BA0
:10ABB9002E3427AB7A71827A6183E012A71774C0A9
:10ABC9001202187E14D8697E0400FF12043674C379
:10ABD9001202187E1479437E04000102AF737CBC13
:10ABE9004420B46402800302AC816CFF0A3F7D23D8
:10ABF9002E2479637A51827A4183E02E3479437A1B
:10AC090071827A6183F00BF0BEF00978DFE4907904
:10AC19004CF07E1479437E04000112D5679079EDDA
:10AC2900691E00020BEA002F10907709793E000295
:10AC39001BEA207E08000A90770912D0D3793E00DA
:10AC4900021BEA2090792BE01A3B2E3427AB7A714C
:10AC5900827A6183E012A4E774C01202187E14D8C4
:10AC6900577E0400FF12043674C31202187E147949
:10AC7900437E04000102AF737E14D82F7E0400FFC7
:10AC890012062374C01202187E14D81E7E0400FF17
:10AC990002AF739079627EEBC07CBC4420B4756DC1
:10ACA90074C01202187E14D88E7E0400FF12043676
:10ACB90074C01202187E1479617E040001120436F0
:10ACC900907963E04420249D681424FD681424F1DC
:10ACD9006808240978157401800A740280067403CF
:10ACE90080027404907705F002AD8CE4907705F04A
:10ACF90074C01202187E14D80D7E0400FF120436A7
:10AD09007E14D7EE7E0400FF12062380767CBC44B5
:10AD190020B46402800302ADA374C01202187E1429
:10AD2900D88E7E0400FF12043674C01202187E14F5
:10AD390079617E040001120436907963E04420248D
:10AD49009D681424FD681424F16808240978147492
:10AD590001800A74028006740380027404907706E5
:10AD6900F08020E4907706F074C01202187E14D89F
:10AD79000D7E0400FF1204367E14D7CF7E0400FF37
:10AD890012062390792BE01A3B2E3427AB7A718275
:10AD99007A6183E012A27F02AAA67E14D7AA7E0452
:10ADA90000FF12062374C01202187E14D7997E047C
:10ADB90000FF02AF73BEE00A501B7E14D7737E04F6
:10ADC90000FF12062374C01202187E14D7617E0494
:10ADD90000FF02AF736CFF0A3F7D232E2479B37AFB
:10ADE90051827A4183E02E3479437A71827A618380
:10ADF900F00BF0BEF00378DFE4907946F07E147929
:10AE0900437E04000112B9DF12B9279076B2793E68
:10AE190000021BEA206CFF0A3F7D232E2479D17A98
:10AE290051827A4183E02E3479437A71827A61833F
:10AE3900F00BF0BEF00278DFE4907945F07E1479EA
:10AE4900437E04000112B9DF12B9279076B6793E24
:10AE590000021BEA2012924402AAA66CFF801C0A77
:10AE69003F7D232E2479627A51827A4183E02E3400
:10AE790079437A71827A6183F00BF0BCFE40E0E499
:10AE89000A3F2E3479437A71827A6183F07E14798C
:10AE9900437E04000112D4E61B3490792B7AEB70BF
:10AEA900BE700E181690792BE01A3B2E3427AB7A18
:10AEB90071827A6183E0BEB000580B7E14D74F7E51
:10AEC9000400FF02AF5590002C0BEA304E34000409
:10AED9001BEA3012389902AAA66CFF801C0A3F7D32
:10AEE900232E2479627A51827A4183E02E34794380
:10AEF9007A71827A6183F00BF0BCFE40E0E40A3F8C
:10AF09002E3479437A71827A6183F07E1479437E93
:10AF19000400011293EB74C01202187E14D88E7EBD
:10AF29000400FF12043674C01202187E1479437E9D
:10AF39000400018035907962E04420B461061290E2
:10AF49009D02AAA67E14D7107E0400FF12062302D2
:10AF5900AAA67E14D6FF7E0400FF12062374C0122F
:10AF690002187E14D6ED7E0400FF12043602AAA64A
:03AF7900DA3B229E
:10B4FA0002BE566E8480007D582D55680E0B556825
:10B50A00EF7D502D5578057F047F15220B5568E095
:10B51A007D5892F77D457D59BF0240127804BF15C8
:10B52A00400C7D487F407F027F257F517F1212BEEB
:10B53A000F5D546E54FFE0E5D0780320D5B2BEC447
:10B54A00FFE0780830E702B2D502BE62A2E792D5E0
:10B55A00BE44FFE068F36CAA7DD47D4C9D4D6843E0
:10B56A00BE4406A078117CA13EA03EA03EA07F0466
:10B57A007F157D4C02BE3250F5800C2E4400202FE0
:10B58A00002F1150020B305C9978F00B8080107CF0
:10B59A00A77C767C657C547C437C327C210A001B28
:10B5AA008078EC7D4C30E52D9F409F5150021B4C1A
:10B5BA007F047F154D894D8A4D8B78122202BE5D1C
:10B5CA009E44002068F72F002F1150020B307CB1E7
:10B5DA0030E4ED80302F042F1550042E0800017C32
:10B5EA00B130E5212E440020780302BE626CAA1E07
:10B5FA001092F71E144C2A92F71E244C4A92F71EF8
:08B60A00344C6A92F702BE32D3
:10B612005D0068115D8878182D002E040020680DE9
:10B622009F117F01222D882E84002078F702BE56BA
:10B6320012BE0F5D542E540020680A2E44804050E2
:10B64200072D4C500A02BE622D4C400302BE5D7DA6
:10B65200514D524D53780BA5B920077F157F040237
:10B66200BE477D594D5A4D5B7806BE84002068EF77
:10B672007DF3ADFB7DFE6DEE7DDBADD22F76E43347
:10B682007DD3ADDA2F7634007DFE0AEB7DD2ADDAC2
:10B692002F76E4337DD1ADDB2F7634007DD9ADD367
:10B6A2002F7634007DFE0AEB7DD0ADDB2F767DD880
:10B6B200ADD32F767DD1ADDA2F76E4337DD9ADD2FD
:10B6C2002F763400AD28ADA02F510A2B7D3E2F518D
:10B6D2007D21AD292F51E4337D287CA1AD90AD129F
:10B6E2002F042C1B7D3AAC5A2F017D2B7D3F7E54BB
:10B6F2000400BE0002500E9E440020780302BE6287
:10B702002F002F1133D5F0F84C3B7CA77C767C655B
:0DB712007C547C437C327C210A0002BE3254
:10B71F0002BE62BE04FFFF6806BE84FFFF7803020D
:10B72F00BE5612BE0F5D54BE54FFE068F27D5C4DF5
:10B73F005468EC5D4478059F117F01222EC4802050
:10B74F0050079D4C380702BE5D9D4C50C37D58C2BB
:10B75F00E44D594D5A4D5B780302BE477E5400109D
:10B76F007EC40037800C1BC468262F002F11500297
:10B77F000B30BF0440107804BF15400A9F049F157B
:10B78F0050021B0C4CAB0330E7DCCAA86CAA80D666
:10B79F00DA1BDA19DA18BE101050149E4400206814
:10B7AF00A52F002F1150020B302CAA50020B700244
:02B7BF00BE3298
:10B7C10074F87EA0FF6E00806E848000BEB0FF68BA
:10B7D100407D4B7C875DB55C7BBF047804BF1568F9
:10B7E10043F4401C7CA97D4B7C9A6CAA6D442F527A
:10B7F10050042E4800016E54FFFF5DB52D158011D8
:10B801007C786CAA6D442F1250042E080001F45C60
:10B811007BBF047804BF15680B7D5820F7067CB008
:05B8210020E701B32245
:0EB826005D006809BE04FFFF68036E0080220B
:10B834007EA020800C7EA01080057EA0086C556D33
:10B84400333392D5500C6E34FFFF6E24FFFF2E1855
:10B8540000012F114006D5F0F97F01227CB41E545B
:10B864001E541E541E542E543FE0A2D592F72F119D
:0FB874002F112F112F117D127D236D337D052292
:10B883007D502D5592D51E541E541E541E541E54C5
:10B893002E54FC0140039F11227C747C637C357C15
:10B8A300527C412F112F112F114E40807E20208C6E
:10B8B300324C732E54FFE0500E7E1CFFFF221E34C9
:10B8C3001E2450034E60800478F430D50C6E34FF90
:0AB8D300FF6E24FFFF2E1800012273
:10B8DD0002BE6268FB02BE567CB5330A543392D564
:10B8ED00602A046C442F1160EA2F112F112F112F94
:10B8FD00112E54037F7E440020AD457D457C147C84
:10B90D00257C367C476C556D3302BE479F117F01F8
:01B91D002207
:10B91E0002CCC102CCBE02CCB9E47C517D312F11D8
:10B92E00332F11332F11334C7B2D0092D5681E0B04
:10B93E000568E32E048FFE50DABE002050D22D0093
:10B94E002D002D005C0068CB7C8002CC9B9F1122C9
:10B95E007F507EC400017ED47B667E94B96F02BF99
:04B96E006C40012206
:10B972007CEACA89CA5BCA6B12D14BDA6BDA5BDA30
:08B98200897E94B96F7CAE22AE
:10B98A007F707F517EC400017ED47A917E94B99DE6
:0AB99A0002BF6C4005E47A7BB02286
:08B9A4007A7BB02E780001222D
:10B9AC007F707F517EC400017ED47B667E94B9BFCC
:06B9BC0002C3DF4001227E
:0EB9C20010F7087E7BB02E780001221B7C223D
:0FB9D000BE04FFFF68087CB030E7036E008022E2
:10B9DF007F409F556CAA7F157F057E4BB02E480088
:10B9EF000112D4A240F4CA4B12BE70DA4B400122AE
:09B9FF007E4BB02E48000180EDE2
:10BA080002BE5602BE627D5020F7F55E547FF06894
:10BA18007ABE547FF068ECCA0BCA1B7C017C125EAC
:10BA2800001F4E00109E543FF00E5430E304C2E352
:10BA38002D002E543FF07E145370AD107C327C21C3
:10BA48000A002E0887FF2E04000BBE102040077E38
:10BA5800101F7E14FFFF5E100F4D05758304CA0B7F
:10BA6800CA1B7F407F51690FFFF1691FFFF3692FE0
:10BA7800FFF5693FFFF712B722DA5BDA4B12B5011F
:0CBA88009E040010D583D79EF800082211
:10D1AE00CA79CA0BCA1B690FFFF9691FFFFB692FEA
:10D1BE00FFFD693FFFFFBE0800007804BE180000A7
:10D1CE0078449F669F77690FFFED691FFFEF692F08
:10D1DE00FFF1693FFFF37F467F5712B7C128079FC4
:10D1EE00009F1102D3047E1CFFFF793FFFEF792FC2
:10D1FE00FFED7E0CFFFF7F1F2E34FFF17911000231
:10D20E001B1A0002D2F46D779F449F55690FFFF9E8
:10D21E00691FFFFB692FFFFD693FFFFF12B7C1506A
:10D22E0061690FFFED691FFFEF692FFFF1693FFF86
:10D23E00F312B8837D737D27E412B8397F407F5196
:10D24E00690FFFED691FFFEF692FFFF1693FFFF3D4
:10D25E0012B4FDBE0800007804BE1800007887697D
:10D26E000FFFF9691FFFFB692FFFFD693FFFFF12DB
:10D27E00B826790FFFF9791FFFFB792FFFFD793F54
:10D28E00FFFF690FFFF9691FFFFB692FFFFD693F64
:10D29E00FFFF12C8DD698FFFED699FFFEF69AFFFDA
:10D2AE00F169BFFFF312B61212C7F4790FFFED79D1
:10D2BE001FFFEF792FFFF1793FFFF37D375E3400CB
:10D2CE00016823690FFFED691FFFEF692FFFF169F9
:10D2DE003FFFF312B826790FFFED791FFFEF792F7D
:10D2EE00FFF1793FFFF3690FFFED691FFFEF692F24
:0DD2FE00FFF1693FFFF39EF80008DA792286
:10BA94003DD20C62C2F2D7F5BE3B6E24F44B128F3A
:10BAA4003E9F9D38A3763CC3BEFA6D1F2A204A8C64
:10BAB4003F4E1F506891BABBBF955D3C7E3CBFFAB8
:10BAC4003FD03C1F081B5AC4BFF3BD3CC9BE45DE72
:10BAD4003FF0000000000000BE06FADB9F1557444B
:10BAE4003E6E8F434D018D63BECE3074FDE8871FDB
:10BAF4003F250783487EE782BF732D2CCE62BD8627
:10BB04003FB466BC6775AAE2BFE4ABBCE625BE538E
:10BB14003FF921FB54442D184031BB797BC569F8AA
:10BB2400C08926DDB9C83D0240B93227D3304CB9AB
:10BB3400C0B61F0795DE70E03FF000000000000073
:10BB4400C062FEA685FF2B0D40A5FF4E58DEAD6EEC
:10BB5400C0C15FBBAA8C6A2212BC1B04A2E192F78B
:10BB64001420E020CAA8CA3B7E74BA947E6400FF05
:10BB7400740812C705DA3B802912BC1B30E102B2FB
:10BB8400F720E0E0CAA8CA0BCA1BCA3B7E74BADC21
:10BB94007E6400FF740712C705DA3BDA5BDA4B12E6
:10BBA400B612DAA85D0068055EA0806C0A2212BC99
:10BBB4001BCA59CA3BCA0BCA1B7E74BB3C7E6400B9
:10BBC400FF740312C705698FFFF9699FFFFB69AF13
:10BBD400FFFD69BFFFFF12B6127F407F51DA1BDA07
:10BBE4000BCA4BCA5B7E74BB1C7E6400FF740312D9
:10BBF400C705DA5BDA4BDA3BDAB830E00912B72270
:10BC0400DAA8B2F7809E7F207F047F427F217F15D0
:10BC14007F5212B722808B7CA05E007FBE0441E07D
:10BC240040051BFD02BE56CAA87E843FC47E945FB5
:10BC3400307EA46DC97EB4C88312B612BE043FF030
:10BC440040107F407F5112B88312B8346E008012C6
:10BC5400B501E45D0068262E040030BE043FF040C8
:10BC64001C7F407F5112B8837CB704C2E07C4BCA6E
:10BC7400B812B83E6E008012B501DAB8035D0068F0
:08BC8400049E040010DAA8225E
:10BC8C003FBC37E9AD397134BFC2490B4D51190175
:10BC9C003FC9999990956BB6BFD555555554C52943
:10BCAC003FF00000000000003FBFD5BA9AAC2F6EE9
:10BCBC003FCF5B75F92C80DE3FD6F61941E4DEF1FF
:10BCCC003FDDAC670561BB4F3FE1E00BABDEFEB483
:10BCDC003FE4978FA3269EE13FE700A7C578463443
:10BCEC003FE921FB54442D187CA05E007FBE047FED
:10BCFC00F04018680302BE567E043FF97E1421FB07
:10BD0C007E2454447E342D1802BE005EA080CAC826
:10BD1C007CCA7CB1540F7D406C9BBE443FF04016F6
:10BD2C00780260127F407F517E043FF06D119F11AD
:10BD3C0012B7224EC0407D405E90F02D449E447F51
:10BD4C006040567EA0A09CA97CB1540F44109EA0CC
:10BD5C00201EB05CAA78F734004CCB7F407F51CAD0
:10BD6C000BCA1B7C4BE412B83E9E040030CA0BCAB3
:10BD7C001B12B6127E843FF06D999F5512B5017F50
:10BD8C00607F71DA5BDA4BDA1BDA0BCA6BCA7B1297
:10BD9C00B4FDDA5BDA4B12B722CA0BCA1BCA3B7E64
:10BDAC0074BC8C7E6400FF740412C705DA3BDA5B4A
:10BDBC00DA4B12B6127CBC540F7EA008A4681A2E63
:10BDCC0054BCAC7E4400FF0B2A806992000269A22D
:10BDDC00000469B2000612B5017CAC30F6167E8404
:10BDEC003FF97E9421FB7EA454447EB42D186E0042
:10BDFC008012B5015D0068085E007F5EC0804C0C4F
:03BE0C00DAC8226F
:0AD30B0012B82612D31512B826221C
:10D31500CA0BCA1B9F449F5569CFFFF969DFFFFB05
:10D3250069EFFFFD69FFFFFF7F067F1712B7C15049
:10D33500707F1F2E34FFF9CA1B7F067F1712B82690
:10D3450012D3D81BFEBE0800007804BE1800006882
:10D355002B7E843FF06D999F55690FFFF9691FFF7B
:10D36500FB692FFFFD693FFFFF12B501790FFFF93B
:10D37500791FFFFB792FFFFD793FFFFF690FFFF94C
:10D38500691FFFFB692FFFFD693FFFFF12B8267973
:10D395000FFFF9791FFFFB792FFFFD793FFFFF8015
:10D3A5001D7F1F2E34FFF9CA1B690FFFF5691FFF8B
:10D3B500F7692FFFF9693FFFFB12D3D81BFE690FF1
:10D3C500FFF9691FFFFB692FFFFD693FFFFF9EF80E
:03D3D5000008222B
:10BE0F007D5054F0B2E46D05B2E42D557D4592D5C9
:10BE1F007D5854F0B2E46D85B2E42D557DC55002C6
:10BE2F00B2D52230F7122E180001780C2E0800011F
:10BE3F0078062E440020681B1E4430D5034E8080A8
:10BE4F005E04000F4D04227E1CFFFF7F01229F1115
:10BE5F007F01227E04FFF020D5021E006D119F117D
:01BE6F0022B0
:10BE700020F20CB42D04D2F2D322B42B02D322240C
:10BE8000D05043BEB00A503E30F3127E94000AAD4B
:10BE90009B0ABB2DB9BEB407FF504AD322D2F1CAC8
:10BEA0005BCA597E8440246D999F5512B6127F401B
:10BEB0007F51DA48E412B83E12B501DAA8DA5B30F5
:10BEC000F0B61BA4D32220F324B4FE0720F01ED228
:10BED000F0D32224EB600424E07012A2F292F0D29C
:10BEE000F3C2F2D322C37E1CFFFF7F01226D4430D8
:10BEF000F30B9D4B20F2027D4BA2F092F230F1E564
:10BF00002D4A20D2E07CB83392F350066E44FFFFF6
:10BF10000B44BE44013450CDCAA87D54CA0BCA1B81
:10BF200012CA82DA1BDA0B7EFBA020F30512B612CE
:0FBF3000800312B722DAA830F20312B826C32218
:10BF3F00540F2490D43440D430F30CBEB04140079A
:10BF4F00BEB05B500224204CCC68021BC00B84D3C4
:10BF5F0089944CCC680B742012BF5680F5CA3B6D88
:10BF6F00889F337CAE7E5BB02E5800017007C37D77
:10BF7F0038DA3B8994B4256BC2F37E5BB02E580040
:10BF8F0001A5F824D0BEB00A501B7E500A20F60D32
:10BF9F00AC5CA52D7CCB70034EF00180DBAC5DA5B6
:10BFAF002D7CDB80D324CFBEB01AA5E850055E00F0
:10BFBF00DFD2F390C367A3E4936011BCB078F7743A
:10BFCF0017934CAB30F6B14EF08080ACA3E4936086
:10BFDF0010BCB078F77416937C3B7423937C2B8939
:10BFEF00147CB08013742012BF5620F205BEC0021D
:10BFFF0050F31B6D29B6000112BF5602BF611B6EB5
:10C00F00691600020B6A00BE08000078087E040063
:10C01F00FF7E14D6E920F2204CCC681C7F10E47E02
:10C02F001B804C8868092E18000104BCBD78F0C233
:10C03F00F6CA0B12C145DA0B7E0BB060BECA0B12EB
:10C04F00BF56DA0B2E0800014CDD68EC1BD078E8E8
:10C05F0080A9D2F07E101080037E10085EB05F8042
:10C06F000AD2F67E100A80057E100AC2F66D119F65
:10C07F00117E00201B6C7E6B7030F6021A3720F198
:10C08F00051B6C7E6B6030F6041A261A2430F005FF
:10C09F001B6D0B6A20A5EC3382F692F6500A7CEAF0
:10C0AF009F229F217F127CAE4C44780F7C457C569B
:10C0BF007C676C772E00F878EF80122F117CB333EA
:10C0CF007C3B9CB140047C3B0B70A5D8EE7CB2301E
:10C0DF00E005DAB8C44C3BCA380B207E00207E3016
:10C0EF0000BE18000078C1BE1008780730F404C2F3
:10C0FF00F480B5CA287CB2BCBD38027CBD12C145E4
:10C10F00DA28BC2D500A1BD0E4CA2812BF3F80F09A
:10C11F007CB213DAB84004C4CAB8C4CA28BEF080CF
:10C12F0040095CDD7805A5DA02600312BF3FDA280B
:10C13F00A5DADD02BF61BEF001680F30F402240200
:03C14F0020F506D2
:10C1520020F70330F6010420F229BCBC5025CAB8EE
:10C162007CBF13B0E67420501174307C8A5E80F07C
:10C17200680812C1855EA00F800312BF56DAB8BCF0
:10C18200BC78DB30F40F743012BF56745830F302AF
:10C19200747812BF5630F605742D02BF56742B20E8
:10C1A200F5F8742020F7F3221B6C7E6BB010F102BD
:10C1B2001B6C20F60B30E704F404D2F27CCB800532
:10C1C20020E7057CDB02BF875EF07F80F81B6E698B
:10C1D2001600020B6A0030F0096D221B0A202E089D
:10C1E20000021B0A8002BF70E46C22BE3010500BAA
:10C1F2007F1F2D312E34FFEE7E39B0227CBF20E727
:10C20200A6742E4EF08002BF5612C34140437CBD3D
:10C212007003047CDB12CC3F7C3D4C3368101B3036
:10C222007CBE20E40912C1EA70044C3378F07CBD74
:10C232007CD3BE44FFFC48216CAABD45581B6D55FA
:10C242009D546C222D511801E47CDB02C2E512C31D
:10C252004140787CBD0412CC3F7DA47CAE7CBDA263
:10C26200F492F0C2F44002600104240612C1457E39
:10C2720030FF0B3012C1EACA3812BF3F20F0044C23
:10C28200DD680312C1FEDA38BC3D78E6740E12BFD7
:10C292003F742B7D4A7CA830F7086EA4FFFF0BA4E5
:10C2A200742D12BF567E4400647D5A8D547DA412B3
:10C2B200BF3F7D5A7EA00A840AAA12BF3F7D5A124E
:10C2C200BF3F9EF80011DA5B02BF61DA5BD2F27EF9
:10C2D200D00002C02412C34140F10A5D2D540B5418
:10C2E20012CC3F7DA47CB97CAE30E701F40420F48B
:10C2F200044CDD6805D2F0C2F4042CBD12C1456CB9
:10C3020033BEA40000681648101BA412C1EACA3842
:09C3120012BF3FDA380B3080E85D
:10C31B000BA41B3012C1EACA3812BF3F4CDD6807B1
:10C32B0012C1FE1BD080E39EF8001230F00312C145
:10C33B00FEDA5B02BF617CEA7CAF10F7037ED006AE
:10C34B007CFA1B6E693600020B6A201B6E691600A5
:10C35B00020B6A00DA49CA5BCA4902CB162D2B20A5
:10C36B004C4248232E0053584F44494355502A4EB4
:10C37B004645470004208001020010400D636870A1
:10C38B0070F97761AACFD7500BC0C0C0C0C0BFC077
:06C39B00C0C1C1C2C2C214
:04D6E90028302900BC
:09C3A10060291B84D2F7D38994B2
:10C3AA0020F315691600020B6A007A0BB02E0800FA
:09C3BA00011B6A00791600022241
:0AC3C3005CCC68061BC07802E4227F
:08C3CD00D3999460020B842255
:0AC3D50012C3CD12D4A240F880C2BA
:10C3DF00CA3B6D886D776D667CAD7E5BB02E580065
:10C3EF000170070A3EC3DA3B8994B425577E5BB0D0
:10C3FF002E5800017C0B24D0BEB00A500B7E500A81
:10C40F00AC5C2CB57CCB80E524CFBEB01A7CB05091
:10C41F00035E00DF90C6D0A3E4936026BCB078F72C
:10C42F007412937C3B7423937C2B8914D2F080BDC0
:10C43F00D2F180B9D2F380B55CEE78A77E34FFFFDE
:10C44F0080A37CB012D4A2500512C3D580887CFB88
:10C45F0012C3CDBCBF68F560DF12C3A1808520F386
:10C46F00021B6E12C3CD60D05CCC78070BC080036B
:10C47F0012C3CD600712C3AA1BC078F420F40520A5
:10C48F00F3020BE080C6D2F67F057E0B70A5BF5E70
:10C49F00162E0800017E0B7010F605BE705D681A2F
:10C4AF00BCB778EDD380427E0B702E08000110F6DA
:10C4BF0005BE705D68EEBCB778EDC3C2F4802AD2BA
:10C4CF00F520F3021B6ED2F45CCC68020BC020F592
:10C4DF000512C3D5600812C3C3700630F40D02C431
:10C4EF004720F5A2C2F412D4A2500412C3A1E41241
:10C4FF00C3AA70E230F50A7E5BB02E580001B45D1E
:10C50F00F602C48B6CFF800D7EF01080087EF00861
:10C51F0080037EF00AD2F45CCC68020BC012C3D544
:10C52F0060BC12C3CDB42D04D2F28003B42B081219
:0CC53F00C3D560AA12C3CDBEF00A683854
:10C54B00BEF0086833B430295CFF78037EF008C274
:10C55B00F412C3C3BEB0786803B4581C5CCC680C2F
:10C56B001BC07808D2F49F118056D2F07EF0108059
:10C57B000E5CFF78037EF00A9F11604412C3A19FEB
:10C58B0011CA1B12C3C37C8BDA1B6034BEB0614073
:10C59B0007BEB07B5002C2E524D05024BEB00A4087
:10C5AB0007BEB011401A24F9BCBF50147D120A0FFC
:10C5BB00AD30AD102D216D000A1B2F10C2F480C1C0
:10C5CB007CB812C3A120F32C20F40B0BE030F20645
:10C5DB009F009F017F101B6E691600020B6A0030D3
:10C5EB00F006793000027D3220F106397000017CB3
:10C5FB00767A0B7002C3E55CCC68020BC012C3D514
:10C60B00D2F420F05112C3C3700302C4479F11CA66
:10C61B001BCA296CFF800ACA1BCA4912C3CD12C39D
:10C62B00C312C3A1DA49DA1B7CDA7CAFCA7B12CF07
:10C63B0070DA7B7CFA7CAD5004C2F480DA20F41300
:10C64B0020F3101B6E691600020B6A001B0A20797F
:10C65B0030000202C48BCA5BCA4B12C3C360AB9FD0
:10C66B0011CA1BCA1BCA1B6CFF800ECA4BCA0BCA52
:10C67B001BCA5B12C3CD12C3C312C3A1DA5BDA1B95
:10C68B00DA0BCA6BCA7B7CDA7CAF12BE70DA7BDA50
:10C69B006BDA4B7CFA7CAD5004C2F480CE20F41BD9
:10C6AB0020F3181B6E69B600020B6AA01B5A0079A7
:10C6BB001500027925000479350006DA5B80947D3C
:06C6CB00386D2202C5E1FA
:10C6D1004C4248535B58504F444943552A4E4645B6
:10C6E10047003B3FFCD0CE17751C21136D2143CA77
:10C6F100020202C4C4C3C4C4C5C5C5C5C5C4C5C43A
:04C70100C6C6C6C61C
:10C70500CAB87F407F5112B612DAB8CA0BCA1B0BE2
:10C715003A00691300022E3800040B3A20693300F1
:10C72500022E380004698FFFF9699FFFFB69AFFF8F
:10C73500FD69BFFFFFCAB812B6120B3A80699300B4
:10C74500022E3800040B3AA069B300022E3800040B
:0DC7550012B501DAB81478CD9EF800082264
:10C762003CEC36E843B040223D3314964D5878A94C
:10C772003D7816193166D0F93DBC3BD650FC29866E
:10C782003DFE8CAC7351BB253E3E4CF5158B8ECADB
:10C792003E7B5253D395E7C43EB62C0223A5C82450
:10C7A2003EEFFCBFC588B0C73F2430912F86C787B4
:10C7B2003F55D87FE78A67313F83B2AB6FBA4E7776
:10C7C2003FAC6B08D704A0C03FCEBFBDFF82C58F70
:10C7D2003FE62E42FEFA39EF3FF000000000000073
:10C7E200C2D502BE6202BE56A5B9F0F930D5F10239
:10C7F200BE5D7D50A2F792D55E547FF0BE547FF0AD
:10C8020068E67E843FF77E9415477EA4652B7EB44E
:10C8120082FE12B6127D502D5592D554E02E547FD1
:10C8220000501178C730D50C7CB144F0047805BEB5
:10C8320020F050B87F407F5112B883CA396D229DD3
:10C84200237CB412B83912B501CA3B7E74C7627E2A
:10C852006400FF740F12C710DA3BDA593E543E549B
:10C862003E543E547D405E447FF06D042D45780277
:05C872006C004D0422E2
:10C877003FCC951A030000003FD2491B304500000A
:10C887003FD999999BA269003FE555555555419266
:10C8970040000000000000003FF000000000000022
:10C8A7003FF306FE0A31B7133FF6A09E667F3BC7EC
:10C8B7003FFAE89F995AD39D3FC62E42FEFA39E0C8
:10C8C7003FD62E42FEFA39E03FE0A2B23F3BAB60D3
:06C8D70002BE6202BE5623
:10C8DD007D802D8840F7D2D568F0C2D57D982E8405
:10C8ED00002040E65E04800F4E043FF07C817C9278
:10C8FD007CA34E80202F222F222F22E4BE448B9624
:10C90D00401D04BE44A5FF401604BE44C567400F3C
:10C91D0004BE44EAC140082E940020E45E10EFCA24
:10C92D0099232323CA3BCAB8CA0BCA1B0A7B2E7490
:10C93D00C89F7E6400FF0B3A806993000269A300D3
:10C94D000469B3000612B501DA5BDA4BCA0BCA1BD8
:10C95D000B3A0069130002692300046933000612C3
:10C96D00B4FDDA5BDA4B6E84800012B722CA0BCAB3
:10C97D001B7E74C8777E6400FF740412C705DA5BF2
:10C98D00DA4B12B612DAB8601C0A7B2E74C8B77E69
:10C99D006400FF0B3A806993000269A3000469B338
:10C9AD00000612B501DA3BDA49CA0BCA1B1E441E3A
:10C9BD00441E441E441E447D249E2403FF7CB41259
:10C9CD00B8397E843FE67E942E427EA4FEFA7EB474
:0DC9DD0039EF12B612DA5BDA4B12B5012207
:10D3D800CA0BCA1B2EF80008690FFFF1691FFFF37B
:10D3E800692FFFF5693FFFF712B8837CB412B83490
:10D3F800790FFFF9791FFFFB792FFFFD793FFFFFB9
:10D4080069CFFFF969DFFFFB69EFFFFD69FFFFFFE8
:10D41800693FFFED692FFFEB1B1AC079D100027934
:10D42800E1000479F10006698FFFF9699FFFFB6944
:10D43800AFFFFD69BFFFFF690FFFF1691FFFF369C8
:0FD448002FFFF5693FFFF712B4FD9EF800102289
:10C9EA003FF00000000000004024000000000000AA
:10C9FA004059000000000000408F40000000000085
:10CA0A0040C388000000000040F86A0000000000EF
:10CA1A00412E848000000000416312D00000000013
:10CA2A004197D784000000004341C37937E0800072
:10CA3A0044EA784379D99DB44693B8B5B5056E17DB
:10CA4A00483D6329F1C35CA549E5E531A0A1C87356
:10CA5A004B905031E2503DA94D384F03E93FF9F56B
:10CA6A005A827748F9301D3267CC0E1EF1A724EBA3
:10CA7A0075154FDD7F73BF3C5D55684C7D055407C6
:10CA8A00682D23232312CAD27D50CA595E54003816
:10CA9A006809243812CAEC7F407F51DA591E5403C0
:10CAAA000354386809247012CAEC7F407F51227CF3
:10CABA00B154386809243812CAD27D5080DF7D50BB
:10CACA001E540303543824706CAA2E54C9EA7E44B7
:10CADA0000FF0B2A806992000269A2000469B20071
:10CAEA0006226CAA2E54C9EA7E4400FF0B2A00696A
:0ECAFA00120002692200046932000602B61220
:10CB08004E614E002B494E46002D494E46007D4051
:10CB18002D447CAE92F67CEA7CBA68265E90E0BE34
:10CB280044FFE0782F7CB1540F7E0400FF60067E3E
:10CB380014CB08D3227E14CB1120F6047E14CB0C20
:10CB4800D322DA099F22CA2BCA2BCA2BCA2BCA881E
:10CB5800C3CA09221E447E5404D1AD542D54500238
:10CB68000B449E28FA239E440133CA2B7CA15EA065
:10CB78000F7CB21E541E541E541E541E547E440074
:10CB880056CA59AD457E44C5109D450A48DA59AD87
:10CB980054DA492D54DA5950020B54CA59CA4BCAAF
:10CBA8006BCA7BCA0BCA1B20F70C12CA82DA1BDAC3
:10CBB8000B12B72280106E54FFFF0B5412CA82DA90
:10CBC8001BDA0B12B612DA7BDA6BDA4BDA497D50D4
:10CBD8005E04000F6D504E10109E543FB02F002F72
:10CBE8001150020B3024F078F4DA59758210BE0027
:10CBF8000A400A9E000ACA020115820B44CA086C40
:10CC0800007EA4000A7DB1AD0A7D016D11ADAB2F88
:10CC1800057EA4000A7DB3AD2AADAB2D1250020BE0
:10CC2800047D236D332F1550042E080001158278DA
:10CC3800CCCA08C3CA59227F0F20E73ABEB01040B9
:10CC48000274100A0B2D109E1400127E19B02EB01B
:10CC5800FB501F4C116817E47A19B01B147E19B0E9
:10CC6800047A19B0B40A0BE47A19B0A5D9ED0B44CB
:0ACC780074017A19B0225EE0BF22B9
:10CC82002D0092D50E104E10807D422D445002B2DE
:10CC9200D54E50806C447CB8222C44500C2E180087
:10CCA20001A5BD00040B806816A2D57CB8137C4B8D
:10CCB2007CB592E77C5B227E1CFFFF229F11227EC5
:0BCCC20024FF8020D5026C456D33225A
:10CCCD0002CCB96E00807CB1337CB033680D046842
:10CCDD00EF7CB5337CB43378037F10220468E17D9B
:10CCED005092F77D457D51BF2140067C807F017FAD
:10CCFD001212CC827EA1D05CB004780320D5C17C09
:10CD0D00B00478075002B2D502CCC192D5BE80FFD7
:10CD1D0068F67CB89CB06C00602AB418057C4102A2
:10CD2D00CC9B50FB80032F00047C9B5E900778F614
:10CD3D0030E4067C437D106D0030E3087C437C328B
:10CD4D007C210A0030F5199F10780E2202CCBE1BF3
:10CD5D008068F92F1150020B707CB530E7F1801B04
:10CD6D002D317CB5A5397C5B50110B80780302CC3D
:0ECD7D00C11E341350034E60801A2B02CC9B53
:10CD8B005D22680D5D0078122D220B4068099F1102
:10CD9B00222D000B0078F902CCB912CC825C800BEF
:10CDAB00806808248150072CB0500A02CCC12CB0EB
:10CDBB00400302CCBE7C8B5D1178267CB17CA5BE7A
:10CDCB001080680A5D33780DA5BD80057F1002CCFD
:10CDDB00AB6D0080307F017C5B7CB17CA5AD12809C
:10CDEB00245D337806A5BD80F080E1CA887D41AD16
:10CDFB00437CB17CA5AD122D1450020B047C5BADB2
:10CE0B00232F01DA88A42D05BE008040060B807805
:10CE1B000480982F007C437C507C617C7202CC9BFD
:10CE2B00BE24FFFF6806BE04FFFF780302CCB912D5
:10CE3B00CC825CB00468F57CB8A54868EF7CB87010
:10CE4B00039F1122A5B8000302CCC12E008150070D
:10CE5B009C80380702CCBE9C8050ED0A51C2E74D36
:10CE6B0051780302CCAB7E5400807E901A6C00800C
:10CE7B00061B9068142F11BF1040049F104CAB037E
:10CE8B0030E7EECAA86CAA80E8DA39DA587C4ABED9
:10CE9B005080500A1B8068BC2F1150020B7002CCC3
:01CEAB009BEB
:10CEAC0074F86CAA6E40806E0080BEB0FF68277C60
:10CEBC00837C975C3B5C7BBF10682AF4400D7C380C
:10CECC002D15F45C3B500F0B04800B7C792D35F445
:10CEDC005C7B50020B24BF10680B7CB020E7067CF7
:06CEEC00B420E701B322AF
:10CEF2007EA020800C7EA01080057EA0086C556D5F
:10CF0200333392D5500C6E34FFFF6E24FFFF2E1880
:10CF12000001A5EC3340062F11D5F0F6227CBA248D
:0FCF22007EA2D5137C767C65A5CC92E77C5B2242
:10CF31007CB5337CB43392D54E5080248140039F1D
:10CF410011227C457C567C676C7724E0500E7E1C58
:10CF5100FFFF221E341E2450034E60800478F430FB
:0FCF6100D50C6E34FFFF6E24FFFF2E1800012247
:10CF700020F20CB42D04D2F2D322B42B02D32224FB
:10CF8000D0503EBEB00A503930F3137E200AAC298F
:10CF90000A0B2D01BE04003F50467C91D322D2F1F2
:10CFA0007F726D117E04412012CD8B7F017D5F7CED
:10CFB0004BE412CEFC12CCD37F2730F0BB1B80D3C6
:10CFC0002220F322B4FE0720F01CD2F0D32224EB5F
:10CFD000600424E07010A2F292F0D2F3C2F2D322E5
:10CFE000C37E1CFFFF22E430F30B7CB930F202F465
:10CFF00004A2F092F230F1E82CB820D2E3A2E7923A
:10D00000F35002F404B4260050D6CAA87F7112D09F
:10D010006A7F17DAA87DE520F30512CD8B80031215
:0CD02000CE2B7D5E30F20312D02CC32218
:0ED02C005D226809BE24FFFF68036E4080226B
:10D03A003F8000004120000042C80000447A0000FE
:10D04A00461C400047C35000497424004B18968080
:10D05A004CBEBC205A0E1BCA6753C21C749DC5AE77
:10D06A007C7B600654076816232312D08F7CB75442
:10D07A0038680A7F1012D08C12CD8B7F01227CB7C0
:10D08A00543803241C6CAA2E54D03A7E4400FF0B59
:07D09A002A006912000222C6
:0300000002D457D0
:10D457007584017E44041FE47A49B01B4478F97E41
:03D46700F80020AA
:03D49F0002024046
:10D46A007E0400FF7E14FC0B0B0A405D44682629EB
:10D47A005000020A25693000032E0800050B44807B
:10D48A000E7E0BB07A1BB02E1800012E0800011B6D
:05D49A004478EE80D390
:10D0A100C2D57CB430E708B2D56E24FFFF0B247CD7
:10D0B100B630E712B2D56E34FFFF0B348D326E24D9
:10D0C100FFFF0B2480028D3230D5066E34FFFF0B3B
:02D0D100342207
:10D0D3007D51AD037D027D21AD052D12AD352D2191
:01D0E300222A
:10D0E400C2D57CB030E708B2D59F229F207F027C56
:10D0F400B430E713B2D59F229F217F1212D15D9FD6
:10D10400229F207F02800312D15D30D5069F229F8B
:04D11400217F122243
:10D118006CAA6C00BE08000068281E540B54501EF0
:10D128007E1B807A0B802E1800012E080001800ECD
:10D138000B1A401B0A402E1800022E0800021B542E
:03D1480078EE225C
:10D14B00B40A07740D12D155740A3099FDC299F5C2
:02D15B00992217
:10D4A200BEB0094005BEB00E4003B42002D322C371
:01D4B2002257
:10D4B30010000B12D6E1B40D02740A02D14B90791D
:03D4C30042E02222
:10D4C6007D23BE24000048037D32226D339D322227
:10D4D6007F01BE08000048037F10229F119F102283
:10D4E600CA3B7F302EF8000380020B747E3BB012DD
:10D4F600D4A240F674017AFBB07E3BB0BEB02B6876
:10D5060003B42D167F130B747E1BB0BEB02D6805B9
:10D516007E700180026C777AFB706D33793FFFFE77
:10D52600801B690FFFFE7E14000AAD107E3B701A49
:10D53600379E3400302D31793FFFFE0B747E3BB0B1
:10D5460012D6D340DD7EFBB06006693FFFFE800A3F
:10D55600693FFFFE6E34FFFF0B349EF80003DA3B93
:01D5660022A2
:10D56700CA3B7F302EF8000580020B747E3BB01259
:10D57700D4A240F674017AFBB07E3BB0BEB02B68F4
:10D5870003B42D167F130B747E1BB0BEB02D680538
:10D597007E700180026C777AFB709F11793FFFFEE6
:10D5A700792FFFFC80287E08000A693FFFFE692F5C
:10D5B700FFFC12D0D37E3B301A139E1400301A02A0
:10D5C7001A002F10793FFFFE792FFFFC0B747E3B6B
:10D5D700B012D6D340D07EFBB0600A693FFFFE6928
:10D5E7002FFFFC8014693FFFFE692FFFFC6E34FF9D
:10D5F700FF6E24FFFF2E1800019EF80005DA3B227C
:10D60700CA0B80082E1800012E0800017E1BB07A75
:07D617000BB070F0DA1B22DA
:08D61E002E0800012E18000186
:0ED626007E0BB06005BE1BB068EE9E1BB022EE
:10D634007F7180187E0BB0600C693FFFFD1B34794D
:10D644003FFFFD7803E480180B140BF47E7B607EAF
:10D654000B70BC7668DEBC7608047401800274FF2B
:05D664002EF800002279
:10D669006D3380020B347F200B147E2BB070F522B2
:10D679007CABBE08000078037F10227E0BB0BCBAD9
:0FD6890078037F102270039F11220B1480ED2273
:10D69800CAF87F20800A7E1BF07A2BF00B340B54DB
:10D6A80069FFFFFC7DEF1BE479EFFFFC4DFF78E697
:09D6B8007F102EF80000DAF822C0
:10D6C1007D437F1080071B447A0BB00B144D4478C7
:02D6D100F52240
:02FD6A00000097
:10D15D0074104D00780B4D2278278D317D126D2284
:10D16D00227D437D326D222F112D445002A50FBF1C
:10D17D001040049F100B901478ED7F016D227D34CB
:10D18D00227D417D138D247D022F004004BD04407E
:10D19D00049D040B141478F17D237D317D106D00F9
:01D1AD00225F
:0ED6D300BEB0304007BEB03A5002D322C32290
:08D6E1003098FDE599C2982282
:00000001FF
